:100000000C94560F0C94870F0C94870F0C94870F49
:100010000C94870F0C94870F0C94870F0C94870F08
:100020000C94870F0C94870F0C94870F0C94870FF8
:100030000C94870F0C94870F0C94870F0C94870FE8
:100040000C94870F0C94870F0C94870F0C94870FD8
:100050000C94870F0C94870F0C94870F0C94B39912
:100060000C94870F0C942B740C9401740C94870FD0
:100070000C94870F0C94870F0C94870F0C94870FA8
:100080000C94870F0C94870F0C94870F0C94870F98
:100090000C94870F0C94870F0C94870F0C94A0225C
:1000A0000C94870F0C94870F0C94870F0C94870F78
:1000B0000C94870F0C94870F0C94870F0C94870F68
:1000C0000C94870F0C94870F0C94870F0C94870F58
:1000D0000C94870F0C94870F0C94870F0C94870F48
:1000E0000C94870F07634236B79BD8A71A39685616
:1000F00018AEBAAB558C1D3CB7CC5763BD6DEDFD4A
:10010000753EF6177231BF000000803F0800000006
:10011000BE922449123EABAAAA2ABECDCCCC4C3EFC
:1001200000000080BEABAAAAAA3E00000000BF00EB
:100130000000803F0000000000084178D3BB4387E7
:10014000D1133D190E3CC3BD4282AD2B3E68EC82FB
:1001500076BED98FE1A93E4C80EFFFBE01C4FF7F80
:100160003F00000000000C94A1120C94FF1C0C94A2
:10017000646B0C94910F0C9431680C94D51E0C9404
:1001800024580C94DF960C94C1950C9477120C941F
:100190004A760C94EB3F0C943C500C9457850C948D
:1001A00048310C949E970C9487900C94CA460C94FA
:1001B000E8120C9438100C948E100C94B96D0C94B9
:1001C000ED110C94A10F0C94C1690C9402140C94C1
:1001D000D10F0C9405510C94CB6B0C94E5110C943D
:1001E00003470C94AD790C94C3160C943A340C94D8
:1001F00072500C94F16D0C94B5750C9467690C9465
:10020000153C0C9481140C9447510C94B52B0C9410
:10021000F4110C94BE0F0C941F400C9437100C94E6
:1002200011190C9426310C944F6C0C9459300C9489
:1002300023160C9471320C946E310C94AD110C9405
:10024000A80F0C945C460C94714C0C94DC300C940C
:10025000B7180C9472300C94376C0C945F6A0C9441
:1002600054900C94EBA50C94EC500C949E750C944B
:10027000071C0C9458310C949B2C0C94E7300C9474
:10028000C7310C94CD110C948F130C94CC790C9431
:10029000B96B0C94D9580C94E5A50C9482900C94ED
:1002A00082510C94462B0C9439970C9419310C9470
:1002B00084310C94890F0C945D900C94BFA80C941D
:1002C00011470C94323C0C9447B00C9492AA0C94B5
:1002D00092A10C94F4460C942C610C9404790C9427
:1002E0004C900C9400850C943D850C94DC960C94F9
:1002F000F7240C9472440C9424300C949B6C0C9452
:100300001A850C94C22E0C94896A0C94363F0C9476
:10031000C90F0C94822B0C94FF750C9479900C945B
:10032000E5960C942A690C9407850C9442600C9411
:10033000A03F0C94D20F0C94503C0C94993C0C941C
:100340000E470C94F3140C949EAB0C941A1C0C9452
:1003500089690C94381D0C9475900C941E850C942E
:10036000806A0C94EEB00C9498970C94C9AF0C94DE
:10037000772F0C9436100C9495750C947D900C94FA
:1003800040970C94ABA30C941B730C94176C0C94B7
:10039000806B0C94AF120C9455B00C94126B0C94AF
:1003A0008E110C940E6A0C94743C0C947F110C9476
:1003B00050900C94802C0C94DD460C94C33F0C940C
:1003C00097120C94F6790C94276E0C945E120C9490
:1003D000F96A0C9465120C941D470C941B2C0C9418
:1003E00061900C94E81B0C947B690C9403320C9480
:1003F000EB190C94D3B00C94796A0C948D770C940F
:100400007D140C945A100C94B72C0C94762B0C94ED
:10041000611E0C9469510C9447100C94DC3F0C94B1
:100420001F460C94A7190C94AD310C94B8120C947F
:10043000016C0C94682F0C9468800C941C130C9421
:1004400017140C94C56C0C946B900C948B500C94FA
:1004500057900C9484750C94BF500C9436520C94A5
:1004600029350C9428310C946F900C94EE310C9437
:10047000B3120C9412520C94D6110C942B690C9458
:10048000A1970C94A41D0C9442900C94744B0C9462
:1004900041B00C94F40F0C94695E0C94DD180C942C
:1004A000A4310C94D9310C94FD300C9421160C9489
:1004B000836A0C9418690C948D110C94862F0C94FB
:1004C00004320C94F20F0C94CA180C94A8110C94DA
:1004D0000F520C9452600C948F6B0C94E2600C944D
:1004E0009B140C946A2B0C940A2D0C94DD140C9420
:1004F000B5120C94312C0C9467900C943A320C94F5
:10050000995D0C94B6460C94B7510C9448900C9499
:1005100000470C943F300C94612F0C945A140C94A7
:10052000D26B0C94C66A0C9491320C946E2F0C947E
:10053000E7310C9438320C9406500C94B5B20C94FC
:10054000E80F0C94783F0C9458690C94976D0C94B8
:1005500015520C9476B00C9411760C9461100C9496
:1005600083900C949B970C94F83F0C94A6970C9452
:100570005C300C94FCB00C94F3310C948D0F6364DC
:10058000696E6F70737578585B002F00496E3A2062
:10059000003D00494E3A003D004C4547414359203B
:1005A000494E3A00000020002300260029002C00BC
:1005B0002F003200000100000301060109012D3E59
:1005C00000200023002D3E00200050656E6465640D
:1005D0003A2023007261770076616C0074656D705B
:1005E00000736174006875650066616E0052474271
:1005F00000485356006D6F646500536574436D6425
:100600003A0053746F726564204558543A0073750C
:1006100066666978436F64653A00584F4E004841FA
:100620004C54002074696D653A004374726C20521A
:1006300065733A002054533A0020543A003D00506C
:10064000696E3A004F4E3A416C726561647920419F
:1006500063746976650A0048414C543A416C72658E
:1006600061647920496E6163746976650A00584F48
:100670004E3A416C726561647920416374697665B4
:100680000A00584F464620736B69707065642E20CF
:100690005072657620636D643A005475726E6564BD
:1006A000206F66662066726F6D3A00526573746FD4
:1006B0007265642066726F6D3A0049676E6F72658D
:1006C000642C206368616E6E656C20636D643D0010
:1006D00020457865633A004163746976653A00485D
:1006E000414C543A416C726561647920496E616392
:1006F000746976650A00584F4E3A416C72656164C0
:1007000079204163746976650A00584F4646207324
:100710006B69707065642E205072657620636D641D
:100720003A005475726E6564206F66662066726F5B
:100730006D3A00526573746F7265642066726F6DF6
:100740003A004E6F7420656E6F756768206D656D39
:100750006F727920666F722067726F7570206F708C
:1007600065726174696F6E00206D73203A0041728A
:100770006D656420666F7220002044697361726D3C
:10078000656400536B697070656420686F6D69659E
:10079000207374756666004F75744F664D656D6F96
:1007A0007279210A0020436D643A00205375623D3E
:1007B00000204974656D3D0052414D3D00282D29B2
:1007C0002000282B2920002076616C756520697334
:1007D000200020756E6B6E6F776E0A005D3D005BCA
:1007E0000020696E76616C6964002000206F6B00E8
:1007F0003A00206661696C6564003A005265747263
:1008000079696E67206D6F6462757320434D440A89
:1008100000207365632072656D61696E696E6700A3
:100820005374617475732064656666657265640AE5
:100830000020002D3E00436F6E76657274696E670E
:1008400020002D3E0057726F6E67204173736967F9
:100850006E6D656E742000524742783A200048530E
:10086000562064697361626C65640020764C65761D
:10087000656C3A0020436F6E76563A0020436F6EE7
:1008800076533A0020486F743A00436F6C643A0024
:1008900020436F6E76657274656420563A00436F2C
:1008A0006E76657274656420533A002D3E0057726F
:1008B0006F6E672041737369676E6D656E7420009B
:1008C0002D3E0057726F6E672041737369676E6DBE
:1008D000656E74200053617665643A002053756636
:1008E000663A002041543A00436F6E6669672063A0
:1008F00068616E676564206C6F63616C6C792C2035
:10090000706F7274616C2064697361626C656400FD
:100910002F636F6E6669672E6A736F6E0072656211
:100920006F6F742000436D643A20002F636F6D6D0C
:10093000616E642F002F72616D2F002F6974656DD9
:100940002F002F6974656D2F004C6F636174696FA0
:100950006E3A20687474703A2F2F6C617A79686FE0
:100960006D652E72752F707761003F6D61633D007C
:100970002669703D0026706F72743D00266E616DB1
:10098000653D002F002000436F6D706C6574652E0F
:100990002052656D6F766520746F70696320002446
:1009A000636F6D6D616E6400536B697070696E6723
:1009B0002E2E00436C65616E5570207265746169FE
:1009C0006E656420746F70696320004F75744F66A4
:1009D0004D656D6F727921005D20003A5B000A0061
:1009E0003A004D41433A00554450205379736C6F9F
:1009F0006720696E697469616C697A65642E0A00A2
:100A00005379736C6F6720706172616D733A003E49
:100A1000003C00543A0043757272656E74204C417C
:100A20004E20636F6E6669672869702C646E732C44
:100A300067772C7375626E6574293A000A55736581
:100A400020746865736520636F6D6D616E64733AC1
:100A5000202768656C7027202D20746869732074C6
:100A60006578740A276D61632064653A61643A624F
:100A7000653A65663A66653A3030272073657420BA
:100A8000616E642073746F7265204D41432D616403
:100A9000647265737320696E20454550524F4D0A4C
:100AA000276970205B69705B2C646E735B2C6777C1
:100AB0005B2C7375626E65745D5D5D5D27202D2016
:100AC000736574207374617469632049500A2773D5
:100AD00061766527202D20736176652063757272BB
:100AE000656E7420636F6E66696720696E204E566E
:100AF00052414D3B204F4E7C4F4646202D20656E87
:100B000061626C652F64697361626C6520617574E4
:100B10006F736176650A2767657427205B636F6E64
:100B200066696720616464725D27202D20676574A3
:100B300020636F6E6669672066726F6D20707265E4
:100B40002D636F6E666967757265642055524C201F
:100B5000616E642073746F726520616464722C200E
:100B60004F4E7C4F4646202D20656E61626C652F8E
:100B700064697361626C6520646F776E6C6F616429
:100B8000206F6E20737461727475700A276C6F61C8
:100B90006427202D206C6F616420636F6E66696727
:100BA0002066726F6D204E5652414D0A2770776451
:100BB00027202D20646566696E6520616E64207350
:100BC000746F7265204D5154542070617373776F48
:100BD00072640A276F746170776427202D20646522
:100BE00066696E6520616E642073746F726520485B
:100BF000545450204150492070617373776F726470
:100C00000A276C6F67205B73657269616C5F6C6F3C
:100C1000676C6576656C5D205B7564705F6C6F6793
:100C20006C6576656C5D27202D20646566696E6550
:100C3000206C6F67206C6576656C2028302E2E370F
:100C4000290A276B696C6C27202D2074657374202A
:100C50007761746368646F670A27636C65617227E4
:100C6000202D20636C65617220454550524F4D0A1E
:100C7000277265626F6F7427202D207265626F6F17
:100C80007420636F6E74726F6C6C657200536F6664
:100C900074207265626F6F74696E672E2E2E00521B
:100CA000414D3D000A5379736C6F6720000A312D66
:100CB0007769726520000A6D71747420000A696E8C
:100CC0007075747320000A6974656D7320000A439F
:100CD0006F6E666967757265643A0020416464727C
:100CE0003A00646576230009445332343832206573
:100CF00072726F720009526573657420646F6E655D
:100D00000009436865636B696E6720666F72203106
:100D10002D5769726520646576696365732E2E2E82
:100D2000004453323438322D3130302070726573C4
:100D3000656E74004572726F7220312D7720696E76
:100D4000697420233220467265653A0077737461B6
:100D5000742E20467265653A005465726D2E2046E9
:100D60007265653A004572726F7220312D77206985
:100D70006E697420233100467265653A004453322F
:100D80003438325F3130305F4932435F544F5F3126
:100D9000575F42524944474520696E6974003B00E1
:100DA0003D0050696E3A003B003D4C4F570054687F
:100DB00065726D6F3A004F6E6520776972652052DB
:100DC000656164790A004170706C79696E672063AF
:100DD0006F6E666967004C6F6164656420455441BD
:100DE000473A004E6F2073746F72656420636F6EB4
:100DF000666967004C6F616465642066726F6D2080
:100E0000454550524F4D006C6F6164206661696CBE
:100E10006564004C6F6164696E6720436F6E66693C
:100E2000672066726F6D20454550524F4D00436FED
:100E30006E666967206175746F736176653A000A42
:100E40005379736C6F67206465627567206C657693
:100E5000656C3A0053657269616C20646562756700
:100E6000206C6576656C3A0053617665640A0053C0
:100E700065742064796E616D69632049500A00458C
:100E80004550524F4D20636C65617265640A004D98
:100E90005154542050617373776F7264207570647D
:100EA000617465640A004F54412050617373776F19
:100EB000726420757064617465640A00636F756C98
:100EC00064206E6F742070617273653A20005570F3
:100ED00064617465640A004E6F2049502061647239
:100EE0006573730052656C656173696E6720736F1B
:100EF000636B657420616E64207265747279002082
:100F00005361766564004C6F6164696E6720485474
:100F1000545020636F6E666967206F6E2073746132
:100F2000727475703A004F4646004F4E002B002DEC
:100F300000455461673A2000476574204554414795
:100F40003A2000485454502F312E31202569002575
:100F5000733A2025730D0A0020485454502F312E27
:100F6000310D0A486F73743A2025730D0A4163638B
:100F70006570743A202A2F2A0D0A436F6E6E6563DE
:100F800074696F6E3A20636C6F73650D0A00257388
:100F90000020000D0A00474554006661696C6564D5
:100FA00020746F20636F6E6E6563740A0045525241
:100FB0004F523A205365727665722072657475726D
:100FC0006E65642000436F6E666967206E6F7420E3
:100FD0006368616E6765640A00446F6E652E0A007F
:100FE000436F6E6669672070617273696E67206611
:100FF00061696C65640A00676F7420436F6E66698F
:10100000670A00667265652000436F6E6669672037
:101010005552493A20687474703A2F2F0020446565
:101020006661756C7420636F6E66696720736572A4
:1010300076657220757365643A20006C617A796810
:101040006F6D652E7275000A282D294D554C544937
:1010500056454E54000A282B2950574D5F52454C97
:101060004159000A282D294D444E53000A282D29A4
:1010700055415254425249444745000A282B2953AE
:1010800059534C4F47000A282D29504944000A283B
:101090002D294D43503233303137000A282D294154
:1010A00052544E4554000A282B294F5441000A2817
:1010B0002D29535049204C4544000A282D294D4FD5
:1010C000544F5220435452000A282D2941432048AE
:1010D00041494552000A282D2943435338313120D4
:1010E000262048444331303830000A282B29524505
:1010F00053544152545F4C414E5F4F4E5F4D5154DB
:10110000545F4552524F5253000A282D29484152EC
:101110004452455345542C207573696E6720736F94
:101120006674000A282D29434F554E544552000A33
:10113000282D29444854000A282B29445332343896
:10114000322D313030000A282B294F5749524500A3
:101150000A282D294D4F44425553000A282D294471
:101160004D58000A282B2957697A6E65743531303D
:1011700030000A282B294672656552616D20707215
:10118000696E74696E67000A282B295741544348D9
:10119000444F47000A4669726D77617265204D4180
:1011A0004320416464726573732064653A61643AF4
:1011B00062653A65663A66653A6566006C617A7999
:1011C000686F6D652E7275000A436F6E66696720E1
:1011D0007365727665723A003230313130334C00CB
:1011E00020432B2B2076657273696F6E3A00333281
:1011F00065376462645F323032322D30322D3134E3
:10120000000A4C617A79686F6D652E7275204C69A1
:1012100067687448756220636F6E74726F6C6C657A
:10122000722000204F464600204F4E002042595069
:1012300041535300757074696D6500667265656829
:10124000656170002054696D65723A00204C6F63CF
:101250006B733A002000204C6F636B733A000A52A4
:10126000414D3D0020457870697265640A00202D6B
:10127000746172676574207A6F6E652D0020416C11
:1012800061726D20457870697265640A0020636D33
:10129000643A00204375723A00205365743A005353
:1012A0006176656420746F20454550524F4D005360
:1012B0006176696E6720636F6E66696720746F2060
:1012C000454550524F4D2E2E002069732000446535
:1012D0006C6574696E6720636F6E662E2052414D97
:1012E000207761733A0053746F70706564005374B3
:1012F0006F7070696E67206368616E6E656C7320D5
:101300002E2E2E004E6F7420756E6C6F636B6564AD
:1013100020696E20313073202D20636F6E74696EEA
:101320007565202E2E2E00556E6C6F636B696E678F
:1013300020636F6E666967202E2E2E0020696E690D
:10134000740052656C61792D4F75742023002073F1
:10135000746F700052656C61792D4F757420230095
:101360003D3E003A0070756220616374696F6E20C3
:101370000069646C65006F66660068656174696E1B
:10138000670066616E00647279696E6700636F6FF3
:101390006C696E670020697320004F7574200055DA
:1013A0006E6B6E6F776E2073756666697820005578
:1013B0006E6B6E6F776E20636D642000616374697D
:1013C0006F6E0072656C61794374723A200020413F
:1013D0006464723A00646576230020616C69766506
:1013E00000204E6F64653A00312D77697265206385
:1013F0006F756E743A2000312D77697265207368BD
:101400006F72746564005B305D3A2000202D202DE2
:10141000202D20EFBBBF003E003E31202D200020BC
:10142000002E00696E00735F6F7574006D79686FD0
:101430006D6500202D3E2000456D69743A20002026
:101440002D3E20004974656D436D643A2000202DC7
:101450003E20004974656D3A2000005EBCE2613FA9
:10146000DD83C29C7E20A3FD1F419DC3217FFCA282
:10147000401E5F01E3BD3E6082DC237D9FC1421CB4
:10148000FEA0E1BF5D0380DE3C62BEE0025CDF8166
:10149000633D7C22C09E1D43A1FF4618FAA4277914
:1014A0009BC584DA3866E5BB5907DB856739BAE442
:1014B00006581947A5FB7826C49A653BD987045A74
:1014C000B8E6A7F91B45C6987A24F8A6441A99C726
:1014D000257B3A6486D85B05E7B98CD2306EEDB3D4
:1014E000510F4E10F2AC2F7193CD114FADF3702E02
:1014F000CC92D38D6F31B2EC0E50AFF1134DCE9034
:10150000722C6D33D18F0C52B0EE326C8ED0530DE5
:10151000EFB1F0AE4C1291CF2D73CA947628ABF593
:1015200017490856B4EA6937D58B5709EBB53668C1
:101530008AD495CB2977F4AA4816E9B7550B88D6F3
:10154000346A2B7597C94A14F6A8742AC896154BA5
:10155000A9F7B6E80A54D7896B35436F6E6E656399
:101560007465642E00436F6E6E2E2061626F72741C
:101570006564003E3E2000496E76616C69642063BC
:101580006F6D6D616E64003E3E3E004E6F204D41BA
:101590004320636F6E666967757265643A20736590
:1015A00074206669726D776172652773204D4143BF
:1015B0000A004E6F2076616C696420454550524F99
:1015C0004D20646174612E20496E697469616C6993
:1015D0007A696E672E00476F7420495020616464F9
:1015E000726573733A00276970205B69705B2C64C5
:1015F0006E735B2C67775B2C7375626E65745D5DD3
:101600005D5D27202D207365742073746174696398
:101610002049500A004661696C656420746F20633C
:101620006F6E6669677572652045746865726E6570
:1016300074207573696E6720444843502E20596F9B
:10164000752063616E20736574206970206D616E12
:1016500075616C6C7921000A757365732044484389
:10166000500A00204D41534B3A002047573A002082
:10167000444E533A004C6F616465642066726F6D2E
:1016800020666C6173682049503A0053746172742B
:10169000696E67206C616E0041424344454647488D
:1016A000494A4B4C4D4E4F50515253545556575832
:1016B000595A6162636465666768696A6B6C6D6ECE
:1016C0006F707172737475767778797A30313233DE
:1016D0003435363738392B2F3D004261736963202A
:1016E0000061726475696E6F3A004F544120696EF3
:1016F000697469616C697A65640A004445464155BC
:101700004C542070617373776F726420666F72201F
:101710004F5441204150492E20557365206F74610C
:1017200070776420636F6D6D616E6420746F2073D9
:1017300065740070617373776F726400757074699B
:101740006D652C66726565686561700024737461EF
:10175000747300333265376462645F323032322D25
:1017600030322D3134004C6967687448756220004E
:10177000246E616D6500726561647900546F6F203D
:101780006D616E79204D51545420636F6E6E6563A8
:1017900074696F6E206572726F72732E205265735A
:1017A00074617274204C414E00207472792061671C
:1017B00061696E20696E2035207365636F6E647396
:1017C000006661696C65642C2072633D004177613D
:1017D0006974696E6720666F722072657461696EE4
:1017E000656420746F7069637300636F6E6E656308
:1017F0007465642061732000202E2E2E00207573E6
:1018000065723A003A000A417474656D7074696ECD
:1018100067204D51545420636F6E6E656374696F19
:101820006E20746F200024737461746500646973A2
:10183000636F6E6E6563746564005573696E6720CF
:101840004D5154542070617373776F7264206672C7
:101850006F6D20636F6E66696700446576696365C6
:10186000204E616D653A004174206C65617374208F
:10187000646576696365206E616D6520616E6420C4
:1018800062726F6B6572204950206D7573742062AF
:101890006520636F6E666967757265640052656284
:1018A000696E6420737563636573732E20495020DD
:1018B000616464726573733A004572726F723A20A4
:1018C000726562696E64206661696C0052656E655E
:1018D00077656420737563636573732E20495020A8
:1018E000616464726573733A004572726F723A2074
:1018F00072656E65776564206661696C000A4E6F7B
:10190000206C696E6B00526573746F72696E67202C
:10191000636F6E6669672066726F6D204545505231
:101920004F4D00416363657074696E6720636F6D2E
:101930006D616E64732E2E2E0A004E6F204D515431
:101940005420636F6E66696775726564004C6F61E1
:1019500064696E6720636F6E6669672066726F6D7B
:1019600020706F7274616C2064697361626C65646D
:101970002E2075736520676574204F4E20746F208C
:10198000656E61626C6500436F6E6669672069739E
:101990002076616C696400436F6E74696E756520B2
:1019A000776974682070726576696F75736C7920D9
:1019B0006C6F6164656420636F6E66696700000028
:1019C0002200250028002B002E00310034000201E7
:1019D0000000050108010B0100000A0B02090C0DB3
:1019E0000E080703040100000000000000000000D2
:1019F00000000000000000000000000000000000E7
:101A000000000000121110000000000000000000A3
:101A100000000000000000000000000000000000C6
:101A20002100240027002A002D003000330001018E
:101A30000000040107010A0101021020200808101B
:101A4000204010204080020102010804020101022E
:101A50000408102040808040201008040201800407
:101A60000201804020100804020108040201010262
:101A70000408102040800102040810204080050561
:101A80000505070508080808020202020A0A0808F4
:101A90000404040401010101010101010303030322
:101AA00003030303040707070C0C0C0C0C0C0C0CB1
:101AB0000202020206060606060606060B0B0B0BC2
:101AC0000B0B0B0B2F64617461002F736B657463D8
:101AD00068004163636573732D436F6E74726F6C3E
:101AE0002D416C6C6F772D486561646572733A2087
:101AF000436F6E74656E742D747970652C436F6ED0
:101B00006E656374696F6E2C417574686F72697A63
:101B10006174696F6E2C507261676D61004163631F
:101B20006573732D436F6E74726F6C2D416C6C6FA7
:101B3000772D4D6574686F64733A20504F53542C61
:101B40004745542C4F5054494F4E530041636365F1
:101B500073732D436F6E74726F6C2D416C6C6F7765
:101B60002D43726564656E7469616C733A2074729A
:101B70007565004F5054494F4E530044454C4554F1
:101B800045005055540047455400504F5354006190
:101B90007574686F72697A6174696F6E3A2000417A
:101BA0007574686F72697A6174696F6E3A20004368
:101BB0006F6E74656E742D4C656E6774683A2000A4
:101BC0006F637465742F73747265616D00696D6104
:101BD00067652F6A70656700696D6167652F676962
:101BE0006600746578742F68746D6C006170706C39
:101BF00069636174696F6E2F6A736F6E00746578C4
:101C0000742F706C61696E00436F6E74656E742D15
:101C1000547970653A2000436F6E6E656374696F26
:101C20006E3A20636C6F7365004163636573732D57
:101C3000436F6E74726F6C2D416C6C6F772D4F72A9
:101C40006967696E3A20687474703A2F2F6C617AF4
:101C500079686F6D652E727500556E6B6E6F776E5D
:101C6000004F4B004D6F766564207065726D616E3C
:101C7000656E746C7900496E7465726E616C205388
:101C80006572766572204572726F72005061796C70
:101C90006F616420546F6F204C61726765004E6FF6
:101CA0007420666F756E64005757572D41757468C0
:101CB000656E7469636174653A204261736963207B
:101CC0007265616C6D3D224163636573732072655B
:101CD00073747269637465642200556E617574680B
:101CE0006F72697A6564005061796C6F616420730A
:101CF000697A652077726F6E670042616420726551
:101D0000717565737400485454502F312E31200082
:101D100020000000000000000000004F4E00000006
:101D2000000000004F4646000000000000524553EE
:101D3000540000000000544F47474C450000004845
:101D4000414C540000000000584F4E0000000000BD
:101D500000584F46460000000000494E435245419E
:101D6000534500444543524541534500484541547D
:101D70000000000000434F4F4C00000000004155A0
:101D8000544F000000000046414E5F4F4E4C59003A
:101D900044525900000000000053544F500000000E
:101DA00000004849474800000000004D454449559F
:101DB0004D0000004C4F57000000000000545255E9
:101DC00045000000000046414C534500000000451E
:101DD0004E41424C4544000044495341424C454425
:101DE0000052474200000000000048535600000027
:101DF00000000057726F6E67207061796C6164003B
:101E0000202D3E2041543A004368616E2074797061
:101E1000653A004E6F2073746F7265642076616C52
:101E2000756573202D2064656661756C743A2000B9
:101E30002D3E005075623A2000636D640046414EAD
:101E40005F4F4E4C590044525900434F4F4C00488D
:101E5000454154004155544F002D3E005075623AA3
:101E600020007365740064656C002D3E005075623F
:101E70003A20002D3E005075623A2000556E6B6E80
:101E80006F776E20636D64200A004F4646004F4E08
:101E900000536176656420455441473A00536574A8
:101EA00020455441473A2000B5B292A111241FBEEB
:101EB000CFEFD1E2DEBFCDBF00E00CBF15E0A0E068
:101EC000B2E0E4E0FEE801E00BBF02C007900D9233
:101ED000A639B107D9F72AE0A6E9B5E001C01D92FD
:101EE000AD36B207E1F71FE0C5E5DFE000E006C070
:101EF00021970109802FFE010E94B8C1C435D10786
:101F000080E00807A9F70E94A4A10C94F0C60C94E5
:101F10000000FC01818D928D0895FC0184899589D2
:101F2000089525EA33E0FC0131832083FB014089D9
:101F3000518962897389FC01428353836483758369
:101F40000895DC01ED91FC91048CF58DE02D199440
:101F5000CF93DF931F92CDB7DEB76983DC01ED919C
:101F6000FC910280F381E02D41E050E0BE016F5F03
:101F70007F4F19950F90DF91CF910895FC019485C3
:101F8000FB018485981303C081E0943009F480E05C
:101F9000089521E0FC018485843009F420E0822F3B
:101FA00008950895CF93DF931F92CDB7DEB769836D
:101FB000DC01ED91FC910280F381E02D41E050E0E5
:101FC000BE016F5F7F4F19950F90DF91CF910895FC
:101FD000DC01ED91FC91068CF78DE02D199591E0D7
:101FE00089270895862F089581E086270895DC01CA
:101FF00080E0615038F0ED91E827F0E0E65AFB4EC2
:102000008491F7CF0895FC01818191E09093DA07E4
:102010008093FC071092DB071092FD070895209132
:102020003F06260F3327331F21323105ECF4209170
:10203000D407FC0190E080E0243069F082E008954C
:10204000A0913F062191AC01435E594FA40FB52FDB
:10205000B11D2C930196861798F380913F06680F67
:1020600060933F0680E0089581E008950895089503
:10207000E091650680916406E81730F4F0E0EA59D3
:10208000F94F808190E008958FEF9FEF0895909130
:102090006506809164062FEF3FEF981748F4E92F0B
:1020A000F0E0EA59F94F208130E09F5F9093650698
:1020B000C90108958091640690916506891B990B6A
:1020C0000895CF92DF92EF92FF920F931F93CF93D9
:1020D000DF937C01CB018A012091DA07222389F06A
:1020E000EB016B01C40ED51ECC15DD0569F06991BD
:1020F000D701ED91FC910190F081E02DC701199578
:10210000F3CF642F0E940F10C801DF91CF911F9170
:102110000F91FF90EF90DF90CF900895CF93DF93D2
:102120001F92CDB7DEB769832091DA072223F9F039
:102130002091FD07203258F021E030E0FC0133838C
:10214000228390E080E00F90DF91CF9108958091FD
:10215000DB07E82FF0E0E452F84F998190838F5F1E
:102160008093DB078093FD0781E090E0ECCF61E096
:10217000CE0101960E940F10F7CF8F929F92AF92DF
:10218000BF92CF92DF92EF92FF920F931F93CF9364
:10219000DF9300D000D000D01F921F92CDB7DEB7E2
:1021A0007C018E010F5F1F4F68018AE0882E912C01
:1021B000A12CB12CC601801B910B41155105610565
:1021C000710581F0CB01BA01A50194010E942DC1D6
:1021D000942F852F605DF60161936F01A901692F2E
:1021E000782FE8CFF801E80FF91FD7010150110946
:1021F00022912D93E017F107D9F7E80EF91EF701A8
:1022000010822B960FB6F894DEBF0FBECDBFDF91C4
:10221000CF911F910F91FF90EF90DF90CF90BF90E3
:10222000AF909F908F900895FC01DC018D918111FA
:10223000FDCF30E020E050E040E08AE0919199232A
:1022400001F1443051055CF59E3271F42F3F3105A8
:1022500009F02CF5DB01A40FB51F12962C934F5FEC
:102260005F4F30E020E0EACF829FD001839FB00D26
:102270001124292F990F330B205331092A0F3B1FAB
:10228000DDCF2F3F310509F054F4443051053CF4C3
:10229000640F751FFB01228381E090E0089590E0B8
:1022A00080E00895CF93DF931F921F92CDB7DEB7E2
:1022B0008091610A9091620A009711F48DE69AE08C
:1022C000BE016F5F7F4F681B790B072E000C880BD8
:1022D000990B0F900F90DF91CF9108959FE9980F80
:1022E000963010F4875508959FEB980F963010F4B0
:1022F0008753089580538A3008F080E00895DC0108
:1023000015968D919C91009739F0DC01ED91FC912F
:102310000680F781E02D19940895089583E090E0F8
:10232000089590E0FC01E258F54EE491F0E0EE0FE4
:10233000FF1FE254F64EA591B4912C91885C954E06
:10234000FC018491822391E009F490E0892F0895A3
:102350008091B5059091B6050895FC018481958121
:102360000895DC011196EC911197E295EF70E15020
:10237000EB3008F039C0F0E08827EE53FE4E8F4F67
:102380000C94B8C1E511E511F411CD11CD11D611A0
:10239000ED11ED11ED11CD11CD1114966D917D91D1
:1023A0008D919C9117970E94EABF089514966D91A4
:1023B0007D918D919C9117972AE030E040E050E0AC
:1023C0000E944FC1CA01B901EECF14966C9170E022
:1023D00090E080E00E94E8BF089514966D917D9191
:1023E0008D919C911797089560E070E0CB0108955E
:1023F000FC01A7812A2F2E7FD1F0818182958F70D9
:1024000081508330A0F4A695A150BB0B2BE531E0A1
:102410000E94CFC124E630E040E050E00E944FC16E
:10242000DA01C90187569F4FAF4FBF4F08958FEF15
:102430009FEF0895DC01ED91FC91309729F0908594
:102440009F7081E0953009F080E00895FC01A4813F
:10245000B581109721F118969C9118979F708EEF77
:10246000890F823010F091111AC019964D935D9327
:102470006D937C931C97A481B58118969C911897B5
:10248000907F926018969C930480F581E02D808562
:10249000982F907F903619F48F70806A8087089506
:1024A000DC0119968D919C91009739F0DC01ED913A
:1024B000FC910280F381E02D19940895DC01ED91E7
:1024C000FC91008CF18DE02D1994CF93DF93EC01FA
:1024D000E881F9810484F585E02D199529893A89E7
:1024E0002F5F3F4F3A8B298BDF91CF910895CF9388
:1024F000DF93EC018E8581110DC081E090E0498968
:102500005A892C853D854217530708F080E0DF91FA
:10251000CF910895E881F9810484F585E02DCE01FD
:1025200019958F3F910549F780E090E0F0CFFC01CD
:10253000848595856817790708F4CB01928B818B88
:102540000895DC011E962C911E97222339F0ED91FF
:10255000FC910190F081E02D6FEF19940895FC013A
:1025600087859089089581E0089590E080E008953E
:10257000CF93DF93CDB7DEB760970FB6F894DEBF89
:102580000FBECDBF19821A821B821C821D821E8241
:102590001F8218868A818F7080618A836FEF3E81E7
:1025A0009F81888529817A815B814C814C873E8718
:1025B000888B372F452F5C857E85892F988960967B
:1025C0000FB6F894DEBF0FBECDBFDF91CF91089557
:1025D000CF92DF92EF92FF920F931F93CF93DF93EF
:1025E000CDB7DEB760970FB6F894DEBF0FBECDBF94
:1025F0007C016B01BA01A901CE0101960E94BD10B8
:10260000D701ED91FC910288F389E02D9801AE018C
:102610004F5F5F4FB601C701199560960FB6F894EA
:10262000DEBF0FBECDBFDF91CF911F910F91FF9005
:10263000EF90DF90CF900895CF92DF92EF92FF92CC
:102640000F931F93CF93DF93CDB7DEB7AF970FB63E
:10265000F894DEBF0FBECDBF7C016A0105EA13E02E
:102660001A8309831C861B8688EE93E0A0E0B0E005
:102670008D879E87AF87B88B8DE793E09A87898790
:10268000188F0F8B198E1A8E1B8E1C8E84E089A3D7
:102690001BA70AA71CA61DA61EA61FA680912D0873
:1026A00090912E08A0912F08B09130088EA39FA37F
:1026B000A8A7B9A78B839C83AD83BE8318861F828E
:1026C000AE01465D5F4FCE0101960E94507A813087
:1026D0009105B1F4D701ED91FC910488F589E02DC5
:1026E0001DA30CA38CA59DA5AEA5BFA58EA39FA3DE
:1026F000A8A7B9A7A601BE016C5D7F4FC7011995B8
:10270000AF960FB6F894DEBF0FBECDBFDF91CF916D
:102710001F910F91FF90EF90DF90CF900895CF928F
:10272000DF92EF92FF920F931F93CF93DF93CDB77A
:10273000DEB7AF970FB6F894DEBF0FBECDBF7C01FA
:102740006A0105EA13E01A8309831C861B8688EE5A
:1027500093E0A0E0B0E08D879E87AF87B88B8DE7D0
:1027600093E09A878987188F0F8B198E1A8E1B8E8C
:102770001C8E84E089A31BA70AA71CA61DA61EA663
:102780001FA680912D0890912E08A0912F08B0913E
:1027900030088EA39FA3A8A7B9A78B839C83AD8382
:1027A000BE8318861F82AE01465D5F4FCE01019643
:1027B0000E94507A81309105B1F4D701ED91FC91DE
:1027C0000684F785E02D1DA30CA38CA59DA5AEA5C1
:1027D000BFA58EA39FA3A8A7B9A7A601BE016C5D44
:1027E0007F4FC7011995AF960FB6F894DEBF0FBEA5
:1027F000CDBFDF91CF911F910F91FF90EF90DF90B0
:10280000CF900895CF93DF93EC01888D843061F0F1
:102810000E941680E88DF0E0EE0FFF1FE157F94FA0
:102820001182108284E0888FDF91CF910895EF921A
:10283000FF921F93CF93DF93FC01208D243039F05A
:1028400080E0DF91CF911F91FF90EF9008957B0181
:10285000EC0110E0812F0E94D98081110FC0188FE8
:10286000888D843069F3FD86EC861A8E198E20E0FF
:10287000A70162E00E942A8081E0E3CF883179F3EA
:102880001F5F143039F7ECCFCF93C82F0E946F949D
:1028900004C09695879577956795CA95D2F7611587
:1028A00071058105910521F461E070E080E090E020
:1028B000CF9108950F931F93CF93DF931F92CDB7BE
:1028C000DEB78C01DC01ED91FC910084F185E02DF7
:1028D0001995892B79F0BE016F5F7F4FF8018485D0
:1028E0000E94DB78898190E00F90DF91CF911F915A
:1028F0000F9108958FEF9FEFF7CFFC0184850C9423
:102900003E79CF93DF931F92CDB7DEB741E050E021
:10291000BE016F5F7F4FFC0184850E943E791816CF
:10292000190634F4898190E00F90DF91CF910895DA
:102930008FEF9FEFF9CFFC018485843011F00C9468
:102940001C7990E080E00895CF93C62F0E94031079
:1029500061EE83E398E00E948E106C2F83E398E091
:102960000E948E10CF910C9427921092D40781E090
:102970008093D3071092AE0761E084E10E948B90B0
:1029800061E085E10E948B90E9EBF0E080818E7F31
:10299000808380818D7F808388E48093B80085E484
:1029A0008093BC0008956DE27FE0811102C06FE268
:1029B0007FE08FEB98E00C94BF736DE87CE08FEBC9
:1029C00098E00E94BF73F0E0E0E0199584EF91E099
:1029D000089562EC77E0811102C06DEB77E080E74B
:1029E00099E00C94BF734F925F926F927F92AF9277
:1029F000BF92DF92EF92FF920F931F93CF93DF93DB
:102A000000D000D0CDB7DEB77C01D62E809119065C
:102A1000882309F4BEC0D70114969C9180910402CA
:102A2000891708F4B6C08091170690911806BAE08D
:102A30006B13F0C089539A4FFC011082D70118968E
:102A40000D911C910115110509F49FC0F8016185D4
:102A500072856115710591F4458056806780708498
:102A60008091210890912208A0912308B091240818
:102A7000481659066A067B0609F487C0D8011B96DA
:102A80004D915C911C974115510509F47EC0F701E9
:102A9000248153968C91539790E0322F377002C067
:102AA000959587953A95E2F780FF6FC0A22EB12CDD
:102AB000C501887F9370892B39F451968D919C9133
:102AC000887F9370A82AB92AD8018D919C91DC0146
:102AD000ED91FC916115710509F486C00688F789AE
:102AE000E02D1995019709F050C06CE3F801808141
:102AF00091810E94CC72A50170E060E02AE0D801CB
:102B00008D919C910E947C72F8012281808191813B
:102B100069E174E1222311F067E174E10E94BF735F
:102B2000D8011D966D917C911E978D919C910E946C
:102B3000597360E2F801808191810E94CC72D801C2
:102B40001F966D917C9150978D919C910E94597325
:102B5000F8012281808191816CE074E1222311F0DF
:102B600066E074E10E94BF7367EC75E0D8018D9157
:102B70009C910E945973F80180819181DC01ED9153
:102B8000FC91008CF18DE02D199510921806109291
:102B90001706D70115968D919C911697009709F409
:102BA0004DC014963C9120910502231708F446C0AD
:102BB000DC01ED91FC910190F081E02D6D2D1995D6
:102BC00026960FB6F894DEBF0FBECDBFDF91CF9132
:102BD0001F910F91FF90EF90DF90BF90AF907F908B
:102BE0006F905F904F9008950488F589E02D25EA55
:102BF00033E03A832983D80115964D905D906D900E
:102C00007C9018974B825C826D827E82BE016F5FE2
:102C10007F4F67CF8F3491050CF0BBCFBDE06B17B2
:102C200009F4B7CF9C012F5F3F4F309318062093D4
:102C3000170689539A4FFC016083ABCF81E090E087
:102C4000BFCF0C94E7B5CF93C1E068EE73E080E0AE
:102C500090E00E942A926C2F8FEB98E00E94998955
:102C6000CF5FC43191F784EF91E0CF910895CF9376
:102C7000DF93009709F484C0FC012081222309F42A
:102C80007FC0EC0162E67EE10E9483B8892B09F4E3
:102C900056C069E37EE1CE010E9483B8892B09F416
:102CA00051C065EF75E0CE010E9483B8892B09F40D
:102CB0004CC061EF75E0CE010E9483B8892B09F406
:102CC00047C06DEE75E0CE010E9483B8892B09F4F0
:102CD00042C069EE75E0CE010E9483B8892BF1F104
:102CE00065EE75E0CE010E9483B8892BD1F161EECB
:102CF00075E0CE010E9483B8892BB1F16CED75E0CF
:102D0000CE010E9483B8892B91F168ED75E0CE0168
:102D10000E9483B8892B71F166E67EE1CE010E94A4
:102D200083B8892B51F164ED75E0CE010E9483B820
:102D3000892B31F58EE090E0DF91CF91089582E00C
:102D400090E0FACF81E090E0F7CF88E090E0F4CF18
:102D500085E090E0F1CF86E090E0EECF87E090E074
:102D6000EBCF89E090E0E8CF8AE090E0E5CF8BE020
:102D700090E0E2CF8CE090E0DFCF8DE090E0DCCF20
:102D800090E080E0D9CFCF93DF93EC0164E573E16D
:102D900080E799E00E94BF736C817D8180E799E0B4
:102DA0000E94A0896EE473E180E799E00E94BF73FE
:102DB00080E799E00E94C87260E08C810E94B9901F
:102DC0001092B6051092B50581E090E0DF91CF91A9
:102DD0000895EF92FF921F93CF93DF93192F7B01FA
:102DE000C82FD92FD7FF03C0D195C195D10961E074
:102DF0008C2F0E94B99082E0E816F10499F460E00B
:102E00008C2F0E948B906CE272E180E799E00E9427
:102E1000BF7380E799E0DF91CF911F91FF90EF9012
:102E20000C94C872612FEF2851F46095661F6627D5
:102E3000661F8C2F0E948B9068E272E1E6CF661FBE
:102E40006627661F8C2F0E948B9063E272E1DDCFB4
:102E5000CF93DF9300D000D01F921F92CDB7DEB783
:102E6000EAEAF8E0128A118A80E090E19587848787
:102E700084E890E0948B838B81E0868780E090E209
:102E8000908B87871C821B828DE792E09A838983CF
:102E9000FE83ED838FEF9FEF98878F836FEA72E158
:102EA0008FEB98E00E94BF736091B0057091B105FF
:102EB000CE0101960E9456758AEA98E00E945E1241
:102EC0006FE972E18FEB98E00E94BF738FEB98E09F
:102ED0000E94C8720E94FD9928960FB6F894DEBF32
:102EE0000FBECDBFDF91CF910895FC018681978100
:102EF000009799F0FC0120852F70223029F461851C
:102F00007285838594850895253039F460E00E94A8
:102F1000D484009711F0FC01F2CF60E070E0CB01A7
:102F20000895CF93DF93EB0163E0FC0180819181F1
:102F30000E94D484009761F0FC0120852F7022301C
:102F400039F4818592858C239D23DF91CF9108955B
:102F500090E080E0FACFCF93C62F63E0FC01808140
:102F600091810E94D484FC01892B19F19085892FCD
:102F70008D70F9F4907F9260908781859285A3850A
:102F8000B4858827AA27BB278C2B81879287A387A4
:102F9000B4876AEF75E080E799E00E94BF736C2FF9
:102FA00080E799E00E94998980E799E0CF910C949D
:102FB000C872CF91089563E0FC01808191810E94E5
:102FC000D484009719F0FC01818508958FEF08954E
:102FD000FF920F931F93CF93DF93CDB7DEB7649724
:102FE0000FB6F894DEBF0FBECDBF8C01F62E8FE278
:102FF00090E09A838983FE01339688E0DF011D9279
:103000008A95E9F7F8016681FF2011F081E06827D1
:10301000D80114968C910E948B90F801878190853D
:10302000A185B285883E9340A105B10508F48BC007
:103030006AE973E180E799E00E94BF73D8011496B2
:103040006D917C9180E799E00E94A08965E973E128
:1030500080E799E00E94BF736F2D70E080E799E0F0
:103060000E94A08980E799E00E94C8726CEB73E12E
:10307000CE0101960E9478B8F801828193810E9466
:10308000DB17FF2009F46BC062E873E18D3051F06B
:1030900066E873E18E3031F06DE873E18B3011F04A
:1030A0006AE773E1CE010B960E948CB865E673E186
:1030B00080E799E00E94BF73D8011296ED91FC91D0
:1030C00013970190F081E02D60817181ED91FC9169
:1030D0000288F389E02D9E012F5F3F4FAE01455FCF
:1030E0005F4FC8011995BC0180E799E00E94A08953
:1030F00063E673E180E799E00E94BF73D8011296FE
:10310000ED91FC910190F081E02D6081718180E76B
:1031100099E00E945973BE016F5F7F4F80E799E08D
:103120000E94597360E673E180E799E00E94BF73E3
:10313000BE01655F7F4F80E799E00E94597380E789
:1031400099E00E94C87264960FB6F894DEBF0FBE75
:10315000CDBFDF91CF911F910F91FF90089566E74A
:1031600073E1823009F49ECF61E773E19BCF892B35
:1031700071F0FB01828193810E948B8666EA7EE07A
:103180008FEB98E00E94BF7388EC90E0089590E088
:1031900080E0F2CF892B71F0FB01828193810E9444
:1031A00028866FE87EE08FEB98E00E94BF7388EC82
:1031B00090E0089590E080E0F2CF80919C0890919B
:1031C0009D08892B51F00E94279B882331F06FE7DF
:1031D0007EE08FEB98E00E94BF731092BC081092C3
:1031E000BB0880E090E19093B7088093B60884E82C
:1031F00090E09093BE088093BD0881E08093B8086A
:1032000080E090E29093BA088093B9088AEA98E047
:103210000E94A1128AEA98E00E945E1288EC90E077
:103220000895EF92FF920F931F93CF93DF93CDB743
:10323000DEB72C970FB6F894DEBF0FBECDBF8C0162
:103240007B0185EA93E09A8389831B821C821D821D
:103250001E8298878F8319861A861B861C860530E6
:103260001105ECF0BE01695F7F4FF7018085918504
:103270000E941411892B99F0CE0107960E9459875C
:10328000BE01695F7F4FF701868197810E9414110B
:10329000892B61F0CE0107960E942F880EC0CE01C7
:1032A00001960E9459870430110554F7CE0101960A
:1032B0000E942F88033011058CF1BE01695F7F4F9A
:1032C000F701848195810E941411892B39F1CE0177
:1032D00007960E94C487BE01695F7F4FF701828114
:1032E00093810E941411892B01F1CE0107960E944F
:1032F000EE8668E67EE08FEB98E00E94BF7388EC74
:1033000090E02C960FB6F894DEBF0FBECDBFDF91D4
:10331000CF911F910F91FF90EF900895CE010196EC
:103320000E94C48702301105B4F6CE0101960E94B6
:10333000EE8601301105E9F6CE0101960E94EE8677
:103340006FE67EE08FEB98E00E94BF73D2CF0F93C1
:103350001F93CF93DF938C01EB010297C4F08A8116
:103360009B810E9417B88093050299270E94648967
:103370000230110549F08C819D810E9417B880931D
:10338000040299270E946E89C8ECD0E002C0C0E90F
:10339000D1E064E57EE08FEB98E00E94BF7360911E
:1033A00005028FEB98E00E9499896FE37EE08FEB36
:1033B00098E00E94BF73609104028FEB98E00E9436
:1033C00099898FEB98E00E94C872CE01DF91CF916E
:1033D0001F910F910895CF93DF93EB010297A4F112
:1033E0006AE27FE08A819B810E9465B8892B29F47B
:1033F0000E949A886F770E94F48866E27FE08A8153
:103400009B810E9465B8892B29F40E949A88606884
:103410000E94F4886EE27EE08FEB98E00E94BF731A
:103420000E949A886095661F6627661F70E08FEB82
:1034300098E00E94A0898FEB98E00E94C87288EC07
:1034400090E0DF91CF9108950E942817F8CFDF9286
:10345000EF92FF920F931F93CF93DF938C01FC01A8
:10346000808191810E94A889C82FD0E0C430D10505
:1034700084F40E945A77009721F0FC012085207F78
:103480002087BC01F801808191810E947A89219670
:10349000EDCFF801C081D18160E0CE010E94D484DB
:1034A000FC01D184F801D08661E0CE010E94D48471
:1034B0007C01F8019383828362E0CE010E94D48470
:1034C000F8019583848364E0CE010E94D484F801DE
:1034D00097838683F0E1DF1250C08BE090E00E947A
:1034E0004BB5EC011B830A8384E392E099838883C4
:1034F0001E82C8010E94B58997FD47C09D838C83B9
:103500008C819D81009719F08634910524F080E22A
:1035100090E09D838C83E114F10409F445C0F70128
:1035200080858F70853009F03FC0C7010E94A8894F
:103530008230D0F161E0C7010E94D484FC01908503
:103540009F70923051F561857285838594850E94C4
:10355000EABF20E030E04AE754E40E9449C00E94FC
:10356000BCC2611571058105910511F16F837887E2
:1035700089879A87F801D287C187DF91CF911F9100
:103580000F91FF90EF90DF900895919581959109AB
:103590009D838C8381E08E83B3CF933029F4618542
:1035A000728583859485D5CF60E070E0CB01D1CF63
:1035B00088E893E1A0E0B0E08F839887A987BA8775
:1035C000D9CFCF93DF93EC01798368831A8619866C
:1035D0001B861E8A1D8A0E941A12882329F0CE019A
:1035E000DF91CF910C94271ADF91CF910895CF925C
:1035F000DF92EF92FF920F931F93CF93DF93EC0133
:103600006A017B018E819F81892BD9F48881998100
:103610000E94A889082F10E00530110594F40E943B
:103620005A77009721F0FC012085207F20879F8317
:103630008E83BC01888199810E947A890F5F1F4F18
:10364000EBCFEE81FF81309749F18085982F9F70F5
:1036500019F5807F82608087EE81FF81C186D286E6
:10366000E386F48662E076E080E799E00E94BF732B
:103670002AE030E0B701A60180E799E00E94D3720A
:1036800080E799E0DF91CF911F910F91FF90EF902C
:10369000DF90CF900C94C8729230F1F2DF91CF910D
:1036A0001F910F91FF90EF90DF90CF900895EF92D0
:1036B000FF920F931F93CF93DF93EC018B011D8239
:1036C0001C821A821B82E880F980E114F10409F45B
:1036D00072C08091B0059091B105892B09F46BC03F
:1036E000672B09F48701F80180858F708630A9F473
:1036F00067EA73E0C8010E945F84009719F0FC013B
:1037000081858A8368E875E0C8010E945F8400971C
:1037100009F458C0FC0181858B8369EA73E0C70115
:103720000E945F84009709F043C06CE875E080E771
:1037300099E00E94BF736B8180E799E00E949989AC
:103740006AE875E080E799E00E94BF736A8180E7CC
:1037500099E00E94998980E799E00E94C872E88008
:10376000F9800E945A778C010097D1F0FC01808586
:10377000807F8260808711861286138614868081FE
:103780009181009711F00E94E7B589EA93E00E94C9
:10379000AEC5F80191838083B801C7010E947A8980
:1037A00069EA73E0888199810E945F84009719F02B
:1037B00009969D838C83DF91CF911F910F91FF908C
:1037C000EF900895F801808191810E9417B8A4CFED
:1037D0001F93CF93DF93FC01162FC389D48981896E
:1037E00092899C012F5F3F4F328B218BC80FD91FCD
:1037F000CE010E9407C1181721F0612FCE010E944F
:103800000FC181E090E0DF91CF911F910895FC01FD
:1038100081899289248535858217930740F423890D
:103820003489820F931F0E9407C190E008958FEFA3
:103830009FEF08952F923F924F925F926F927F92E7
:103840008F929F92AF92BF92CF92DF92EF92FF92B0
:103850000F931F93CF93DF93CDB7DEB762970FB669
:10386000F894DEBF0FBECDBF5C014B0129013A01C8
:10387000CA01B9010E94B5C21B013F926F9384EE49
:1038800093E09F938F93CE0101967C019F938F933A
:103890000E949EC60F900F900F900F900F900F9068
:1038A00020E030E0A901C301B2010E94EBC218166A
:1038B00024F077FA709477F87094F7010190002063
:1038C000E9F731976F01CE18DF088EE28083A2E01E
:1038D000B0E0AC0FBD1FAC0DBD1DBA8BA98BB10103
:1038E00037FE03C0719561957109072E000C880B96
:1038F000990B0E94EABF9B01AC01C301B2010E9477
:10390000D6C120E030E040E251E40E9449C00E946C
:10391000B5C2605DE989FA896083FE01EC0DFD1D89
:103920001382D501ED91FC910288F389E02D980175
:10393000A701B401C501199562960FB6F894DEBFD0
:103940000FBECDBFDF91CF911F910F91FF90EF90F0
:10395000DF90CF90BF90AF909F908F907F906F90AF
:103960005F904F903F902F9008959B0190E00496B8
:10397000982F8827642F820F931F0C94C078CF93C1
:10398000DF93C82FD0E02496DC2FCC27C60FD71F9B
:103990000E9445788FE00E945A788D2F0E945A78B5
:1039A0008C2F0E945A7880E00E945A78C82F0E947B
:1039B00043788C2FDF91CF910895CF93DF93C82F59
:1039C000D62F472F60E170E00E94B51C4D2F61E1BA
:1039D00070E08C2FDF91CF910C94B51C90E0982F64
:1039E000882744E050E0845F9B4F0C949178FC0161
:1039F0008485843011F00C94D98080E00895CF93B1
:103A0000DF93FC0124852430D9F0EC010E94F71CDF
:103A1000843189F0882379F0883169F021E08C3194
:103A200059F4E881F9810084F185E02DCE011995E2
:103A300021E0892B09F420E0822FDF91CF910895B6
:103A400080E0FBCF44E050E0BC018FE090E00C94BC
:103A5000917844E050E0BC0185E090E00C949178CE
:103A600044E050E0BC0181E090E00C94917808952E
:103A70008F929F92AF92BF92CF92DF92EF92FF927E
:103A80000F931F93CF93DF93CDB7DEB72D970FB66C
:103A9000F894DEBF0FBECDBF7C0110E000E038EE31
:103AA000832E33E0932EA12CB12C4DE2C42E43E0A3
:103AB000D42E1C821B828D829E82AF82B886DA82CF
:103AC000C9820D87CE0101960E94F71C811135C075
:103AD000F7014481558120E061E0802F0E942A8017
:103AE00080E590E00E94968E63E070E0802F0E9457
:103AF000BF1C833129F462E070E0802F0E94F58EB4
:103B0000F70184819581000F111FF801E157F94FEA
:103B1000918380832D960FB6F894DEBF0FBECDBF84
:103B2000DF91CF911F910F91FF90EF90DF90CF9099
:103B3000BF90AF909F908F9008950F5F1F4F0430FC
:103B4000110509F0B6CFE6CFCF92DF92EF92FF9248
:103B50001F93CF93DF93FC011485143089F1EC019E
:103B600080E590E00E94968E68E070E0812F0E94D0
:103B7000F58E0E946F946B017C01CE010E94F71CB0
:103B80008823A1F062E370E080E090E00E942A9236
:103B90000E946F946C197D098E099F09683E7340DD
:103BA0008105910550F38C850E941680EC85F0E02C
:103BB000EE0FFF1FE157F94F1182108284E08C87CE
:103BC000DF91CF911F91FF90EF90DF90CF900895FC
:103BD0004F925F926F927F928F929F92AF92BF921D
:103BE000CF92DF92EF92FF921F93CF93DF93CDB7E7
:103BF000DEB72D970FB6F894DEBF0FBECDBF7C01A8
:103C00009FE8A92E96E0B92E10E0D12CC12C28EE09
:103C1000422E23E0522E612C712C3DE2832E33E0A4
:103C2000932E1C821B824D825E826F8278869A82DE
:103C300089821D87D5012D913D915D01F701848118
:103C4000958128173907B1F4CE0101960E94F71C1F
:103C5000843199F1CE0101960E94F71C8C3151F408
:103C6000CE0101960E949B14892B21F4CE0101966E
:103C70000E94A41D1F5F1430A1F6CD2841F4D70186
:103C8000ED91FC910084F185E02DC70119952D96E9
:103C90000FB6F894DEBF0FBECDBFDF91CF911F915D
:103CA000FF90EF90DF90CF90BF90AF909F908F905C
:103CB0007F906F905F904F900895CC24C394D12C47
:103CC000D9CF8F929F92AF92BF92CF92DF92EF9215
:103CD000FF920F931F93CF936C015B017A01FC015C
:103CE000C485C430A1F481E090E0F601938382831F
:103CF000F12CE12CC701CF911F910F91FF90EF9014
:103D0000DF90CF90BF90AF909F908F9008958A01E1
:103D10004130584010F000E018E080E590E00E944B
:103D2000968E8C2F0E94AD8F4C0163E070E08C2F3B
:103D30000E94BF1C873111F08C3129F58016910645
:103D400060F380E590E00E94968E9801A50170E0F6
:103D500060E08C2F0E944D8F60E270E08C2F0E94FB
:103D6000F58E62E070E08C2F0E94BF1C84FD13C0B2
:103D700063E070E08C2F0E94BF1C811107C08C2F64
:103D80000E941680B0CF10E000E0DBCF80E590E02D
:103D90000E94968EE6CF40E162E070E08C2F0E9498
:103DA000B51C012B09F0A6CF9ECF3F924F925F9298
:103DB0006F927F928F929F92AF92BF92CF92DF923B
:103DC000EF92FF920F931F93CF93DF93CDB7DEB7A0
:103DD0002D970FB6F894DEBF0FBECDBF6C015B010F
:103DE0004A010E94E81D8FE8E82E86E0F82E312C6B
:103DF00010E000E098EE492E93E0592E612C712CD2
:103E00001C821B824D825E826F8278868DE293E0F7
:103E10009A8389833D86F701219131917F01F601D3
:103E2000848195812817390771F4CE0101960E948B
:103E3000F71C873141F4A401B501CE0101960E941F
:103E4000611E080F191F3394F4E03F12D9CFC80147
:103E50002D960FB6F894DEBF0FBECDBFDF91CF9188
:103E60001F910F91FF90EF90DF90CF90BF90AF9098
:103E70009F908F907F906F905F904F903F900895AC
:103E8000CF93DF9391E090931C068823B9F0C09103
:103E9000B800D091BA008091BC008A7B8093BC00AE
:103EA00060E084E10E948B9060E085E10E948B904D
:103EB0000E94B514D093BA00C093B800DF91CF919F
:103EC0000895CF92DF92EF92FF920F931F93CF93BB
:103ED000FC01C1810E9412916B017C018091D40789
:103EE000811164C081E08093D4078093D3079FEF52
:103EF0009093D2071092D1071092D0078093AF070A
:103F00008091AF07CC0FC82BC093AF078091AE074D
:103F1000813009F081C01092AE070E9412916B01AE
:103F20007C018091AF078093BB008091D607909170
:103F3000D707A091D807B091D907892B8A2B8B2B53
:103F4000A1F00E9412910091D6071091D7072091FD
:103F5000D8073091D9076C197D098E099F0906177A
:103F600017072807390708F442C08091BC0083FD79
:103F7000D8CF85EC8093BC000E9412916B017C012C
:103F80008091D407813009F449C08091D107811113
:103F900067C08091D107E0EBF7E0A6E6B6E090E0DD
:103FA000981751F121912D939F5FFACF8091D607F9
:103FB0009091D707A091D807B091D907892B8A2B68
:103FC0008B2B09F48BCF0E9412910091D607109190
:103FD000D7072091D8073091D9076C197D098E0930
:103FE0009F09061717072807390708F077CF809130
:103FF000D5070E94401F80E01092650680936406FA
:1040000083E398E00E944710CF911F910F91FF909A
:10401000EF90DF90CF90089585EEACCF8091D607DA
:104020009091D707A091D807B091D907892B8A2BF7
:104030008B2B09F4A5CF0E9412910091D607109105
:10404000D7072091D8073091D9076C197D098E09BF
:104050009F09061717072807390708F091CFC7CF20
:1040600081E099CFAF92BF92CF92DF92EF92FF9211
:104070001F93CF93DF93EC010E946F946B017C013F
:1040800028EEC20E23E0D21EE11CF11C10E08BE4EE
:10409000A82EB12C0E946F946C157D058E059F058E
:1040A00098F460EFCE010E94A414CE010E94611F1B
:1040B000182F80FF0BC0ED85FE85309709F019950C
:1040C000C5010197F1F7E6CF81E08A83812FDF9167
:1040D000CF911F91FF90EF90DF90CF90BF90AF9066
:1040E00008951F93CF93DF93EC01162F0E94322087
:1040F000CE010E94031062ED83E398E00E948E10CF
:10410000612F70E06095709584E0660F771F8A9547
:10411000E1F7612B83E398E00E948E100E942792C2
:10412000CE010E94611F811711F084E08A83DF9124
:10413000CF911F910895CF93DF93EC0163EC0E9420
:10414000A414CE01DF91CF910C94611F0F931F93A4
:10415000CF93DF93EC010E94322080FD36C0CE0168
:104160000E949B2060E0CE010E947120CE010E943F
:104170003220CE010E94031064EB83E398E00E949A
:104180008E100E942792CE010E943220082F10E04C
:1041900082FF16C082E08A838881882341F0CE01A5
:1041A0000E949B20682F6160CE010E9471201595AE
:1041B0000795802F8170DF91CF911F910F91089506
:1041C0008A81823049F71A82E7CF80E0F4CFCF931B
:1041D000DF93EC010E949B20682F6460CE01DF9189
:1041E000CF910C9471200F931F93CF93DF93EC0129
:1041F000162F042F0E943220002319F0CE010E94B6
:10420000E720CE010E94031065EA83E398E00E9454
:104210008E10612F83E398E00E948E10DF91CF9182
:104220001F910F910C9427926F927F928F929F9281
:10423000AF92BF92CF92DF92EF92FF920F931F93B4
:10424000CF93DF93FC01248521118CC0872E762E1D
:10425000EC010E94A620882309F486C0CE010E94AA
:10426000322040E060EFCE010E94F32010E000E039
:1042700066246A94AA24A394B12CE02EE694E694D2
:10428000E694F12C802F8770650101C0CC0C8A95D3
:10429000EAF78B85082E000C990B0817190734F5DF
:1042A000FE01EE0DFF1D93809C20CE010E94322066
:1042B000CE010E94031068E783E398E00E948E100D
:1042C000992011F080E8982E692D83E398E00E94F0
:1042D0008E100E942792CE010E943220982F907457
:1042E00085FF0BC0992369F08EEF2AC0992493941F
:1042F00008171907D1F2912CD8CF911102C087FF6E
:10430000602EFE01EE0DFF1D938187FF28C0C92A94
:10431000C3820F5F1F4F0034110509F0AECF6B86CB
:10432000FFEF6F1202C081E08C872396E72DF82DF6
:10433000CF01089629912193E817F907D9F781E071
:10434000DF91CF911F910F91FF90EF90DF90CF9071
:10435000BF90AF909F908F907F906F900895C09482
:10436000C922D6CF80E0ECCF8FEFEACFEF92FF9259
:104370000F931F93CF93DF938C017B0140E065E5A2
:104380000E94F320E70188E0E80EF11C699140E00B
:10439000C8010E94F320CE15DF05C1F7DF91CF9150
:1043A0001F910F91FF90EF900895CF92DF92EF92BF
:1043B000FF920F931F93CF93DF938C01EB017A0150
:1043C000FC01858196810E94A6208823C1F1BE014F
:1043D000F801858196810E94B62140E06EEBF801DC
:1043E000858196810E94F320E7016701F9E0CF0EF5
:1043F000D11CF801E580F680C7010E943220C70178
:104400000E94031066E983E398E00E948E100E94E8
:104410002792C7010E94322061EEC7010E94A414B6
:10442000C7010E94611F8993CC16DD0611F7F801C0
:10443000858196810E94A62091E0813009F090E06C
:10444000892FDF91CF911F910F91FF90EF90DF9017
:10445000CF900895CF93DF93EA010E94D521982F42
:10446000882341F068E0CE010E94F70F91E0288593
:10447000281390E0892FDF91CF910895CF93DF9398
:1044800000D000D000D0CDB7DEB7AE014F5F5F4F98
:104490000E942A22882331F08D818F33A9F020F4E5
:1044A0008F31A1F080E007C08F3521F08F37D1F731
:1044B0008CE001C08BE029960FB6F894DEBF0FBEEA
:1044C000CDBFDF91CF9108958AE0F5CF89E0F3CF9A
:1044D00085ED8093BC008091D6079091D707A0917D
:1044E000D807B091D9070796A11DB11D23E0B69555
:1044F000A795979587952A95D1F72091BC0024FD23
:1045000003C01092D40708954091D6075091D70761
:104510006091D8077091D907452B462B472B69F33B
:104520000097A105B10541F025E32A95F1F70000B8
:104530000197A109B109E1CF8091D5070C94401FE3
:104540001F920F920FB60F9211240BB60F922F935A
:104550003F934F935F936F937F938F939F93AF930B
:10456000BF93EF93FF938091B900887F803609F461
:104570004DC008F040C0883209F4A9C028F5803148
:1045800009F49DC0C8F4882309F4FBC0883009F4FD
:1045900096C0FF91EF91BF91AF919F918F917F91C5
:1045A0006F915F914F913F912F910F900BBE0F90A4
:1045B0000FBE0F901F901895883109F488C0803283
:1045C00041F78093D20714C0803409F49DC040F4B1
:1045D0008033B9F38833E9F68093D20785ECB0C015
:1045E000803509F485C0883509F496C0883489F689
:1045F0000E946822CECF883909F48CC038F58837FC
:1046000029F050F4883611F0803719F683E0809352
:10461000D4071092630657C0883809F47BC08039EC
:1046200019F0803809F0B5CF80916306803208F028
:1046300071C0E091630681E08E0F809363068091E4
:10464000BB00F0E0ED5BF94F80833DC0803B39F06B
:10465000E0F4803A09F479C0883A09F09ACF84E00E
:104660008093D4071092400610923F06E0913D06D9
:10467000F0913E06199580913F0681110FC081E0AF
:1046800080933F0610921D0609C0803C09F4A6CF16
:10469000883C09F4A3CF883B09F07BCFE09140062A
:1046A00081E08E0F80934006F0E0E35EF94F808159
:1046B0008093BB009091400680913F0629C0809175
:1046C000AF078093BB0085EC8093BC0062CF9091D4
:1046D000D1078091D007981758F5E091D10781E074
:1046E0008E0F8093D107F0E0E055F84F8081E9CF3D
:1046F000E091D10781E08E0F8093D1078091BB00BC
:10470000F0E0E055F84F80839091D1078091D00779
:104710009817C8F285E8D8CFE091D10781E08E0FD5
:104720008093D1078091BB00F0E0E055F84F808383
:104730008091D30781115CCF81E08093AE0784EA3A
:104740008093BC001092D40724CF85EC8093BC00EA
:104750001092D40780916306803230F4E0916306B2
:10476000F0E0ED5BF94F10826091630670E0E0913C
:104770004106F091420683E496E019951092630693
:1047800008CF1092D20734CF4F925F926F927F92F0
:10479000AF92BF92CF92DF92EF92FF920F931F934F
:1047A000CF93DF9300D01F92CDB7DEB72B013C0132
:1047B00029833A834B835C83A6019501C801B70125
:1047C000640D751D861D971D211531054105510587
:1047D00011F00E942DC129813A814B815C816217C1
:1047E000730784079507D0F424153505460557054A
:1047F00030F521E0822F0F900F900F900F90DF91F6
:10480000CF911F910F91FF90EF90DF90CF90BF90CD
:10481000AF907F906F905F904F9008954616570627
:104820006806790650F421E089819A81AB81BC81C8
:1048300084159505A605B705E8F220E0DBCF21E059
:104840004616570668067906A8F2F7CF8F929F9210
:10485000AF92BF92CF92DF92EF92FF920F931F938E
:10486000CF93DF937C014A015901C0911A06D09180
:104870001B06062F660F110B209709F45CC0888574
:104880008F70863009F055C06CEA73E0CE010E944B
:104890005F846C0182E08816910449F061EB73E05B
:1048A000E3E08E16910429F0D0E0C0E006C065EB8D
:1048B00073E0CE010E945F84EC01C114D104D9F1F0
:1048C000F60180858F708430B1F561857285A8010D
:1048D000C7010E9447C6A8016AEB73E0C7010E94A6
:1048E00029C6209779F188858F70843059F56985BC
:1048F0007A85A801C7010E9429C6A8016AEB73E066
:10490000C7010E9429C6A114B10429F0A801B5016C
:10491000C7010E9429C6C701DF91CF911F910F9156
:10492000FF90EF90DF90CF90BF90AF909F908F90CF
:104930000895D0E0C0E0A8016CE274E1C7010E94D4
:10494000BAB8C9CFF2E08F16910481F083E08816DF
:10495000910429F06091880670918906CACFA80158
:1049600066E274E1C7010E949CB8C7CFA80163E268
:1049700074E1F8CFCF92DF92EF92FF920F931F93E3
:10498000CF93DF93CDB7DEB7C154D1090FB6F894FA
:10499000DEBF0FBECDBF6C01AB0130E020E060E4B4
:1049A000CE0101967C010E942624F701019000208F
:1049B000E9F731978F010E191F09A801B701C60148
:1049C0000E9439C6892B11F010E000E0C801CF5BCE
:1049D000DF4F0FB6F894DEBF0FBECDBFDF91CF9192
:1049E0001F910F91FF90EF90DF90CF900895CF929D
:1049F000DF92EF92FF920F931F93CF93DF93CDB788
:104A0000DEB7C054D1090FB6F894DEBF0FBECDBFDC
:104A10008091970690919806059709F449C0611511
:104A2000710509F445C069017A018B0140E450E049
:104A3000CE0101960E9447C66FE270E0CE0101965A
:104A40000E940EC6892B41F4980143E050E060E4D7
:104A5000CE0101960E9426244FE350E0B601CE011C
:104A600001960E9429C60E947A84882309F18091C8
:104A70009706909198060697D9F48091FE078111C8
:104A800017C0B701CE0101960E943D9581E090E0EC
:104A9000C05CDF4F0FB6F894DEBF0FBECDBFDF9115
:104AA000CF911F910F91FF90EF90DF90CF900895DD
:104AB00090E080E0EDCFEF92FF920F931F93CF93A2
:104AC000DF93EC01A881B981109761F18C91882363
:104AD00049F108811981F8018081882351F08D32D4
:104AE00041F080538A3028F00F5F1F4F19830883ED
:104AF000F0CFC8010E9417B87C016CE270E0C801D9
:104B00000E940EC6009751F419821882C701DF91E6
:104B1000CF911F910F91FF90EF9008950196998387
:104B20008883F4CFF12CE12CF1CF4F925F926F92FA
:104B30007F928F929F92AF92BF92CF92DF92EF922D
:104B4000FF920F931F93CF93DF93CDB7DEB761979B
:104B50000FB6F894DEBF0FBECDBF0E946F949B01CD
:104B6000AC016091C3057091C4058091C505909119
:104B7000C605A12CB12C650118E8E12E13E1F12E38
:104B800000E010E00E94C423882319F1E09086061B
:104B9000F0908706D70112968C91823089F567EFE5
:104BA00073E180E799E00E94BF7380E799E00E947B
:104BB000C87280918606909187060E94A6200E9466
:104BC0006F946093C3057093C4058093C50590935B
:104BD000C60561960FB6F894DEBF0FBECDBFDF915C
:104BE000CF911F910F91FF90EF90DF90CF90BF90EA
:104BF000AF909F908F907F906F905F904F900895AF
:104C00008091C1059091C205892B09F0DDC083E137
:104C100090E00E944BB58C0188E199E6F801928BF7
:104C2000818BF682E5821482108289E0818381E0A3
:104C3000828383831093C2050093C1050E946F9401
:104C40006B017C01F0E1CF0EF7E2DF1EE11CF11CED
:104C5000D8011596ED91FC9116978FEF83871486F6
:104C6000138214821582168217821086118612868C
:104C700014961C9299249394BE01665F7F4FF801AD
:104C8000858196810E94142118160CF071C00E9433
:104C90006F946C157D058E059F0508F069C067E06F
:104CA000CE010A960E94F70F99898913E5CFD801A2
:104CB0008C91811138C015968D919C910E94A620EF
:104CC000BE01665F7F4FF801858196810E94B62103
:104CD00040E064EBD80115968D919C910E94F320E1
:104CE000F801A580B680C5010E943220C5010E944E
:104CF000031067E883E398E00E948E1060E883E386
:104D000098E00E948E100E942792C5010E943220D6
:104D1000B82ED80115968D919C910E94A620B5FCC5
:104D200002C0F8019082AE014F5F5F4FBE01665F27
:104D30007F4FC8010E94D521D8011196BC908A8569
:104D4000803109F48CC2BE01665F7F4FC8010E94AA
:104D50003E228B1558F5F8018181D80111968C936C
:104D6000119714968C9114978F5F14968C9384CF1F
:104D700010E000E08091C1059091C2052091BF052F
:104D80003091C00502171307ECF49801B3E0220F2D
:104D9000331FBA95E1F76091BD057091BE05620FB2
:104DA000731F0E945D920F5F1F4FE4CF8A85803191
:104DB00011F48CE0D2CFBE01665F7F4FC8010E9424
:104DC0003E22CBCFFC0112828091BB059091BC05A5
:104DD0002091BF053091C005821793070CF4D5C010
:104DE0000E946F942B013C01E0918606F0918706AA
:104DF000309759F08FEF83871486138214821582BF
:104E0000168217821086118612864091BF05509136
:104E1000C005E091B705F091B80590E080E08417F7
:104E200095070CF48EC088248394912C809186067B
:104E300090918706009709F48DC02091BF053091AD
:104E4000C005F3E0220F331FFA95E1F76091BD052D
:104E50007091BE05620F731F0E94142118160CF08A
:104E600079C08091BF059091C00541970CF072C048
:104E70000E946F949B01AC01A12CB12C650118E834
:104E8000E12E13E1F12E00E010E0C301B2010E9417
:104E9000C42381115FC0C090BD05D090BE05A09015
:104EA000BF05B090C005850173E0000F111F7A9512
:104EB000E1F70C0D1D1D67E0C8010E94F70FD80136
:104EC00017969C91F12CE12C8913B0CFEA14FB04C6
:104ED0000CF057C148E050E0B801C6010E94C8C5B7
:104EE000B8E0CB0ED11C892B09F04BC0EE0CFF1C97
:104EF000E091B705F091B805EE0DFF1D808191811D
:104F000081609183808361EE73E180E799E00E9484
:104F1000BF738091BF059091C00563E0880F991F12
:104F20006A95E1F72091BD053091BE05820F931F70
:104F30000E94108D6AED73E180E799E00E94E373AF
:104F400075CF21913191DF0112972E7F2D933C93E4
:104F5000019665CF68EE73E180E799E00E94BF7328
:104F60006091BF057091C00580E799E00E94A0891B
:104F700080E799E00E94C8721092BC051092BB05B0
:104F80001ECEEFEFEE1AFE0AA1CF0091BD051091E3
:104F9000BE059C0143E0220F331F4A95E1F7020F43
:104FA000131FD8012C91283209F0DBC0AE014F5FEE
:104FB0005F4FB8018091C1059091C2050E942A22DD
:104FC000811105C020E030E04EEF52EC3EC06A8116
:104FD00070E0762F6627770F770F770F2981B8E07B
:104FE0002B9F90011124262B372BF80180818031D3
:104FF000D1F4688570E08F81AB01481B5109CA016B
:105000009695982F8827979587950E94A4C1CB01E4
:105010004097B90113E0660F771F1A95E1F76078A2
:105020009C01260F371F213854EE35075CF2B90179
:10503000330F880B990B0E94EABF20E030E040E07C
:105040005CE30E9449C09B01AC01E091B905F0917D
:10505000BA058091BB059091BC05BC01A3E0660F29
:10506000771FAA95E1F7A091BD05B091BE056A0F23
:105070007B1F309709F019950091C1051091C20569
:10508000E090BB05F090BC0573E0EE0CFF1C7A9538
:10509000E1F78091BD059091BE05E80EF91ED7019C
:1050A0008C91803109F463C0B701C8010E943E228F
:1050B000D82E882309F451C0F801858196810E9479
:1050C000A620882309F449C0B701D80115968D910F
:1050D0009C910E94B621F801408164E4858196810B
:1050E0000E94F320D80112968C918823B1F1E7EF4A
:1050F000ED0D4EEE842E42E0942EE33038F4F0E0D5
:10510000EE0FFF1FE157FD4F80809180E114F10405
:1051100089F1F8018381882369F1808181112AC096
:105120000E946F942B013C01092C000CAA08BB08BB
:10513000AE014F5F5F4FB701C8010E94D521898141
:1051400081110BC00E946F94681979098A099B0923
:10515000641575058605970558F38091BB059091F8
:10516000BC0501969093BC058093BB0528CD6CE0EF
:10517000D62EA2CFB401990C880B990B0E942A92CB
:10518000ECCF8091C1059091C205892B09F44ECED8
:1051900088E0815008F44ACEF801E80FF11D9081B3
:1051A0009923B9F3AA0CBB1C8091B7059091B8055F
:1051B000A80EB91ED5018D929C9265ED73E180E732
:1051C00099E00E94BF736091BF057091C00580E7B0
:1051D00099E00E94A0896EEC73E180E799E00E945B
:1051E000BF738091BF059091C00523E0880F991F80
:1051F0002A95E1F72091BD053091BE05820F931FDE
:105200000E94108D80E799E00E94C8728091BF05CE
:105210009091C00533E0880F991F3A95E1F76091AE
:10522000BD057091BE05680F791FFB018081883232
:1052300061F48091C1059091C2050E945D928091B8
:105240008606909187060E94E7208091BF05909185
:10525000C00501969093C0058093BF05E7CDFCE0A3
:10526000FB1508F478CDA5CD61E072E18FEB98E0F5
:105270000E94BF736EEE71E18FEB98E00E94BF73E6
:1052800060EE71E18FEB98E00E94BF7368ED71E111
:105290008FEB98E00E94BF738FEB98E00E94C8727A
:1052A00068EC71E18FEB98E00E94BF736CEB71E1E9
:1052B0008FEB98E00E94BF7364E971E18FEB98E097
:1052C0000E94BF7367E871E18FEB98E00E94BF73A3
:1052D00062E771E18FEB98E00E94BF7363E671E1D2
:1052E0008FEB98E00E94BF736BE571E18FEB98E064
:1052F0000E94BF7360E571E18FEB98E00E94BF737D
:1053000066E471E18FEB98E00E94BF7367E371E19F
:105310008FEB98E00E94BF736FE271E18FEB98E032
:105320000E94BF7363E271E18FEB98E00E94BF734C
:1053300069E071E18FEB98E00E94BF736AEE70E163
:105340008FEB98E00E94BF7365ED70E18FEB98E002
:105350000E94BF7368EC70E18FEB98E00E94BF730E
:105360006AEB70E18FEB98E00E94BF736EEA70E128
:105370008FEB98E00E94BF7366EA70E18FEB98E0D4
:105380000E94BF736BE970E18FEB98E00E94BF73DE
:105390006EE870E18FEB98E00E94BF7366E870E101
:1053A0008FEB98E00E94BF736BE770E18FEB98E0A2
:1053B0000E94BF736CE670E18FEB98E00E94BF73B0
:1053C00063E670E18FEB98E00E94BF7365E570E1E2
:1053D0008FEB98E00E94BF7367E470E18FEB98E079
:1053E0000E94BF738FEB98E00C94C872009789F00D
:1053F000FC0120852F70253061F40E94D484009731
:1054000041F0FC0120852F70243019F481859285AC
:10541000089590E080E00895CF92DF92EF92FF929E
:105420000F931F93CF93DF9300D000D0CDB7DEB79B
:105430008091190681119AC08091970690919806E3
:1054400002970CF493C08091B0059091B10500973C
:1054500009F48CC06EEB73E00E945F848C010097AE
:1054600009F484C00E94A889E82EF12CE114F1040B
:1054700009F47CC070E060E0C8010E94F6296C016C
:10548000EA94EF2809F481C061E0C8010E94D48445
:10549000FC0101851285CE0101960E94998ECE01F4
:1054A00001960E94B78E60E07AE08FEB98E00E9450
:1054B000BF73B6018FEB98E00E94597365EC73E0FF
:1054C0008FEB98E00E945973B8018FEB98E00E942F
:1054D000A08965EC73E08FEB98E00E9459736DE949
:1054E00077E08FEB98E00E9459738FEB98E00E9471
:1054F000C87262E072E08EE899E00E941714D092C0
:105500008409C092830910938609009385098DE967
:1055100097E0892BE9F58CEB93E0909388098093D1
:10552000870980918A0690918B06009741F070E080
:1055300060E00E94F6299093890680938806809106
:10554000880690918906009731F190938A0980939B
:10555000890910928C0910928B0981E080931906B9
:1055600067EE79E08FEB98E00E94BF7326960FB646
:10557000F894DEBF0FBECDBFDF91CF911F910F9189
:10558000FF90EF90DF90CF90089502E012E083CF7C
:105590008DE997E0C2CF82EA92E0892B19F48CEB77
:1055A00093E0D3CF82EA92E0D0CF2F923F924F92F6
:1055B0005F926F927F928F929F92AF92BF92CF92A3
:1055C000DF92EF92FF920F93CF93DF9300D01F9261
:1055D000CDB7DEB77C017A8369835C834B83DB01C3
:1055E0001C92FC016081662309F44DC030FF4BC062
:1055F000F9E06F9FB00111246E5E724ECD010E94E2
:10560000BAB8D70111968C91807F41F04B815C81B3
:1056100067EC73E089819A810E9429C6E981FA8149
:1056200001900020E9F7319789819A81E81BF90BF5
:105630001C012E0E3F1EAB81BC81AE1BBF0B119710
:10564000BC83AB83D7011196EC9111978E2F807F8D
:1056500009F4BCC0E295EF70E150EC3008F0B6C040
:10566000F0E08827E95CF44D8F4F0C94B8C1462BCD
:10567000B52B1B2C802C9B2C822B312C312C312CCC
:10568000762B6A2BB72C29803A80DCCFF7018481F6
:10569000282F30E050E040E0002359F030E0A4E64D
:1056A000B0E00E9481C12FEF30E040E050E00E9466
:1056B0004FC15F934F933F932F9389EC93E09F9358
:1056C0008F93FC81FF938B818F933F922F920E9447
:1056D00061C677C0F70187818F9386818F9385811B
:1056E0008F9384818F938CEC93E0E9CFF7018781CE
:1056F0008F9386818F9385818F9384818F9380EDA3
:1057000093E0DDCFF701C480D580E680F780C70144
:10571000B6012AE030E040E050E00E944FC197FF20
:1057200007C090958095709561957F4F8F4F9F4FE3
:105730009F938F937F936F93C701B6012AE030E068
:1057400040E050E00E944FC15F934F933F932F93EF
:1057500084ED93E09F938F93FC81FF938B818F93D4
:105760003F922F920E9461C62CC0C7010E94F8117F
:10577000BC01F701C680D780D0FADD24D0F894812F
:10578000F580EB80BC80292F30E050E040E077FDD1
:1057900035C0011135C07F936F931F921F921F92E6
:1057A0009F931F92FF92DF92CF928BED93E09F9396
:1057B0008F939C819F93AB81AF933F922F920E94D6
:1057C00061C60FB6F894DEBF0FBECDBF89819A8146
:1057D0000F900F900F900F90DF91CF910F91FF904E
:1057E000EF90DF90CF90BF90AF909F908F907F9081
:1057F0006F905F904F903F902F900895002361F03D
:10580000292F30E0A4E6B0E00E9481C12FEF30E004
:1058100040E050E00E944FC15F934F933F932F931E
:105820001F92FF92DF92CF928EED93E09F938F9322
:10583000BF92EF9295CF15968C9115971F928F93EB
:1058400016969C91169717968C9181708F939F93C3
:1058500081EE93E09F938F93BC81BF93EB81EF9395
:1058600034CF14968D909D90AD90BC90179720E00A
:1058700030E0A901C501B4010E94E3BF2401350154
:1058800087FF04C077FA709477F87094C301B2016F
:105890000E94B5C26B01072E000C880B990B0E9469
:1058A000EABF9B01AC01C301B2010E94D6C120E056
:1058B00030E048EC52E40E9449C00E9440C30E947C
:1058C000B5C2062F772E20E030E0A901C501B40152
:1058D0000E94E3BF87FF07C07F920F93DF92CF92B2
:1058E00087EE93E0B7CF7F920F93DF92CF9288EE4F
:1058F00093E09F938F939C819F93AB81AF93E5CE71
:1059000014968C9114971F928F9315968C911597DE
:105910001F928F9316968C911F928F938EED93E02A
:105920009F938F93BC81BF93EB81EF933F922F9214
:105930000E9461C646CF17968C9117971F928F933E
:1059400014968C9114971F928F9315968C9115979E
:105950001F928F9316968C911F928F938BED93E0ED
:105960009F938F93BC81BF93EB81EF93F9CE1496F5
:105970006D917C914B815C81C1010E9447C626CF0D
:10598000EF92FF920F93CF93DF93CDB7DEB7A0973F
:105990000FB6F894DEBF0FBECDBF7C0100E020E063
:1059A00033E040E250E0BE016F5F7F4F0E94D52A96
:1059B000BE016F5F7F4F80E799E00E94597363EEED
:1059C00078E080E799E00E94BF73F70161816295FA
:1059D0006F7080E799E00E9499896CED78E080E72C
:1059E00099E00E94BF73F70161816F7080E799E0D1
:1059F0000E94998980E799E00E94C872A0960FB62C
:105A0000F894DEBF0FBECDBFDF91CF910F91FF9015
:105A1000EF900895AF92BF92CF92EF92FF920F93C3
:105A20001F93CF93DF9300D000D01F921F92CDB76A
:105A3000DEB75C0109831A832B833C834D835E832D
:105A40006F83788763EC73E180E799E00E94BF730E
:105A5000CE0101960E94C02C6CEB73E1C7010E943D
:105A600083B8009709F45AC08981811130C00A8136
:105A70000F70013089F128F010E00230F1F5CC20F0
:105A8000C1F0CE0101960E94E184F50102811381EB
:105A9000892B91F0C8010E947517672B682B692B21
:105AA00041F480E00E944414AB01BC01C8010E9493
:105AB000F71A81E090E032C040E050E0BA01C8013E
:105AC0000E94F71A60E0C5010E94E817F2CF823009
:105AD000E1F1A0F58130A9F16FEA73E180E799E087
:105AE0000E94BF73698180E799E00E94998980E7ED
:105AF00099E00E94C87201E010E06FE973E180E76D
:105B000099E00E94BF73B80180E799E00E94A089E4
:105B100080E799E00E94C87290E080E028960FB676
:105B2000F894DEBF0FBECDBFDF91CF911F910F91D3
:105B3000FF90EF90CF90BF90AF9008958A5085303E
:105B400058F6F50102811381A5CF40E050E0BA017B
:105B5000F50182819381B4CFCF92DF92FF920F93B0
:105B60001F93CF93DF938C01EB016A01CB010E945D
:105B70001A12F82E882309F458C0D0FE05C0F80187
:105B80006081CE010E94AB17D1FE46C0F801818131
:105B900082958F704481558166817781873030F09E
:105BA0008930D0F096EF980F923090F0EC81FD8123
:105BB000309771F090859F702EEF290F223010F0F2
:105BC000911106C08295807F90859F70892B808778
:105BD000CE010E94261220C0EC81FD813097E1F0B9
:105BE00080858F709EEF980F923010F0811114C055
:105BF0004187528763877487EC81FD818085807F30
:105C000083608087EC81FD818085982F907F90361E
:105C100019F48F708067808765ED78E080E799E000
:105C20000E94BF73C8010E94C02C8F2DDF91CF91BD
:105C30001F910F91FF90DF90CF900895CF92DF9248
:105C4000EF92FF920F931F93CF93DF93611571052E
:105C500009F474C06A017B018C01CB010E941A1205
:105C6000D82F8823C1F1D70114968D919C9100976C
:105C700009F446C0FC01C0852C2F2F703EEF320F77
:105C8000323010F0211131C0C595C595C595C59527
:105C9000D0FE72C0C7010E94DB17F8018083CC23BD
:105CA000F1F1C295C07F81818F70C82BC183D7016C
:105CB00014968D919C91009771F1FC0120852F70B5
:105CC000223001F581859285A385B485F80184830E
:105CD0009583A683B7838D2FDF91CF911F910F916D
:105CE000FF90EF90DF90CF900895253049F460E069
:105CF0000E94D484009721F0DC011896CC91C4CF87
:105D0000C0E0C6CF253039F460E00E94D48400970B
:105D100011F0FC01D7CF80E090E0DC01D7CFD701B4
:105D20001496ED91FC9180858295807F859585956F
:105D300085958595823021F0833081F0D0E0CBCFFE
:105D40004185528563857485F80181818F70806AF1
:105D500081834483558366837783BDCF4185528594
:105D600063857485F80181818F70806781834483A6
:105D7000558366837783AFCFCC2389F2C295C07FEA
:105D8000F80191CF0F931F93CF93DF9300D000D0F2
:105D90001F921F92CDB7DEB719821A821B821C8216
:105DA0001D821E821F8218862A812F702A83FC0181
:105DB00002811381C8010E94DB178230D1F0853047
:105DC000C1F08823B1F040E052E0B801CE01019665
:105DD0000E941E2ECE0101960E94E18428960FB6E5
:105DE000F894DEBF0FBECDBFDF91CF911F910F9111
:105DF000089590E080E0F2CFCF93DF9300D000D001
:105E00001F921F92CDB7DEB7FC01862F8F70618184
:105E1000607F682B618388E0DE01119601900D920E
:105E20008A95E1F729813A814B815C816D817E8180
:105E30008F81988528960FB6F894DEBF0FBECDBF30
:105E4000DF91CF910895CF93DF9300D000D01F92C0
:105E50001F92CDB7DEB7FC01608398E0DE0111969A
:105E600001900D929A95E1F729813A814B815C81ED
:105E70006D817E818F81988528960FB6F894DEBF5C
:105E80000FBECDBFDF91CF910895DC011196EC914B
:105E90001197E295EF70E150EB3008F037C0F0E079
:105EA0008827EA5AF04D8F4F0C94B8C1682F682F9D
:105EB000862F612F612F772F6E2F6E2F6E2F612F00
:105EC000612F14966D917D918D919C9117970895F6
:105ED00014966C9170E090E080E0089514966D91B6
:105EE0007D918D919C9117970E94B5C2089514964B
:105EF0006D917D918D919C9117972AE030E040E063
:105F000050E00E944FC1CA01B901089560E070E0FD
:105F1000CB010895CF93DF93EC016115710539F43E
:105F20008F8181708F8381E0DF91CF910895898186
:105F3000982F92959F7029F180E09430A8F79B01EB
:105F4000770F440B550B2959310941095109A4E632
:105F5000B0E00E946EC12BE531E040E050E00E94CD
:105F60004FC137FF02C030E020E02536310514F084
:105F700024E630E02F5F220F8F818170282B2F8342
:105F8000D2CF8F7080628983DACF2F923F924F9267
:105F90005F926F927F928F929F92AF92BF92CF92B9
:105FA000DF92EF92FF920F931F93CF93DF93CDB7C2
:105FB000DEB76A970FB6F894DEBF0FBECDBF1C01E7
:105FC00009871A872B873C874D875E876F87788B79
:105FD00022E1E216F10408F035C0F701E455FD4F67
:105FE00030813D8BCE0109960E94F81197FD04C0C7
:105FF000BC01C1010E948A2F9A85892F8F70D1011F
:106000001196EC911197E07FE82B1196EC93119784
:1060100089858C93E295EF70EC3008F063C0F0E076
:106020008827EA5EFF4C8F4F0C94B8C104323F3092
:106030003F30A431243038326E31AD31AD31AD3125
:106040006E316E311D8ACECF10E092959F709D30DB
:1060500008F010C4E92FF0E08827EE5CFF4C8F4F6A
:106060000C94B8C172307132913271323A323A3294
:10607000713271323A343A34713271324831929518
:106080009F709D3008F014C1E92FF0E08827E45B91
:10609000FF4C8F4F0C94B8C1723026311931DC306F
:1060A0005C305930FD30283158315831E730E73015
:1060B00048318889F10187838F85D10116968C93A9
:1060C00016978E8515968C9315978D8514968C93BF
:1060D00014979295907F11968C9111978F70982BB1
:1060E00011969C93FD89FF2309F463C0D101119699
:1060F0008C9182958F702F2F30E08217130609F450
:1061000058C066E378E080E799E00E94BF73F10130
:10611000618162956F7080E799E00E94998963E3DD
:1061200078E080E799E00E94BF736D8980E799E08D
:106130000E94998961E378E080E799E00E94BF734B
:10614000D1010C9119821A821B821C821D821E822F
:106150001F8218868D898295807F9A819F70892BF6
:106160008A830983EE24EA94FE2C11961C911197E0
:1061700012962C91129713963C91139714964C916A
:10618000149715965C91159716966C91169717961D
:106190007C91CE0101960E94C52FF10120833183AD
:1061A000428353836483758386839783C1010E94EE
:1061B000C02C88E0F1016EC18F859889F10186833A
:1061C000878190FB80F987838E8585838BCF8D8532
:1061D0009E85AF85B889B7FD0EC08F3F9105A1059B
:1061E000B10529F024F08FEF90E0A0E0B0E0D101FC
:1061F00014968C9377CF80E0FACF6D857E858F855E
:10620000988920E0673FBFEF7B078B079B076CF007
:106210002FEF6115EAE07E078105910534F42AE04D
:1062200030E040E050E00E944FC1D10114962C9321
:1062300059CF8F859889F1018683878190FB80F9FA
:1062400087838E8585838D8584834CCF8D85CFCF45
:10625000CD84DE84EF84F88820E030E0A901C70116
:10626000B6010E94E3BF60E087FD0FC020E030E090
:106270004FE753E4C701B6010E94EBC26FEF181657
:1062800024F0C701B6010E94BCC2F10164832ACF89
:10629000D10111968C9111978F70806C11968C930F
:1062A00011978D859E8515969C938E9314971ACF82
:1062B00063EC78E080E799E00E94BF736A8562959D
:1062C0006F7080E799E00E94998960EC78E080E740
:1062D00099E00E94BF73F1016181BFC092959F70E8
:1062E000933091F09C30A1F24D855E856F85788961
:1062F000F10144835583668377839295907F8181F2
:106300008F70982B9183EECEC1010E94E184D10160
:1063100014968C9314978F85988916968C9316975C
:1063200017968C91179790FB80F917968C93179777
:106330008E8515968C93159711968C9111978F7069
:10634000806211968C93CECECE0109960E94E18494
:10635000D10114968C931497EFCF92959F709D3036
:1063600008F065C0E92FF0E08827E654FE4C8F4F17
:106370000C94B8C17230D931033284310332033204
:10638000C731F331F331F331E731EE3148316D8507
:106390007E858F8598890E94EABF20E030E040E248
:1063A00051E40E9443C2F10164837583868397831D
:1063B00099CE6D8570E090E080E00E94E8BFD10149
:1063C00014966D937D938D939C9317978BCE6D85CB
:1063D0007E858F8598890E94EABFE5CF6D857E8591
:1063E0008F859889EACF9295907FF10181818F7096
:1063F000982B91838D859E85AF85B88984839583FD
:10640000A683B7836FCE9295907FD10111968C9120
:1064100011978F70982B11969C938D859E85AF85D3
:10642000B889F10184839583A683B7835BCE6EEA36
:1064300078E080E799E00E94BF736A8562956F708B
:1064400080E799E00E9499896BEA78E080E799E01B
:106450000E94BF73D10111966C9162956F7080E7B5
:1064600099E00E94998980E799E00E94C8723ACE2B
:1064700011E0EBCD4D855E856F857889F101448310
:106480005583668377839295907F81818F70982B57
:10649000918388E0DE01119601900D928A95E1F7D3
:1064A00029813A814B815C816D817E818F819885C4
:1064B0006A960FB6F894DEBF0FBECDBFDF91CF91C5
:1064C0001F910F91FF90EF90DF90CF90BF90AF9012
:1064D0009F908F907F906F905F904F903F902F9004
:1064E0000895963009F4C1C048F46D85913071F07B
:1064F0006FEF70E0933051F060E008C0973009F41E
:10650000C0C09A506D857E859230B0F784E68F8743
:1065100088898E7F888B1E868A858F7080628A87A5
:106520006D872E8530E0AFEFB0E00E9481C1C12CB5
:10653000D12C7601CA946115F4E67F078105910597
:1065400044F424E630E040E050E00E944FC169018D
:106550007A01112309F475C0DA8AC98A2D852E8B38
:10656000022F10E088898695A82FA150BB0BB88F09
:10657000AF8B119609F0A4C09601203831050CF0BC
:1065800087C08FE790E08C199D09809FD001819F83
:10659000B00D909FB00D11242FEF30E00E94CFC1BD
:1065A00021E83EE740E050E00E944FC1D10117963C
:1065B0002C93ABE9B0E0A70196010E946EC13FE7C2
:1065C000432E512C612C712CA30192010E944FC1CA
:1065D0002C593F4F4F4F5F4F5901AEEFB1E0A7012C
:1065E00096010E946EC1A30192010E944FC1D80181
:1065F0000E946EC12FEF30E040E050E00E944FC19A
:1066000089012F3F310519F014F00FEF10E06EE90A
:1066100078E080E799E00E94BF73B50180E799E0D8
:106620000E94A08960E978E080E799E00E94BF734A
:10663000B80180E799E00E94A08980E799E00E9474
:10664000C8726EE578E080E799E00E94BF7380E74A
:1066500099E00E94C87267E578E080E799E00E94BF
:10666000BF73C1010E94C02C3DCD6D857E858F8595
:1066700098892AE030E040E050E00E944FC1B90123
:1066800045CF6D857E858F8598890E94B5C23ECFA6
:10669000A7012058310941095109ABE9B0E00E9436
:1066A0006EC12FE730E040E050E00E944FC12C590E
:1066B0003F4F4F4F5F4F5901D10117961C92A7CF03
:1066C0002F89388DAAEBBFEF0E94C7C124E6822E26
:1066D000912CA12CB12CA50194010E944FC129013C
:1066E0003A01B4E64B0E511C611C711C26E430E0EB
:1066F000AF89B88D0E94CFC1A50194010E944FC1FE
:1067000049015A01EEE18E0E911CA11CB11C298990
:106710003A89203831050CF094C08FE790E0821B55
:10672000930B809FD001819FB00D909FB00D1124DD
:10673000A50194010E9479C19B01AC01AFEFB0E0CB
:106740000E946EC124E63AE640E050E00E944FC14C
:10675000D10117962C93A7019601240D351D461DD6
:10676000571DAEEFB1E00E946EC123EE30E040E075
:1067700050E00E944FC1298B3A8B4B8B5C8BE9898F
:10678000FA89FA8FE98FAFEFB0E0A70196010E9476
:106790006EC12FE730E040E050E00E944FC1790128
:1067A000FE89AF2FB0E029893A894B895C890E9424
:1067B0006EC12FEF30E040E050E00E944FC18901F0
:1067C0002F3F310519F014F00FEF10E06AE878E080
:1067D00080E799E00E94BF732AE030E0B301A20194
:1067E00080E799E00E94D37264E878E080E799E05E
:1067F0000E94BF732AE030E0B501A40180E799E070
:106800000E94D3726CE778E080E799E00E94BF7342
:10681000B70180E799E00E94A08964E778E080E70B
:1068200099E00E94BF73B80180E799E00E94A089B7
:106830006BE678E080E799E00E94BF73698D7A8DFE
:10684000F8CEA70196012058310941095109ABE959
:10685000B0E00E946EC12FE730E040E050E00E94BF
:106860004FC12C593F4F4F4F5F4F7901D1011796C0
:106870001C92ACCF65E478E080E799E00E94BF739A
:106880006A8562956F7080E799E00E94998962E459
:1068900078E01DCDFC019181892F82958F7021F0C8
:1068A000823029F080E008959F70906291839B016F
:1068B00077FF02C030E020E02E3681E0380714F088
:1068C0002DE631E02683878130FB80F9878381E0E4
:1068D00008950F931F93CF93DF938C01FC01C08128
:1068E000D1816FE270E0CE010E9456C60097D9F0C8
:1068F000FC011192CF010E943716EC016EE076E0A8
:1069000080E799E00E94BF73BE0180E799E00E9492
:10691000A08980E799E00E94C872CE01DF91CF91F3
:106920001F910F910895CE010E943716EC01892B1B
:10693000A1F3F80111821082F0CF8F929F92AF9253
:10694000BF92CF92DF92EF92FF920F931F93CF935C
:10695000DF93CDB7DEB767970FB6F894DEBF0FBEF3
:10696000CDBF8C017B014C018BE0880E911C9F8A6E
:106970008E8AF801128611861386168A158A672B6D
:1069800009F463C0A0909906B0909A06A114B104CE
:1069900009F45BC06FE270E0C7010E940EC66C0193
:1069A000892B09F44AC0F701DE01119690E080E0DE
:1069B000BD012191222341F02F3231F08431910524
:1069C00019F02D930196F5CF860F971FFC011082C9
:1069D000C5010E945F84F80191838083B6016F5FD7
:1069E0007F4F4AE050E0C4010E9447C6CE01469660
:1069F0000E946934F801968B858B8E899F89892B3B
:106A000009F41386C8010E941A12882319F0C801DC
:106A10000E94271A67960FB6F894DEBF0FBECDBF4F
:106A2000DF91CF911F910F91FF90EF90DF90CF906A
:106A3000BF90AF909F908F900895B701C5010E94BD
:106A40005F84F80191838083DDCFF8011182108289
:106A5000D9CF8F929F92AF92BF92CF92DF92EF9257
:106A6000FF920F931F93CF93DF93CDB7DEB7C75538
:106A7000D1090FB6F894DEBF0FBECDBF6115710509
:106A800009F486C0FA016B018C01E60FF71F108232
:106A90000E9452114B016EED79E080E799E00E946F
:106AA000BF73B40180E799E00E94A0896BED79E0A3
:106AB00080E799E00E94BF73B80180E799E00E94E7
:106AC000597368ED79E080E799E00E94BF738AE32B
:106AD000881681E098065CF46BEC79E089EC98E02C
:106AE0000E94BF7389EC98E00E94C87251C0B60141
:106AF00080E799E00E94597380E799E00E94C8728C
:106B00001A821982FE0133968EE3DF011D928A9567
:106B1000E9F78091970690919806059709F04CC087
:106B200063E070E0C8010E94BA247C01892B09F05F
:106B300053C0E0914508F0914608808180FF28C04D
:106B400062E070E0C8010E94BA24892BD1F064E2AF
:106B500070E0C8010E9456C6892BD1F463EB79E03E
:106B600080E799E00E94BF73B80180E799E00E9436
:106B7000597380E799E00E94C872C8010E94DB8FB8
:106B800007C061E070E0C8010E94BA24892BF9F6C1
:106B9000C95ADF4F0FB6F894DEBF0FBECDBFDF91ED
:106BA000CF911F910F91FF90EF90DF90CF90BF900A
:106BB000AF909F908F90089561E070E0C8010E94AF
:106BC000BA247C01892B09F562E070E0C8010E94BB
:106BD000BA247C01892B09F1E00EF11E6FE979E0FE
:106BE000C7010E9483B8892B09F5F60101900020A6
:106BF000E9F73197EC19FD093297C0F0C8010E94FE
:106C0000DB8FC6010E948F74C3CF4FE350E0B80101
:106C1000CE0101960E9447C6DFCF68EA79E080E79F
:106C200099E00E94BF7380E799E05ECFF701808111
:106C3000843209F4ADCFB701CE018F5B9F4F0E9424
:106C40009D34CE018F5B9F4F0E941A12882339F129
:106C5000B601CE018F5B9F4F0E946A8A18161906F3
:106C6000F4F489818823D9F0809197069091980651
:106C70000597A9F067E879E080E799E00E94BF7383
:106C8000BE016F5F7F4F80E799E00E94597380E7F4
:106C900099E00E94C872CE0101960E94DB8FCE015E
:106CA0008F5B9F4F0E94501273CFCF93DF93EB0106
:106CB00063E0FC01808191810E94D484FC01892BD6
:106CC000A9F080858D7091F4C095D095CF6FAE01FD
:106CD00070E060E081859285A385B4858C2395233F
:106CE000A623B72381879287A387B487DF91CF91AB
:106CF0000895CF93DF93EB0163E0FC0180819181E4
:106D00000E94D484FC01892BB9F09085892F8D7065
:106D100099F4907F92609087CC27CE01B0E0A0E0FC
:106D20004185528563857485842B952BA62BB72BC3
:106D300081879287A387B487DF91CF910895CF92FF
:106D4000DF92EF92FF920F931F93CF93DF9300D0C8
:106D500000D01F921F92CDB7DEB76C017B0160FFA0
:106D600003C0E894E0F8F3F8F3FC0DC00E94521160
:106D7000663971058105910530F0809197069091F3
:106D800098060597E9F4B70166277370C6010E945B
:106D9000793660E278E080E799E00E94BF738FEF78
:106DA0009FEF28960FB6F894DEBF0FBECDBFDF91E0
:106DB000CF911F910F91FF90EF90DF90CF900895AA
:106DC00019821A821B821C821D821E821F821886D3
:106DD0008A818F708A8340E053E0B601CE0101962C
:106DE0000E941E2E60E073E0C6010E949117E82AFF
:106DF000F92A09811A812B813C814D815E816F8145
:106E00007885C6010E945895CCCF2F923F924F9221
:106E10005F926F927F928F929F92AF92BF92CF922A
:106E2000DF92EF92FF920F931F93CF93DF93CDB733
:106E3000DEB7CC5BD1090FB6F894DEBF0FBECDBF75
:106E40004C01C755DF4F0883C95AD040C655DF4FA4
:106E50001883CA5AD040C555DF4F2883CB5AD0403B
:106E6000C455DF4F3883CC5AD040C355DF4F4883D9
:106E7000CD5AD040C255DF4F5883CE5AD040C1556D
:106E8000DF4F6883CF5AD040C055DF4F7883C05B57
:106E9000D040CF54DF4FF982E882C15BD0402C2C28
:106EA0000E946F94C754DF4F688379838A839B83E2
:106EB000C95BD040C655DF4F8881CA5AD0408F7019
:106EC000682E712CC0909706D0909806C954DF4F59
:106ED000D982C882C75BD040CF54DF4FE881F981A7
:106EE000C15BD040309721F0808181110C948441A6
:106EF000D4011B968C91882341F0C4010B96CF548A
:106F0000DF4F99838883C15BD0406114710411F015
:106F10000C94CD41CF54DF4FE881F981C15BD04063
:106F2000309711F00C948841F401658876886114DB
:106F3000710411F40C94CD41C655DF4F8881CA5AB3
:106F4000D0408F7011F00C94CD41662DCE01875545
:106F50009F4F0E94FC2EC756DF4F2883C959D0404F
:106F6000C656DF4F3883CA59D040C556DF4F4883D5
:106F7000CB59D040C456DF4F5883CC59D040C3566C
:106F8000DF4F6883CD59D040C256DF4F7883CE594A
:106F9000D040C156DF4F8883CF59D040C056DF4F15
:106FA0009883C05AD0400C94CD41F40180819181E6
:106FB000009709F440C2FDE06F16710409F0ACC0FF
:106FC0000E94A889082F10E006301105A4F40E9441
:106FD0005A77009739F0DC0118962C911897207F8A
:106FE00018962C93BC01F401808191810E947A89CA
:106FF0000F5F1F4FE9CF65E0D4018D919C910E94F6
:10700000D4848C01892BE9F410E000E0C801C45459
:10701000DF4F0FB6F894DEBF0FBECDBFDF91CF912B
:107020001F910F91FF90EF90DF90CF90BF90AF90A6
:107030009F908F907F906F905F904F903F902F9098
:107040000895C755DF4F8881C95AD0408031E0F696
:10705000CE0187559F4F0E94452F1616170618061A
:10706000190624F4F80180858D70A1F0D8011896D6
:107070008C9118978F7018968C9369E777E080E76A
:1070800099E00E94BF7380E799E00E94C87201E016
:1070900010E0BCCF0E946F946B017C01CE0187553C
:1070A0009F4F0E94452FC60ED71EE81EF91EF801FD
:1070B000C186D286E386F486C755DF4F8881C95AD8
:1070C000D0408295807F826080876EE677E080E79F
:1070D00099E00E94BF73CE0187559F4F0E94452FB4
:1070E000AB01BC012AE030E080E799E00E94D37256
:1070F00068E677E080E799E00E94BF73D8011996AF
:107100004D915D916D917C911C972AE030E080E774
:1071100099E00E94D372B7CFC755DF4FF880C95AA4
:10712000D040B4E0FB1609F4E0C2BF1530F0FF20F8
:1071300009F476C0B12CA12C95C288EF8F0D823056
:10714000C8F788E0FE01E755FF4FDE011196019078
:107150000D928A95E1F7C655DF4F8881CA5AD04013
:10716000807F09F415C3CE0187559F4F0E94452F9C
:107170008B01672B09F40CC389E0F81203C0119549
:1071800001951109B401CE0187559F4F0E94D789FF
:1071900060E0CE0187559F4F0E94232F6A962FAF44
:1071A0006A976B963FAF6B976C964FAF6C976D96E7
:1071B0005FAF6D976E966FAF6E976F967FAF6F975D
:1071C000A0968FAFA097A1969FAFA19792E0691666
:1071D000710409F428C30CF0DEC2CC24C3946114FA
:1071E000710409F0A7CFC655DF4FE881CA5AD040D5
:1071F000E295EF70E150EB3008F09BC3F0E0882798
:10720000EB5FF64C8F4F0C94B8C1153C153C993C84
:10721000993C993C743C503C503C503C323C323C94
:1072200019821A821B821C821D821E821F8218866E
:107230008A818F708A83C655DF4F8881CA5AD040B1
:10724000807F09F477CFE9E06E16710409F40CC26F
:107250000CF0F4C06114710409F414C122E0621648
:10726000710409F067CFB12CA12CC12C33243A94BE
:10727000B401CE0101960E94D7898A81982F9295F8
:107280009F70945F9F70923060F4C655DF4F988175
:10729000CA5AD04092959F70923019F48F708062D4
:1072A0008A83D40118969C91973071F4C655DF4FAC
:1072B0008881CA5AD040807E803211F0803421F417
:1072C0008A818F7080628A83F401A185B285892FBB
:1072D00090E0109741F0ED91FC911197028CF38DA5
:1072E000E02DCD0119957C01C755DF4F0881C95AA2
:1072F000D040C655DF4F1881CA5AD040C555DF4F20
:107300002881CB5AD040C455DF4F3881CC5AD04069
:10731000C355DF4F4881CD5AD040C255DF4F588109
:10732000CE5AD040C155DF4F6881CF5AD040C055AA
:10733000DF4F7881C05BD040CE0101960E94C52FFF
:10734000CF57DF4F2883C158D040CE57DF4F388307
:10735000C258D040CD57DF4F4883C358D040CC5798
:10736000DF4F5883C458D040CB57DF4F6883C55890
:10737000D040CA57DF4F7883C658D040C957DF4F37
:107380008883C758D040C857DF4F9883C858D0402B
:10739000CE0101960E94C02CCC2051F1C655DF4F82
:1073A0008881CA5AD04082958F709FE0980F9F7055
:1073B000923020F08A5F8F708230D0F48A8182957B
:1073C0008F7081508230A0F42D8130E0AFEFB0E0BB
:1073D0000E9481C12FEF6115F4E67F0781059105B9
:1073E00034F424E630E040E050E00E944FC12D83A9
:1073F00088E0FE013196DE01A755BF4F01900D9246
:107400008A95E1F72AE0B22AD12CD40118968C9102
:10741000873009F013C4BEE54B16B1E05B060CF0F3
:10742000F5C262E477E089EC98E00E94BF7389ECD2
:1074300098E00E94C8720FEF1FEFE8CD8AE068164F
:10744000710409F4BFC09BE06916710409F072CEA3
:10745000B401CE0101960E94D789CE0187559F4F76
:107460000E94F811BC01CE0101960E948A2F88E08B
:10747000FE013196DE01A755BF4F01900D928A950E
:10748000E1F7EDC0C4010E948F4A8C0161E070E019
:107490001816190614F070E060E080E799E00E9489
:1074A000A08967EC73E080E799E00E945973CE01F0
:1074B00087559F4F0E94452FAB01BC012AE030E069
:1074C00080E799E00E94D37280E799E00E94C87239
:1074D000CE0187559F4F101611060CF00BC70E9466
:1074E000452FB12CA12C672B682B692B89F562E005
:1074F000CE0187559F4F0E94232FCF56DF4F288301
:10750000C159D040CE56DF4F3883C259D040CD56F6
:10751000DF4F4883C359D040CC56DF4F5883C459FE
:10752000D040CB56DF4F6883C559D040CA56DF4F95
:107530007883C659D040C956DF4F8883C759D04099
:10754000C856DF4F9883C859D040AA24A394BA2CB8
:10755000CC24C394332433948BCE61E0CE01875581
:107560009F4F0E94232FC757DF4F2883C958D04011
:10757000C657DF4F3883CA58D040C557DF4F4883BE
:10758000CB58D040C457DF4F5883CC58D040C35756
:10759000DF4F6883CD58D040C257DF4F7883CE5835
:1075A000D040C157DF4F8883CF58D040C057DF4FFE
:1075B0009883C059D040AA24A394BA2CCC24C39455
:1075C000312C56CEB401CE0101960E94D789C25506
:1075D000DF4F8881CE5AD0409A8192959F7041F0BA
:1075E000923051F0B12CA12CDD24D394C12C37C1A1
:1075F0009A819F7090629A8390E08536910514F08D
:1076000084E690E08E8388E0FE013196DE01A75586
:10761000BF4F01900D928A95E1F762E0CE01875548
:107620009F4F0E94FC2EEA962FAFEA97EB963FAF52
:10763000EB97EC964FAFEC97ED965FAFED97EE962C
:107640006FAFEE97EF967FAFEF97C158DF4F88830C
:10765000CF57D040C058DF4F9883C058D040A12C9E
:10766000EAE0BE2ED12CC2CFB401CE0101960E9419
:10767000D789C155DF4F6881CF5AD040C055DF4F01
:107680007881C05BD0407170CE0101960E944A346F
:10769000C82E882309F457C188E0FE013196DE0127
:1076A000A755BF4F01900D928A95E1F762E0CE0198
:1076B00087559F4F0E94FC2EE2962FAFE297E396EC
:1076C0003FAFE397E4964FAFE497E5965FAFE5975A
:1076D000E6966FAFE697E7967FAFE797E8968FAFAE
:1076E000E897E9969FAFE997BACFC4010E948F4A05
:1076F000181619063CF562E0CE0187559F4F0E948F
:10770000232FAA962FAFAA97AB963FAFAB97AC9615
:107710004FAFAC97AD965FAFAD97AE966FAFAE97EC
:10772000AF967FAFAF97E0968FAFE097E1969FAFB0
:10773000E197AA24A394BA2CD12CCC24C39433244B
:10774000339463CE61E0CE0187559F4F0E94232F73
:10775000A2962FAFA297A3963FAFA397A4964FAF41
:10776000A497A5965FAFA597A6966FAFA697A79685
:107770007FAFA797A8968FAFA897A9969FAFA99715
:10778000AA24A394BA2CD12CCC24C394312C3DCE62
:1077900005E010E0F1CCB9E06B16710409F4D8C033
:1077A000EAE06E16710409F0C5CCC655DF4F88813A
:1077B000CA5AD04082958F70823009F01CC1C255E0
:1077C000DF4F6881CE5AD040060F111D17FF02C04F
:1077D00010E000E00536110514F004E610E0C25593
:1077E000DF4F0883CE5AD04062E0CE0187559F4FCD
:1077F0000E94FC2E2A962FAF2A972B963FAF2B97ED
:107800002C964FAF2C972D965FAF2D972E966FAF7E
:107810002E972F967FAF2F9760968FAF60976196C8
:107820009FAF61971CCFC12CDECCC355DF4F688161
:10783000CD5AD040060F111D17FF02C010E000E026
:107840000F3F110519F014F00FEF10E0C355DF4F93
:107850000883CD5AD040A12C5AE0B52ED12C332428
:107860003A94D3CDC355DF4F68817981CD5AD0404A
:10787000060F171F17FF02C010E000E005361105C4
:1078800014F004E610E0012E000C220B330BC3555C
:10789000DF4F088319832A833B83CD5AD040DBCF47
:1078A000C355DF4F688179818A819B81CD5AD04051
:1078B0000E94B5C2600F711F77FF02C070E060E0E8
:1078C0006536710514F064E670E0072E000C880B35
:1078D000990B0E94EABFC355DF4F688379838A837F
:1078E0009B83CD5AD040B7CFC355DF4F2881398114
:1078F000CD5AD0404AE0409FC001419F900D1124D5
:10790000820F931F97FF02C090E080E0893EF3E072
:107910009F0714F088EE93E0092E000CAA0BBB0B16
:10792000C355DF4F88839983AA83BB83CD5AD04048
:1079300092CF88E0FE013196DE01A755BF4F01903E
:107940000D928A95E1F7B12CA12CDD24D39487CF39
:10795000C655DF4F8881CA5AD04082958F708230D9
:1079600009F049C0C155DF4F6881CF5AD040C0559A
:10797000DF4F8881C05BD040782F7170060F171FD2
:107980000E3621E012072CF417FF05C00DE611E0BA
:1079900002C010E000E0C155DF4F0883CF5AD0404D
:1079A000C055DF4F8881C05BD04010FB80F9C055C7
:1079B000DF4F8883C05BD04062E0CE0187559F4F88
:1079C0000E94FC2E62962FAF629763963FAF63973B
:1079D00064964FAF649765965FAF659766966FAF95
:1079E000669767967FAF679768968FAF6897699637
:1079F0009FAF699734CE88E0FE013196DE01A7552E
:107A0000BF4F01900D928A95E1F7ECCD2220E1F075
:107A1000D4011296ED91FC9190859F709530A1F460
:107A2000C954DF4F88819981C75BD040059761F0C9
:107A3000CF54DF4F48815981C15BD040BE016755AB
:107A40007F4FCF010E94CF49C755DF4F8881C95A68
:107A5000D040853009F4CAC020F4833079F1C501E3
:107A60006CC0863009F47CC08730C9F7C4010E941D
:107A7000DB17182F863009F062C062E277E080E7FA
:107A800099E00E94BF7366E070E080E799E00E9491
:107A9000A08980E799E00E94C87262E0CE01875514
:107AA0009F4F0E94232F29AF3AAF4BAF5CAF6DAF12
:107AB0007EAF8FAF21969FAF21973CC0C4010E943B
:107AC000DB17853019F00DEF1FEFA0CA63E377E0F5
:107AD00080E799E00E94BF7365E070E080E799E07D
:107AE0000E94A08980E799E00E94C872B401CE018B
:107AF00087559F4F0E94D78961E0CE0187559F4FE0
:107B00000E94232F22962FAF229723963FAF2397D1
:107B100024964FAF249725965FAF259726966FAF93
:107B2000269727967FAF279728968FAF2897299675
:107B30009FAF2997C50181609160312C30C06AE008
:107B400077E080E799E00E94BF73612F70E080E7E3
:107B500099E00E94A08980E799E00E94C872B3CFA3
:107B6000C4010E948F4A18161906CCF1B401CE0147
:107B700087559F4F0E94D78961E0CE0187559F4F5F
:107B80000E94232F29AB3AAB4BAB5CAB6DAB7EAB0A
:107B90008FAB98AFC5018160916046E0342E5C01E7
:107BA0006894A0F8C655DF4F2881CA5AD040322FBA
:107BB0003F70323058F4C755DF4F3881C95AD04032
:107BC000332321F05C016894A0F8B0F8207F59F1CC
:107BD0006894B1F801E010E0D11039C438C266EF02
:107BE00076E080E799E00E94BF736DCFC4010E94E8
:107BF0008F4A18161906A4F462E0CE0187559F4FEC
:107C00000E94232F29A73AA74BA75CA76DA77EA7A1
:107C10008FA798ABC5018160916035E0332EBFCF4F
:107C20006FED76E0DECF40E052E0B401CE01875543
:107C30009F4F0E941E2E8111CBCFCCCF9FEF3912C8
:107C4000B1C0C4010E948F4A332433941816190618
:107C50000CF4ABC0312C67ED76E080E799E00E9430
:107C6000BF73E32C032C000CFF08CD54DF4FF982C7
:107C7000E882C35BD040B70180E799E00E94A08909
:107C800060ED76E080E799E00E94BF736C2D70E0B4
:107C900080E799E00E94A08980E799E00E94C8727D
:107CA000CF54DF4F48805980C15BD040411451040C
:107CB00009F484C06EE87EE1C2010E9483B801E04D
:107CC00010E0892B09F44BC06AE87EE1C2010E94F2
:107CD00083B802E010E0892B09F441C06EE176E040
:107CE000C2010E9483B805E010E0892BC1F16AE16E
:107CF00076E0C2010E9483B806E010E0892B79F19A
:107D00006FE47EE1C2010E9483B80AE010E0892B93
:107D100031F16AE47EE1C2010E9483B80BE010E019
:107D2000892BE9F064E57EE1C2010E9483B80CE092
:107D300010E0892BA1F06DE37EE1C2010E9483B8BF
:107D40000DE010E0892B59F066E47EE1C2010E944B
:107D500083B810E000E0892B11F40EE010E0C401BC
:107D60000E94DB17E82EF12CE114F10431F4CD541C
:107D7000DF4FE880F980C35BD0400115110509F49D
:107D80003CC0E016F106A1F06AEB76E080E799E0EE
:107D90000E94BF73B70180E799E00E94A08980E745
:107DA00099E047CB332009F456CFCC24C39453CF6A
:107DB000CF54DF4F19821882C15BD040C755DF4FC7
:107DC0009881C95AD0409F3008F02AC1E92FF0E0CD
:107DD0008827E251F14C8F4F0C94B8C11F40EB3F04
:107DE000DC3F363F1F40C33FA03F783F1F401F404E
:107DF000F83FF83FF83FF83FF83FD40119968D91CE
:107E00009C91009709F400C9DC01ED91FC91048874
:107E1000F589E02D7201C755DF4F0881C95AD0405E
:107E2000C655DF4F1881CA5AD040C555DF4F28814B
:107E3000CB5AD040C455DF4F3881CC5AD040C355BF
:107E4000DF4F4881CD5AD040C255DF4F5881CE5ABE
:107E5000D040C155DF4F6881CF5AD040C055DF4F69
:107E60007881C05BD04019958C01D0C8C4010E94B4
:107E7000DB17853009F027CE6BEA76E080E799E0E2
:107E80000E94BF7365E070E080E799E00E94A089DE
:107E900080E799E00E94C872B401CE0187559F4FD8
:107EA0000E94D789F4018085853099F46CE0CE0179
:107EB00087559F4F0E94232F29A33AA34BA35CA36E
:107EC0006DA37EA38FA398A76894A0F8B0F8312C77
:107ED00052C061E0CE0187559F4F0E94232F298F0A
:107EE0003A8F4B8F5C8F6D8F7E8F8F8F98A3ECCFE7
:107EF000C4010E94DB17182F8630F9F46AE976E096
:107F000080E799E00E94BF7366E070E080E799E047
:107F10000E94A08980E799E00E94C87262E0CE01C9
:107F200087559F4F0E94232F298B3A8B4B8B5C8B5D
:107F30006D8B7E8B8F8B988FC7CF62E876E001CEFA
:107F400031101EC0B401CE0187559F4F0E94D789C2
:107F500061E0CE0187559F4F0E94232F29873A87E2
:107F60004B875C876D877E878F87988B6894A0F896
:107F7000B0F826E0322E0FEF1FEFCC24C3942CCEA6
:107F80006EE676E02ECE3320A1F062E0CE0187557A
:107F90009F4F0E94232F29833A834B835C836D83F9
:107FA0007E838F8398876894A0F8B0F895E0392E87
:107FB000E2CF67E576E015CEC655DF4F8881CA5A15
:107FC000D0408F708230C8F5C4010E94DB17853025
:107FD00009F07ACF78CDC655DF4F8881CA5AD04094
:107FE0008F70823050F5332019F064E476E0F9CDDB
:107FF000C655DF4F8881CA5AD040282F2F702230B3
:10800000E0F49923D1F0807F31F4B401CE0187559B
:108010009F4F0E94D7896894A0F8F3E0BF2A57CFFA
:10802000C655DF4F8881CA5AD040807F19F46894C2
:10803000B0F84DCF23E0B22A4ACFCC24C394D1105C
:1080400006C2312C0FEF1FEFA114B10439F0A501C6
:10805000B401CE0187559F4F0E94AC2DD4011996D3
:108060008D919C91009709F473C0CF54DF4FE88045
:10807000F980C15BD040DC01ED91FC910488F58969
:10808000E02DC755DF4F0881C95AD040C655DF4F94
:108090001881CA5AD040C555DF4F2881CB5AD040ED
:1080A000C455DF4F3881CC5AD040C355DF4F48818B
:1080B000CD5AD040C255DF4F5881CE5AD040C1551D
:1080C000DF4F6881CF5AD040C055DF4F7881C05B09
:1080D000D04019958C01332021F0632DC4010E94FA
:1080E000AB17C954DF4FE881F981C75BD0403597A2
:1080F00021F0B501C4010E949F366AE276E080E774
:1081000099E00E94BF73B80180E799E00E94A089BE
:1081100063E276E080E799E00E94BF730E946F946B
:10812000AB01BC01C754DF4FC880D980EA80FB8017
:10813000C95BD0404C195D096E097F0980E799E061
:108140000E94968980E799E00E94C8720C940638D4
:10815000F4018085853009F462C0863009F0BBCF18
:10816000C4010E94B5897C01009709F4B4CF712C39
:10817000612C97FF06C0F194E194F10866246394A2
:10818000712CC70101978634910508F0A4CFC7551B
:10819000DF4F0881C95AD04010E0DE2C61E08E2DFF
:1081A0000E94B990672859F10130110521F061E072
:1081B0000C30110509F460E0062F10E08D2D0E94AF
:1081C0008B906FE376E080E799E00E94BF73B70180
:1081D00080E799E00E94A0896DE376E080E799E06E
:1081E0000E94BF73B80180E799E00E94A08980E7F0
:1081F00099E00E94C8726894A0F8B0F874C0013089
:10820000110551F091E080E00C30110509F090E08B
:10821000092F182F602FD2CF01E010E0FBCFF2E042
:108220006F16710409F462C02CE06216710429F023
:108230006A94672809F04FCFDECFC4010E947517FA
:10824000892B49F4D401ED91FC916081718180EF1B
:1082500093E00E94A997CE0187559F4F0E94B111CC
:1082600020E030E048EC52E40E9449C00E94B5C2D0
:10827000CD54DF4F688379838A839B83C35BD0406F
:10828000CD54DF4F48805980C35BD04088E00E94C6
:1082900044146B017C0169E376E080E799E00E9479
:1082A000BF73CD54DF4F68817981C35BD04080E7D5
:1082B00099E00E94A08964E376E080E799E00E945B
:1082C000BF73B701A601662777272AE080E799E008
:1082D0000E947C7280E799E00E94C872B601A201F8
:1082E000C4010E94F71A01E010E0F5CE6894A0F8EE
:1082F000B1F8F9CF0E94452F672B682B692B09F045
:108300002CC9B12CA12C5AC96114710409F045C0C3
:108310008081882311F40C949437CE018F549F4FA1
:108320000E9469343C01C655DF4F8881CA5AD0404B
:108330008F7071F5662DCE0187559F4F0E94FC2EE0
:10834000CF55DF4F2883C15AD040CE55DF4F3883F9
:10835000C25AD040CD55DF4F4883C35AD040CC5588
:10836000DF4F5883C45AD040CB55DF4F6883C55A7E
:10837000D040CA55DF4F7883C65AD040C955DF4F29
:108380008883C75AD040C855DF4F9883C85AD04019
:108390006114710411F40C9494370E9452116B0112
:1083A0002B0168EB77E080E799E00E94BF73B6018C
:1083B00080E799E00E94A08961EB77E080E799E08F
:1083C0000E94BF73D401ED91FC916081718180E7BF
:1083D00099E00E9459736BEA77E080E799E00E9488
:1083E000BF73CF54DF4F68817981C15BD04080E794
:1083F00099E00E94597365EA77E080E799E00E946E
:10840000BF7367E977E0B8ECCB16D10414F40C9491
:10841000133ACE0187559F4F0E94C02CCF54DF4F97
:10842000E881F981C15BD040309711F40C94D537C5
:108430008081843211F00C94D53763E877E080E7CF
:1084400099E00E94BF7380E799E00E94C8720CEF28
:108450001FEF0C9406382F923F924F925F926F92CB
:108460007F928F929F92AF92BF92CF92DF92EF92C4
:10847000FF920F931F93CF93DF93CDB7DEB7C9550C
:10848000D1090FB6F894DEBF0FBECDBF3C01562E0A
:108490006296EFAE62976396FFAE639764960FAFF6
:1084A000649765961FAF659766962FAF6697679638
:1084B0003FAF679768964FAF689769965FAF6997C8
:1084C0006A96CFAE6A972D2C4A2C3B2C009709F464
:1084D0005CC1FC0180858295807F85958595859519
:1084E0008595843009F43CC12CF4882309F441C1FA
:1084F00080E02DC0853009F444C08630C9F76FEFA5
:1085000073E0C3010E945F844C01009709F46FC0BF
:10851000B12CA12CD12CC12C6296EFAC6297639642
:10852000FFAC639764960FAD649765961FAD659732
:1085300066962FAD669767963FAD679768964FAD85
:10854000689769965FAD6997652D0E942B42C75A5F
:10855000DF4F0FB6F894DEBF0FBECDBFDF91CF91D6
:108560001F910F91FF90EF90DF90CF90BF90AF9051
:108570009F908F907F906F905F904F903F902F9043
:10858000089580918D068F5F80938D0686809780F9
:108590008114910431F1A42CB32C6A96CFAC6A9764
:1085A000D22C6296EFAC62976396FFAC63976496A9
:1085B0000FAD649765961FAD659766962FAD66976C
:1085C00067963FAD679768964FAD689769965FADC0
:1085D0006997652DC4010E942B42F401828093802B
:1085E000D7CF80918D06815080938D0681CF63E037
:1085F00074E0C3010E945F847C0168E074E0C30101
:108600000E945F846C01552039F0F1E05F1609F497
:1086100088C010E000E00CC06DE074E0C3010E946F
:108620005F844C0162E174E0C3010E945F848C01AD
:108630008114910409F443010115110509F4830122
:10864000E114F10421F46A96EFAC6A97F22CC1149C
:10865000D10411F4C42CD32C8114910409F492C0D8
:10866000F40180858F70843009F08CC081849284FD
:108670000115110509F491C0F80180858F708430CF
:1086800009F08BC001851285E114F10409F4C9C019
:108690008114910409F490C063E574E180E799E0E6
:1086A0000E94BF73F7016185728580E799E00E949F
:1086B00059736EE474E180E799E00E94BF73B401DE
:1086C00080E799E00E94597380E799E00E94C872A0
:1086D000CE018F5A9F4F0E94C02CC114D10409F0C3
:1086E000F8C0F70180858F70843009F0F0C0618593
:1086F0007285CE0101960E949D34CE0101960E94A2
:108700001A12882349F08114910409F469C0B40154
:10871000CE0101960E946A8ACE0101960E945012F3
:10872000D6C067E174E0C3010E945F844C016CE134
:1087300074E0C3010E945F848C018114910409F0EC
:10874000CDC06DE074E0C3010E945F844C0101154F
:10875000110509F467CF892B09F072CF430170CF5F
:1087600010E000E0912C812CD12CC12CF12CE12CBB
:108770005FCF10E000E0912C812CD12CC12CF12C8A
:10878000E12C5ECF912C812C73CFCA2CDB2C6A9606
:10879000EFAC6A97F22C912C812C00E020E033E0C2
:1087A00040E150E0BE016F5B7F4FCE018F5A9F4F7B
:1087B0000E94D52A8C0168CF64E474E180E799E0D7
:1087C0000E94BF73F7016185728580E799E00E947E
:1087D00059736FE374E180E799E00E94BF7378CF2B
:1087E000CC24C394F12CE12C62960FAD6297639672
:1087F0001FAD639764962FAD649765963FAD6597FF
:1088000066964FAD669767965FAD679768966FAD52
:10881000689769967FAD6997CE0101960E940537EA
:108820007BCFC114D10409F452C00115110509F41C
:108830004EC0F60180858F70843009F044C068E333
:1088400074E180E799E00E94BF73F601618572854B
:1088500080E799E00E94597363E374E180E799E04F
:108860000E94BF73B80180E799E00E94597380E7C6
:1088700099E00E94C872F6016185728540E450E07B
:10888000CE0101960E9447C60E947A848823D9F0BF
:108890008091FE07811117C06FE270E0CE01019652
:1088A0000E940EC6892B51F4F6012185328543E0E2
:1088B00050E060E4CE0101960E942624B801CE016A
:1088C00001960E943D95E114F10409F00ACF81E080
:1088D0003ECE0115110509F0ACCF03CF892B09F06D
:1088E000AFCEA0CE8F929F92AF92BF92CF92DF92E7
:1088F000EF92FF920F931F93CF93DF93CDB7DEB725
:10890000E0970FB6F894DEBF0FBECDBF84E0E0E184
:10891000F2E0DE01119601900D928A95E1F7FE01D9
:1089200035968CE1DF011D928A95E9F7CE0101961B
:10893000DB01685F7F4FFD900F2D10E0E4E015959F
:108940000795EA95E1F70E5A1D4FF8011081FC01D9
:108950001083EF2DEF70F0E0EE5AFD4F1081FC0117
:10896000118302966A177B0731F7198A1A8A809158
:10897000B0059091B105892B09F46CC069017A01A9
:1089800080E799E00E94C87263E17AE080E799E0AD
:108990000E94BF7342E0C701B6010E94648D61E18D
:1089A0007AE080E799E00E94BF73BE016F5F7F4F5E
:1089B00080E799E00E9459736FE07AE080E799E0E0
:1089C0000E94BF7380E799E00E94C872BE016F5F8A
:1089D0007F4F80919B0690919C060E945F844C0182
:1089E00020E030E04EEF52ECC701B6010E94E3BF39
:1089F000882381F120E030E04AEA52E4C701B60161
:108A00000E94E3BF882331F120E030E0A901C701D3
:108A1000B6010E94E3BF8823E9F019A61AA61BA697
:108A20001CA68AA58F7080678AA7CDA6DEA6EFA6B2
:108A3000F8AA6CE0CE0189960E94FC2EB12CA12CE4
:108A4000D12CC12C79018A019B01AC016FEFC401CB
:108A50000E942B42E0960FB6F894DEBF0FBECDBF4A
:108A6000DF91CF911F910F91FF90EF90DF90CF900A
:108A7000BF90AF909F908F9008956F927F928F924A
:108A80009F92AF92BF92CF92DF92EF92FF920F939D
:108A90001F93CF93DF93CDB7DEB7A0970FB6F894AF
:108AA000DEBF0FBECDBF8C01862E7A01DC018D9119
:108AB0009C911197892B09F460C01496ED91FC915B
:108AC000309709F45AC080818071BFEF6B1357C093
:108AD000B1F481E0A0960FB6F894DEBF0FBECDBF13
:108AE000DF91CF911F910F91FF90EF90DF90CF908A
:108AF000BF90AF909F908F907F906F90089543307C
:108B0000510539F3818082942FE082226AEC75E06E
:108B100080E799E00E94BF73D80113966C9180E7BB
:108B200099E00E94998968EC75E080E799E00E94DD
:108B3000BF73D8011496ED91FC9161816F7080E74D
:108B400099E00E94998965EC75E080E799E00E94C0
:108B5000BF73682D80E799E00E94998980E799E0CA
:108B60000E94C872D8011496ED91FC9181818F709A
:108B7000881207C080818F7E808380E0ABCF811117
:108B8000FCCF198E1A8E1B8E1C8E1D8E1E8E1F8E74
:108B900018A28A8D8F708A8FD8011496ED91FC915E
:108BA00081818F70881579F1B3E0EB16F10459F1EA
:108BB00063EC75E080E799E00E94BF73F801638180
:108BC00080E799E00E94998961EC75E080E799E07F
:108BD0000E94BF73D8011496ED91FC9161816F7072
:108BE00080E799E00E9499896EEB75E080E799E053
:108BF0000E94BF73682D80E799E00E94998980E701
:108C000099E00E94C872F80120813181FCE0F815DA
:108C100008F416C1E82DF0E08827EE5EF94B8F4F7F
:108C20000C94B8C11F465C46DD46F4460047DD465D
:108C3000B646DD4603470E47CA4611471D47D801D1
:108C40001496CD90DC90F60181818F70853009F407
:108C5000F7C050F48230C1F06FE274E0C9010E94A5
:108C60005F843C01912C4BC08730D1F08A30A1F752
:108C700068E274E0C9010E945F843C01D6019C90C7
:108C800092FA992490F83BC062E274E0C9010E9414
:108C90005F843C01D6019C9090FA992490F82FC0F3
:108CA00061E274E0C9010E945F843C01F60190809A
:108CB00091FA992490F823C064E374E0C9010E94FA
:108CC0005F843C01D8011496ED91FC91808180FB7A
:108CD000992490F8982F9E7F80FF91609083611473
:108CE000710469F461E0CE0149960E94232F298B1B
:108CF0003A8B4B8B5C8B6D8B7E8B8F8B988FF801B7
:108D0000A080B18063E074E0C5010E945F846C01C3
:108D100068E074E0C5010E945F845C01892B81F4E6
:108D2000C114D10469F460E0CE0149960E94232F5A
:108D300029833A834B835C836D837E838F839887FB
:108D4000D8011496ED91FC916114710409F07CC076
:108D5000898D811179C0B82DBF708B2E8181807F64
:108D6000882A818280818F7E8083B3CE69E374E01C
:108D7000C9010E945F843C01D8011496ED91FC91D9
:108D8000808181FB992490F8982F9D7F81FF9260CC
:108D90009083B5CF6FE374E0C9010E945F843C010A
:108DA000D8011496ED91FC91808182FB992490F872
:108DB000982F9B7F82FF9460EBCF6FE274E0C90134
:108DC0000E945F843C01892B09F04CCF62E0CE0108
:108DD00049960E94232F29873A874B875C876D87A6
:108DE0007E878F87988B3ECF65E474E0C9010E942F
:108DF0005F843C01D8011496ED91FC9190804CCF9A
:108E00006AE474E0F3CF60E574E0C9010E945F8416
:108E10003C01D8011496ED91FC9149CF66E574E0D0
:108E2000F4CF6DE574E0C9010E945F843C01D80174
:108E30001496ED91FC91908023CF63E674E0F3CF1C
:108E4000912C712C612C5BCF83E0E816F104B9F012
:108E5000982D9F70892E8181807F882A81828081D0
:108E60008F7E8083E98CFA8C0B8D1C8D2D8D3E8D31
:108E70004F8D58A1692DC3010E942B422ACE8181BA
:108E80008F70881509F425CE829490EF8922882A64
:108E900081828081806168CF2F923F924F925F9252
:108EA0006F927F928F929F92AF92BF92CF92DF92FA
:108EB000EF92FF920F931F93CF93DF93CDB7DEB75F
:108EC000A3970FB6F894DEBF0FBECDBF5C011B01A8
:108ED000D0909805DD2009F4B8C080918D068F5F91
:108EE00080938D06E0919906F0919A06309709F4E7
:108EF000A4C0868097806090990670909A0661144D
:108F0000710409F496C08114910409F492C0D4014B
:108F100018968C918F70853091F7C4010E94A889B2
:108F2000823068F3B401CE0101960E94E11ACE01AD
:108F300001960E941A12882309F45EC060E074E072
:108F4000CE0101960E949117892B09F455C0188E05
:108F5000198E1A8E1B8E1C8E1D8E1E8E1F8E898D55
:108F60008F70898F40E053E0BE016F5F7F4FCE016D
:108F700048960E941E2E6CEF77E080E799E00E94F1
:108F8000BF7360E074E0CE0101960E9455368A8579
:108F90009B85009789F1DC01ED91FC910488F589AE
:108FA000E02DCC24C394F12CE12C088D198D2A8D51
:108FB0003B8D4C8D5D8D6E8D7F8D19958F3F980704
:108FC000D9F0E981FA8160817181892BE9F480E728
:108FD00099E00E9459736AEF77E080E799E00E9478
:108FE000BF7362EF77E080E799E00E94BF7380E78C
:108FF00099E00E94C872D12CF40182809380CE0146
:1090000001960E94501277CF80E799E00E94597331
:1090100060EF77E080E799E00E94BF736CEE77E045
:1090200080E799E00E94BF7380E799E00E94C872D0
:10903000E3CF80E799E00E94C87280918D0681504D
:1090400080938D06D1101092980565E0D5018D9121
:109050009C910E94D4844C01009709F489C0FC01C2
:10906000D084D594D594D594D59441845284638486
:1090700074840E946F94DD2009F47AC0461A570A5E
:10908000680A790A188E198E1A8E1B8ED88E198D41
:109090001F70106A198F4C8E5D8E6E8E7F8EC3018D
:1090A000B20128EE33E040E050E00E944FC128A317
:1090B00039A34AA35BA3672B682B692B09F5E12C25
:1090C00090E1F92E0D2D2A8D3B8D4C8D5D8D6E8D91
:1090D0007F8DC5010E9458952AE030E048A159A132
:1090E0006AA17BA180E799E00E94D37261E178E0F8
:1090F00080E799E00E94BF7380E799E00E94C87200
:1091000077FE36C0F2E04F1651046104F0E87F06A6
:109110007CF1E12C80E1F82E088D198D2A8D3B8D94
:109120004C8D5D8D6E8D7F8DC5010E945895198285
:109130001A821B821C821D821E821F8218861A813F
:109140001F701A83D982CC24C394F12CE12C0D2DED
:109150002B813C8140E05E816F817885C5010E9452
:109160000537D40118968C9118978F7018968C93A8
:10917000B1E02B163104B9F460E073E0C5010E9440
:109180009117009781F0209197063091980626302C
:10919000310549F4BC01C5010E949F3660E073E0CF
:1091A000C5010E945536F501818592850097D9F455
:1091B00090E080E0A3960FB6F894DEBF0FBECDBF5F
:1091C000DF91CF911F910F91FF90EF90DF90CF90A3
:1091D000BF90AF909F908F907F906F905F904F90D7
:1091E0003F902F900895DC01ED91FC910484F5856A
:1091F000E02D1995892BE1F2F50181859285DC013D
:10920000ED91FC910480F581E02DB1011995D2CF4B
:10921000AF92BF92CF92DF92EF92FF920F931F9384
:10922000CF93DF93CDB7DEB767970FB6F894DEBF65
:109230000FBECDBFE0919906F0919A06309709F4E0
:109240009DC080918D068F5F80938D06068117816A
:10925000E0909906F0909A06E114F10431F10115BD
:10926000110519F1F80180858F708530A9F7C801C3
:109270000E94A889823080F3B801CE0101960E9435
:10928000E11ACE0101960E941A12882331F062E0A1
:1092900070E0CE0101960E944C47F80102811381D3
:1092A000CE0101960E945012D3CF80918D0681503D
:1092B00080938D068091970690919806059709F402
:1092C0005DC00E946F949B01AC016091A2057091FA
:1092D000A3058091A4059091A505A12CB12C650151
:1092E00018EEE12E13E0F12E00E010E00E94C423FE
:1092F000082F882309F442C010E06091B2057091F4
:10930000B30561157105D1F1111138C0FB018085DC
:109310008F708530D9F4CE0101960E94E11A61E088
:1093200070E0CE0101960E944C47892B59F00E94B3
:109330006F946093A2057093A3058093A405909306
:10934000A505102FCE0101960E945012E091B205A2
:10935000F091B305309791F0828193819093B3059A
:109360008093B205892B49F6E0919906F0919A060F
:10937000868197819093B3058093B20567960FB667
:10938000F894DEBF0FBECDBFDF91CF911F910F913B
:10939000FF90EF90DF90CF90BF90AF9008954F92E5
:1093A0005F926F927F928F929F92AF92BF92CF9275
:1093B000EF92FF920F931F93CF93DF93CDB7DEB75A
:1093C00067970FB6F894DEBF0FBECDBF009709F4C4
:1093D000A4C0FC0120852F70253009F09EC02A0111
:1093E0005B018680978080918D068F5F80938D06CC
:1093F0008114910409F48CC0F40180858F7084304D
:1094000009F082C0618572858091990690919A06D3
:109410000E945F843C01009709F476C0FC018085BE
:109420008F70853009F070C0B301CE0101960E94A3
:10943000E11AA114B104A9F0CE0101960E941A12FA
:10944000882379F0C12C7201F501008111812281FC
:1094500033814481558166817781CE0101960E94D6
:10946000053760E0C3010E94D4840097D1F1FC016C
:1094700020852F702230A9F581859285A385B4853A
:109480000797A105B10569F561E0C3010E94D48485
:10949000A201B5010E94CF49A114B10489F5882326
:1094A00079F180918D06815080938D06CE010196D1
:1094B0000E94501281E067960FB6F894DEBF0FBE8F
:1094C000CDBFDF91CF911F910F91FF90EF90CF9083
:1094D000BF90AF909F908F907F906F905F904F90D4
:1094E0000895A114B10461F4CE0101960E941A12EC
:1094F000882331F0CE0101960E948F4A892B89F68C
:10950000CE0101960E945012F4018280938070CFA8
:1095100080918D06815080938D0680E0CCCFFF92A4
:109520000F931F93CF93DF9300D000D01F921F9211
:10953000CDB7DEB78C0119821A821B821C821D8274
:109540001E821F8218868A818F708A83D801ED91CE
:10955000FC916081718180E799E00E9459736AEE05
:1095600077E080E799E00E94BF73C8010E941A1259
:10957000811119C061EE77E080E799E00E94BF7326
:1095800080E799E00E94C8720FEF1FEFC80128968C
:109590000FB6F894DEBF0FBECDBFDF91CF911F9104
:1095A0000F91FF900895C8010E94DB17F801908584
:1095B000973039F0853049F1D0F48130E9F08230CC
:1095C00021F1D80119968D919C91009721F1DC0130
:1095D000ED91FC910688F789E02D199501E0892B22
:1095E00009F400E0802F0E94E91410E0CFCF86300C
:1095F00019F08A50833028F762EC77E080E799E031
:109600000E94BF7301E010E0C1CF80E00E94E91426
:1096100010E000E0BBCF40E052E0B801CE0101967F
:109620000E941E2EF8018085873071F160F483302E
:1096300009F451C0843061F062ED77E080E799E091
:109640000E94BF73E5CF883009F445C08930A1F787
:10965000CE0101960E94E1848C0167EC77E080E7FF
:1096600099E00E94BF73B80180E799E00E94A08949
:1096700080E799E00E94C87291E080E0012B09F434
:1096800090E0092F182F82CF0280F381E02D808592
:109690008F70853031F56FED77E080E799E00E94BB
:1096A000BF7350E040E070E060E0F8018281938198
:1096B0000E94CF49F82E082F10E06CED77E080E78C
:1096C00099E00E94BF738F2D0E94E91480E799E012
:1096D0000E94C8725BCFCE0101960E94452F8B017C
:1096E000BCCF10E000E0B9CF2F923F924F925F9233
:1096F0006F927F928F929F92AF92BF92CF92DF92A2
:10970000EF92FF920F931F93CF93DF93CDB7DEB706
:1097100060970FB6F894DEBF0FBECDBFDC01129686
:109720006D917C916115710509F48CC04C01198211
:109730001A821B821C821D821E821F8218868A81C9
:109740008F708A8340E052E0CE0101960E941E2E67
:10975000CE0101960E94E1841C01F4018281938173
:109760000E9475172B013C01D40117962D913D9154
:109770004D915C911A97D1010E9479C12FEF30E091
:1097800040E050E00E942DC129873A874B875C87D3
:109790000E946F949B01AC0189859A85AB85BC853D
:1097A0000097A105B10509F468C0A12CB12C650191
:1097B0007C018D01C301B2010E94C4238987411439
:1097C000510461047104F1F1D40117968D919D91BA
:1097D0000D90BC91A02D8D879E87AF87B88B0E947E
:1097E0006F949B01AC018D859E85AF85B8890097EC
:1097F000A105B10561F0A12CB12C65017C018D01A1
:10980000C301B2010E94C423882309F451C0D401CA
:1098100012966D907C9080E00E944414AB01BC01D4
:10982000C3010E94F71A232869F0F40184810E9481
:109830009111D40116969C91891304C061E0C40172
:109840000E94E81790E080E060960FB6F894DEBFC3
:109850000FBECDBFDF91CF911F910F91FF90EF9081
:10986000DF90CF90BF90AF909F908F907F906F9040
:109870005F904F903F902F90089591E099879FCFF0
:10988000B985BB23F1F060E0C4010E94E817F40140
:10989000828193810E948F4A892BA1F640E050E09B
:1098A000BA01D40112968D919C910E94F71ACACFE9
:1098B000F40184810E949111D40116969C91891320
:1098C000DFCF232809F4BECFF40184810E949111D7
:1098D000D40116969C918913B5CFB985B111B2CF39
:1098E000ADCFCF93DF93EC0162E473E180E799E0C1
:1098F0000E94BF736C817D8180E799E00E94A089FE
:109900006CE373E180E799E00E94BF7380E799E020
:109910000E94C87261E08C810E94B9906E818C8136
:109920000E948B908A819B81009729F040E050E053
:10993000BA010E94F71A81E090E09093B6058093F7
:10994000B5058A819B810E948F4A892B59F40A8030
:10995000DB81C02D80E00E944414AB01BC01CE012C
:109960000E94F71A81E090E0DF91CF9108952F9245
:109970003F924F925F926F927F928F929F92AF929F
:10998000BF92CF92DF92EF92FF920F931F93CF93EC
:10999000DF93CDB7DEB7C955D1090FB6F894DEBF56
:1099A0000FBECDBF0E946F949B01AC016091AA05D0
:1099B0007091AB058091AC059091AD05A12CB12CB7
:1099C000650110E3E12E15E7F12E00E010E00E94A2
:1099D000C423882309F4FFC1E0919906F0919A0607
:1099E000309709F4F8C180918D068F5F80938D06C2
:1099F0002680378010E02114310409F434C1F101CC
:109A000080858F708530F9F460E0C1010E94D484B4
:109A1000FC0181859285A385B4850597A105B105D3
:109A200091F4B101CE0101960E94E11ACE01019696
:109A30000E941A1266968FAF6697811108C0CE01F8
:109A400001960E945012F10122803380D4CF2596D6
:109A50001CAE1DAE1EAE1FAE259729961CAE1DAEC8
:109A60001EAE1FAE299740E052E0BE016F5F7F4FF0
:109A7000CE018F5B9F4F0E941E2ECE0101960E9449
:109A800075176B017C0169966FAF69976A96DFAEB7
:109A90006A97CE0101960E94B5894C01CE018F5B79
:109AA0009F4F0E94B11165966CAF7DAF8EAF9FAF97
:109AB0006597CE0101960E94DB17182FB601DD0CC9
:109AC000880B990B0E94EABF20E030E048EC52E49A
:109AD0000E9443C22B013C01CE0101960E948F4A95
:109AE00068969FAF8EAF689769E972E180E799E069
:109AF0000E94BF7342E065966CAD7DAD8EAD9FADAB
:109B000065970E94648D63E972E180E799E00E94A5
:109B1000BF7342E0C301B2010E94648D6DE872E13F
:109B200080E799E00E94BF73612F70E080E799E0C1
:109B30000E94A089E114F10409F48EC088E00E941B
:109B400044149B01AC0144275527B70190E080E005
:109B5000AA24AA94BA2CC12CD12C17E2E12E19E028
:109B6000F12E00E010E00E94C423882371F1F1017E
:109B70006081718189EC98E00E9459736DE772E110
:109B800089EC98E00E94BF73F101608171818AE6DF
:109B900094E00E94A99790E080E0BC0169964FADE7
:109BA00069976A965FAD6A97CE0101960E94F71A8F
:109BB00062E070E0C4010E94E916CE0101960E94A5
:109BC000501266961FAD66973ECF20E030E048E128
:109BD00052E4C301B2010E94EBC218163CF4F10139
:109BE0006081718186E794E00E94A99768968EADA6
:109BF0009FAD6897892B19F461E070E0DBCF20E01E
:109C000030E040E85FE365966CAD7DAD8EAD9FAD15
:109C100065970E94D6C19B01AC01C301B2010E94AD
:109C2000E3BF70E060E087FDC5CFA30192016596B8
:109C30006CAD7DAD8EAD9FAD65970E94E3BF1816EC
:109C4000DCF66EE672E180E799E00E94BF7380E780
:109C500099E00E94C872B1CF64E672E180E799E0B2
:109C60000E94BF73AACF80918D06815080938D068C
:109C70000E946F946093AA057093AB058093AC0526
:109C80009093AD050E9452112B013C010E946F94EC
:109C90006B017C010E947A84882309F466C080915C
:109CA000FE07811162C030E020E041E050E060E456
:109CB000CE0101960E94262440E450E06CE477E156
:109CC000CE0101960E949CB86AEB73E0CE0101962A
:109CD0000E9403C640E450E06BE372E1CE010196BE
:109CE0000E949CB8B301A201CE018F5B9F4F0E94DE
:109CF000BD10BE016F5B7F4FCE0101960E943D9566
:109D000030E020E041E050E060E4CE0101960E94A6
:109D1000262440E450E06CE477E1CE0101960E94F5
:109D20009CB86AEB73E0CE0101960E9403C640E442
:109D300050E064E372E1CE0101960E949CB8C70135
:109D4000B60128EE33E040E050E00E942DC1BA0198
:109D5000A901CE018F5B9F4F0E94BD10BE016F5BBA
:109D60007F4FCE0101960E943D95112309F44DC00D
:109D70006EE572E180E799E00E94BF730E94521184
:109D8000AB01BC0180E799E00E94968966E572E12B
:109D900080E799E00E94BF7360918D06062E000C4B
:109DA000770B80E799E00E94A08964E472E180E784
:109DB00099E00E94BF734091A6055091A70560915C
:109DC000A8057091A90580E799E00E94968980E72F
:109DD00099E00E94C872C75ADF4F0FB6F894DEBFF1
:109DE0000FBECDBFDF91CF911F910F91FF90EF90EC
:109DF000DF90CF90BF90AF909F908F907F906F90AB
:109E00005F904F903F902F90089564E572E180E756
:109E100099E00E94BF730E945211AB01BC0180E720
:109E200099E00E9496896CE472E1B2CF3F924F9222
:109E30005F926F927F928F929F92AF92BF92CF92DA
:109E4000DF92EF92FF920F931F93CF93DF93CDB7E3
:109E5000DEB7CE56D1090FB6F894DEBF0FBECDBF28
:109E6000DC0114962D913C91232B09F419C69B011A
:109E7000225031092230310508F091C23B014C01DA
:109E8000FC018281803409F4F7C208F04AC08430B2
:109E900008F085C2809197058F5F80939705A30195
:109EA0006FEFC4010E943D45D40112960C911297A8
:109EB0000695017013961C9113978AEC810F8031DF
:109EC00008F043C063E874E08D919C910E945F8428
:109ED0007C010097D1F1FC0180858F708530A9F558
:109EE0008091AF09181324C08091B009803401F526
:109EF0008091B1099091B2095C01990FCC08DD08FD
:109F000060E0C7010E94D484FC0181859285A3850D
:109F1000B485A816B906CA06DB060CF065C0512C3C
:109F20003EC0823409F4A8C208F439C28058AFCFC9
:109F30001093AF0980E48093B009812F0E94F590BF
:109F40009093B2098093B109D7CF212F30E0F90166
:109F5000E852F64E8491F901E85CF54E1491F9014E
:109F6000E258F54EF490FF2009F43BC081110E94A5
:109F70002490EF2DF0E0EE0FFF1FEC55FA4FA59166
:109F8000B491EC911E2331E020E009F430E0832FFE
:109F9000922F552453940817190609F0C0CFF3E007
:109FA0006F16710409F488C0D4011496ED91FC91E8
:109FB000E181EF70E150EC3008F07EC0F0E08827DE
:109FC000EB51F04B8F4F0C94B8C1065082513C506E
:109FD000725082518B508251BF50EC500551475105
:109FE000695190E080E0D5CF61E0C7010E94D48440
:109FF00055245394FC0181859285A385B4858A15E7
:10A000009B05AC05BD050CF0CACF89CF0E946F94AB
:10A010009B01AC0144275527D4011496ED91FC9186
:10A020006281738190E080E0AA24AA94BA2CC12CAA
:10A03000D12C18EEE12E13E0F12E00E010E00E948A
:10A04000C4238823C9F1F4010081118165E474E01F
:10A05000C8010E945F84892B41F46AE474E0C8015E
:10A060000E945F84892B09F40EC142E050E063E056
:10A07000C4010E943D4520C00E946F949B01AC0129
:10A0800044275527D4011496ED91FC916281738188
:10A0900090E080E0AA24AA94BA2CC12CD12C1CE216
:10A0A000E12EFF24F39400E010E00E94C42342E07C
:10A0B00050E064E0811184C0D4011496ED91FC91CC
:10A0C000808183FB992790F9951509F4D2C1982FC7
:10A0D000907E09F439C1982F907E90528F71892B10
:10A0E000808358C10E946F949B01AC01442755277F
:10A0F000D4011496ED91FC916281738190E080E02F
:10A10000AA24AA94BA2CC12CD12C16E9E12EF12C48
:10A1100000E010E0CACF0E946F949B01AC0144277D
:10A120005527D4011496ED91FC916281738190E0E2
:10A1300080E0AA24AA94BA2CC12CD12C18EEE12ECE
:10A1400013E0F12E00E010E00E94C423882309F4FC
:10A15000B3CFF4010081118160E574E0C8010E9471
:10A160005F84892B41F466E574E0C8010E945F8436
:10A17000892B09F488C042E050E068E079CF0E9462
:10A180006F949B01AC0144275527D4011496ED919F
:10A19000FC916281738190E080E0AA24AA94BA2C99
:10A1A000C12CD12C1CE2E12EFF24F39400E010E03E
:10A1B0000E94C42342E050E069E0882309F47CCF88
:10A1C000C4010E943D450E946F94D4011496ED9104
:10A1D000FC917383628370CF0E946F949B01AC01EA
:10A1E00044275527D4011496ED91FC916281738127
:10A1F00090E080E0AA24AA94BA2CC12CD12C16E9B4
:10A20000E12EF12C00E010E0D3CF0E946F949B016F
:10A21000AC0144275527D4011496ED91FC9162813D
:10A22000738190E080E0AA24AA94BA2CC12CD12C8E
:10A2300018EEE12E13E0F12E00E010E00E94C4239E
:10A24000882309F439CFF401008111816DE574E0B0
:10A25000C8010E945F84892B39F463E674E0C80169
:10A260000E945F84892B21F042E050E06BE000CF38
:10A270006FE374E0C8010E945F8442E050E066E052
:10A28000892B09F4F5CE42E050E06DE0F1CE0E945A
:10A290006F949B01AC0144275527D4011496ED918E
:10A2A000FC916281738190E080E0AA24AA94BA2C88
:10A2B000C12CD12C1CE2E12EFF24F39400E010E02D
:10A2C0000E94C423882309F4F7CE42E050E06CE0FA
:10A2D00077CF0E946F949B01AC0144275527D4018E
:10A2E0001496ED91FC916281738190E080E0AA2444
:10A2F000AA94BA2CC12CD12C16E9E12EF12C00E045
:10A3000010E0DECF0E946F949B01AC0144275527DB
:10A31000D4011496ED91FC916281738190E080E00C
:10A32000AA24AA94BA2CC12CD12C18E5E12E12E053
:10A33000F12E00E010E00E94C423882309F4BCCE73
:10A3400042E050E060E094CE0E946F94D4011496F5
:10A35000ED91FC91159773836283E181EF70552035
:10A3600009F445C0E230F1F050F4EE23E9F1D401F4
:10A370001496ED91FC91808150FA83F9B1CEE530CD
:10A3800089F0A3016AE0E73091F7C4010E943D45DE
:10A390008111EDCF8091970581508093970590E0D2
:10A3A00080E080C3F4010081118169E374E0C80199
:10A3B0000E945F84892BA9F460E574E0C8010E94C3
:10A3C0005F84892B71F466E574E0C8010E945F84A4
:10A3D000892B39F461E274E0C8010E945F84892B03
:10A3E00019F0A30166E0D1CFA30161E0CECFE15027
:10A3F000ED3008F0BCCFF0E08827EE5FFD4A8F4FCC
:10A400000C94B8C10F52B75112521252B751155293
:10A41000B751365236523652365236521252A30184
:10A4200062E0B3CFA30165E0B0CF0D911C9169E369
:10A4300074E0C8010E945F84892BA9F460E574E090
:10A44000C8010E945F84892B71F466E574E0C8013D
:10A450000E945F84892B39F461E274E0C8010E9494
:10A460005F84892B19F0A30167E08FCFA30160E01F
:10A470008CCF8F71806434CEB3E06B16710409F415
:10A480008ECF63E874E0F401808191810E945F8443
:10A490008C01D40113968C919091AF098913EBC074
:10A4A0009091B009903409F0E6C08091B109909183
:10A4B000B2093C010115110509F40DC1F80120850F
:10A4C0002F70253009F007C1C8010E94A889382ED5
:10A4D000F3E0F81708F0DBC063E0C8010E94D48401
:10A4E000DC0119968D919C913AE0E32EE89E600183
:10A4F000E99ED00C1124A396DFAECEAEA39762E006
:10A50000C8010E94D484DC0119968D919C91E89E2B
:10A510002001E99E500C11246201052C000CEE086C
:10A52000FF08AF96CCAEDDAEEEAEFFAEAF9761E00A
:10A53000C8010E94D4845C0160E0C8010E94D484F8
:10A54000DC011996CD90DD90ED90FC901C97A796BC
:10A55000CCAEDDAEEEAEFFAEA7979301072C000C9C
:10A56000440B550B2C193D094E095F09A396CEAC3F
:10A57000DFACA397B601DD0C880B990BAF96CCAC82
:10A58000DDACEEACFFACAF976C197D098E099F096D
:10A590000E941DC1D50119962D913D914D915C915F
:10A5A0001C97A796CCACDDACEEACFFACA7972C19F2
:10A5B0003D094E095F09A7962CAF3DAF4EAF5FAF87
:10A5C000A7970E944FC1AF96ACACBDACCEACDFAC90
:10A5D000AF97A20EB31EC41ED51E45E0E42E3E1456
:10A5E00009F468C081E090E0A396EEACFFACA397BD
:10A5F000A701FF0C660B770B4A155B056C057D0503
:10A600000CF461C0B601A5016201052C000CEE0836
:10A61000FF084C155D056E057F050CF459C06A01F5
:10A620007B0122E032126BC06301770CEE08FF0859
:10A6300060E0C8010E94D484FC0181859285A385D5
:10A64000B485C816D906EA06FB060CF444C261E0DC
:10A65000C8010E94D484FC0181859285A385B485BC
:10A660008C159D05AE05BF050CF099CE81E090E0FC
:10A67000A0E0B0E033C28093AF0990E49093B009BA
:10A680000E94F5909093B2098093B10912CF8AE0AD
:10A69000869D5001879DB00C11240B2C000CCC081A
:10A6A000DD08512C412C20E038E2A3963FAF2EAFBD
:10A6B000A39798CF64E0C8010E94D484DC01199666
:10A6C0008D919C9191CF66246A9423E0722E9CCF49
:10A6D000712C612CA6CF2AE0289F6001299FD00C05
:10A6E00011240D2C000CEE08FF08512C412C20E009
:10A6F00038E2A3963FAF2EAFA39781E090E0D4015C
:10A700001496ED91FC91428153819301241B350BEA
:10A7100037FF03C0319521953109821793070CF457
:10A72000BFC08081982F929596959770963008F0CB
:10A73000BAC09F5F9295990F907E8F71892BB2C09E
:10A74000F70161857285DB018C91811154C2A114DE
:10A75000B10409F472C0D50118968C9118978F70C6
:10A76000843009F06AC019966D917C91CE010196F2
:10A770000E949D34CE0101960E941A12882309F48A
:10A7800058C06114710409F45FC0E114F10431F0A0
:10A79000F70180858F70843009F441C025961CAE86
:10A7A0001DAE1EAE1FAE259729961CAE1DAE1EAE69
:10A7B0001FAE299723961FAD23971F7023961FAFB7
:10A7C000239781E022968FAF2297CC24C394F12C5B
:10A7D000E12C01E024962FAD249725963FAD2597D7
:10A7E00040E027965FAD279728966FAD289729966A
:10A7F0007FAD2997CE0101960E9405371AC0011539
:10A80000110529F0F80180858F70843019F06AE80D
:10A8100074E0F1C161857285FB01808196CF61850D
:10A820007285FB018081882321F0CE0101960E9470
:10A830006A8ACE0101960E945012D4011496ED91BD
:10A84000FC9173826282ABCD0115110531F0D80104
:10A8500018968C918F708430E9F025961CAE1DAE51
:10A860001EAE1FAE259729961CAE1DAE1EAE1FAEA6
:10A87000299723961FAD23971F7023961FAF239709
:10A8800082E022968FAF2297CC24C394F12CE12C46
:10A8900002E0A0CFF80161857285DB018C91C3CF06
:10A8A00080818F7180838081803AB8F0C201550C1D
:10A8B000AA0BBB0BC816D906EA06FB0671F0A396D5
:10A8C000EEADFFADA397CF01FF0FAA0BBB0BC816D0
:10A8D000D906EA06FB0609F062CD6416750609F48E
:10A8E0005ECD6D961CAE1DAE1EAE1FAE6D976B9607
:10A8F0008FAD6B978F7080666B968FAF6B976D96F1
:10A900008CAD9DADAEADBFAD6D9765968CAF9DAF77
:10A91000AEAFBFAF65976996CCAEDDAEEEAEFFAE23
:10A92000699763E975E080E799E00E94BF73D401FD
:10A9300013966C9180E799E00E94998961E975E02E
:10A9400080E799E00E94BF73CE018F5A9F4F0E940B
:10A95000C02C6FEF73E0F401808191810E945F84CD
:10A96000B12CA12CD12CC12C6296EFAC62976396CE
:10A97000FFAC639764960FAD649765961FAD6597BE
:10A9800066962FAD669767963FAD679768964FAD11
:10A99000689769965FAD69976FEF0E942B42D4016B
:10A9A0000D911C9163E074E0C8010E945F847C01FA
:10A9B00068E074E0C8010E945F848C010097E1F1B7
:10A9C000FC0180858F708430B9F56185728540E423
:10A9D00050E0CE0101960E9447C66FE270E0CE01C2
:10A9E00001960E940EC6892B59F4D80119962D9113
:10A9F0003C9143E050E060E4CE0101960E942624A1
:10AA000000E020E032E040E150E0BE016F5B7F4FAC
:10AA1000CE018F5A9F4F0E94D52A0E947A848823A4
:10AA200059F08091FE07811107C0BE016F5B7F4F17
:10AA3000CE0101960E943D95E114F10409F4FDCE8A
:10AA4000F70180858F70843009F0F7CE61857285BB
:10AA5000CE0101960E949D34CE0101960E941A12E9
:10AA6000882309F4E6CECC24C394F12CE12C629621
:10AA70000FAD629763961FAD639764962FAD649791
:10AA800065963FAD659766964FAD669767965FADE5
:10AA9000679768966FAD689769967FAD6997AACEFC
:10AAA0008FEF9FEFC259DF4F0FB6F894DEBF0FBE96
:10AAB000CDBFDF91CF911F910F91FF90EF90DF906D
:10AAC000CF90BF90AF909F908F907F906F905F904E
:10AAD0004F903F90089580E090E0DC01F4012481E4
:10AAE0003581F90142815381052E000C660B770BED
:10AAF00084179507A607B70709F451CC3C01D40188
:10AB00000D911C9163E074E0C8010E945F845C01B8
:10AB100068E074E0C8010E945F846C01A114B10474
:10AB200019F4892B09F489CE64E374E0C8010E940A
:10AB30005F847C016FE274E0C8010E945F848C0135
:10AB400069E975E080E799E00E94BF73F4016381D1
:10AB500080E799E00E94998967E975E080E799E0CC
:10AB60000E94BF73B30180E799E00E94A08980E74B
:10AB700099E00E94C872C114D10409F4E8CDD6014D
:10AB800018968C9118978F70843009F0E0CD199643
:10AB90006D917C9140E450E0CE0101960E9447C641
:10ABA0000E947A84882309F4D2CD8091FE07811116
:10ABB000CECD6FE270E0CE0101960E940EC6892BC9
:10ABC00051F4F6012185328543E050E060E4CE0186
:10ABD00001960E9426246114710409F410CEE11438
:10ABE000F10439F0D70118968C918F70843009F4F4
:10ABF000A7CD67E874E0CE0101960E943D95A7CDF0
:10AC00008F929F92AF92BF92CF92DF92EF92FF927C
:10AC10000F931F93CF93DF9300D000D0CDB7DEB753
:10AC20002091AE053091AF05232B09F4C5C02091CA
:10AC3000A1052111C1C04C018091A1058F5F8093B6
:10AC4000A10580918D068F5F80938D060E946F9481
:10AC50009B01AC0160919D0570919E0580919F05BF
:10AC60009091A005A12CB12C65011BE0E12EF12CE7
:10AC700000E010E00E94C423882309F452C0E09150
:10AC8000AE05F091AF050681178101151105B9F1E7
:10AC9000F80180858F70863071F56FEF73E0C80121
:10ACA0000E945F840097D1F0FC0120852F70253031
:10ACB000A9F4E680F780E114F104E9F0FA82E98270
:10ACC000B801CE0101960E94571BB401CE01019636
:10ACD0000E94164FF701E280F380EDCF1A830983BB
:10ACE00070E060E0CE0101960E94571BB401CE01D6
:10ACF00001960E94164FF80102811381C6CFF3E03E
:10AD00008F16910451F00E946F9460939D0570938B
:10AD10009E0580939F059093A0051092AF09109215
:10AD2000B00983E088169104E9F10E946F949B01B9
:10AD3000AC016091990570919A0580919B05909165
:10AD40009C05A12CB12C650118E8E12E13E1F12E30
:10AD500000E010E00E94C423882321F1E091AE05B9
:10AD6000F091AF05068117810115110589F0F801F1
:10AD700080858F70863041F41A83098370E060E02B
:10AD8000CE0101960E94571BF80102811381ECCF7E
:10AD90000E946F946093990570939A0580939B0528
:10ADA00090939C0580918D06815080938D068091B3
:10ADB000A10581508093A10526960FB6F894DEBFB9
:10ADC0000FBECDBFDF91CF911F910F91FF90EF90FC
:10ADD000DF90CF90BF90AF909F908F9008954F924B
:10ADE0005F926F927F92AF92BF92CF92DF92EF927B
:10ADF000FF920F931F93CF93DF93CDB7DEB7679783
:10AE00000FB6F894DEBF0FBECDBF67E273E180E7F7
:10AE100099E00E94BF7380E799E00E94C8720E9487
:10AE20006F942B013C0180918D06882341F10E9493
:10AE30006F949B01AC01A12CB12C650110E1E12EB6
:10AE400017E2F12E00E010E0C301B2010E94C4231A
:10AE5000811115C00E94107580919D06811162C0FC
:10AE60008091970690919806059711F00E940849E5
:10AE70000E94B74C82E090E00E940056D4CF8091AF
:10AE80008D06882351F064E073E189EC98E00E941C
:10AE9000BF7389EC98E00E94C8726EEE72E180E7A1
:10AEA00099E00E94BF7380E799E00E94C872809188
:10AEB000B4058F5F8093B405E0919906F0919A06EE
:10AEC0003097D1F10681178101151105A9F1D8013B
:10AED00018968C918F708530B9F7C8010E94A889A7
:10AEE000882391F3F80160817181CE0101960E945F
:10AEF0009D34CE0101960E941A12882359F08A854A
:10AF00009B85009739F0DC01ED91FC910284F3857B
:10AF1000E02D1995CE0101960E945012F801028190
:10AF20001381D2CF80919B0690919C06892B09F4C6
:10AF300097CF0E94952594CF1092B3051092B20539
:10AF400066EE72E180E799E00E94BF7380E799E0C6
:10AF50000E94C87264E670E080E090E00E942A924D
:10AF60001092190610928E066EEC72E180E799E05D
:10AF70000E94BF730E945211AB01BC0180E799E0AF
:10AF80000E9496898091B0059091B1050E94468EED
:10AF90001092B1051092B0051092AF051092AE0557
:10AFA00010929A061092990610921B0610921A0699
:10AFB00010928B0610928A061092890610928806CB
:10AFC00010929C0610929B0669EC72E180E799E072
:10AFD0000E94BF730E945211AB01BC0180E799E04F
:10AFE0000E94968980E799E00E94C87210928C06B0
:10AFF0008091B40581508093B40567960FB6F8949C
:10B00000DEBF0FBECDBFDF91CF911F910F91FF909B
:10B01000EF90DF90CF90BF90AF907F906F905F9058
:10B020004F9008958091FE078F5F8093FE07A8954B
:10B0300083E090E00E9400560E9410758091FE0708
:10B0400081508093FE070895CF92DF92EF92FF9296
:10B050000F931F93CF93DF93FC012485243059F085
:10B0600090E080E0DF91CF911F910F91FF90EF90E2
:10B07000DF90CF9008956A018B01EC01F12C8F2DA8
:10B080000E94D980811127C0FC868C85843041F3D1
:10B0900020910202309103022F5F3F4F21F1309344
:10B0A000030220930202409102025091030220E029
:10B0B00061E00E942A80F80182818F3FB9F4838188
:10B0C0008F3FF9F484818F3FE1F485818F3FC9F48C
:10B0D00084E08C87C5CF8B7F8831B1F2F394F4E0A4
:10B0E000FF12CDCFD2CF20E030ECD9CF811109C0F3
:10B0F0008381811106C08481811103C085818823E9
:10B1000039F3C114D10421F3FC8480E590E00E945E
:10B11000968EB8016E5F7F4F8F2D0E94EE1CB60198
:10B120008F2D0E94DD1C64E070E08F2D0E94F58E53
:10B130000E946F946B017C01F4E9CF0EF1E1DF1EF8
:10B14000E11CF11CCE010E94F71C873149F161E03E
:10B1500070E080E090E00E942A920E941258CE0196
:10B160000E94F71C882309F4B3CF0E946F94C6167F
:10B17000D706E806F90630F78C850E941680EC8524
:10B18000F0E0EE0FFF1FE157F94F1182108284E0CB
:10B190008C8765E675E183ED98E00E94E37360CFEC
:10B1A0006AE575E183ED98E00E94E37381E090E049
:10B1B00059CFA89583E090E00C9400565F926F926F
:10B1C0007F928F929F92AF92BF92CF92DF92EF9237
:10B1D000FF920F931F93CF93DF93CDB7DEB76D9799
:10B1E0000FB6F894DEBF0FBECDBF8091B005909131
:10B1F000B105892B09F421C480918D0681111DC4EC
:10B2000080918D068F5F80938D0666EC7DE08FEBDD
:10B2100098E00E94BF738FEB98E00E94C872009183
:10B22000B0051091B1056EE874E0C8010E945F841A
:10B2300090939A068093990664E974E0C8010E948D
:10B240005F8490931B0680931A066FEC74E0C8012C
:10B250000E945F849093AF058093AE056BE974E024
:10B26000C8010E945F8490938B0680938A060E9497
:10B270000C2A60EA74E08091B0059091B1050E94BB
:10B280005F8490939C0680939B06009709F4BBC152
:10B2900020919D062111B7C1DC011696ED90FC901E
:10B2A0008091860690918706892B51F081E08093EA
:10B2B0009D0666EB7DE08FEB98E00E94BF7355C062
:10B2C0006DE77DE080E799E00E94BF7380E799E039
:10B2D0000E94C87267E77DE080E799E00E94BF7333
:10B2E0000E945211AB01BC0180E799E00E9496894F
:10B2F00080E799E00E94C8728FE090E00E944BB511
:10B300008C0188E1F80181831282108216861586ED
:10B3100010926506109264061092DB071092FD07EA
:10B320000E94B51486E3A82E80E1B82EB0923E06A6
:10B33000A0923D0697E3C92E90E1D92ED092420605
:10B34000C09241061093870600938606012B09F0F0
:10B35000B1C065E67DE089EC98E00E94BF7389EC9E
:10B3600098E00E94C87210929D061092C00510923B
:10B37000BF05CC24C394D12CE114F10409F443C1DA
:10B3800080919D06882309F43EC1D70118968C91BF
:10B3900018978F70863009F089C00D911C91FE01BD
:10B3A00031965F014801F0E18F0E911C3501D80103
:10B3B0008C910E946E11582EF80181810E946E11AD
:10B3C0005294A0EF5A22582AD5015D925D010E5F7A
:10B3D0001F4F8016910659F762EE7CE08FEB98E0E4
:10B3E0000E94BF736091BF057091C0058FEB98E01C
:10B3F0000E94A0896BED7CE08FEB98E00E94BF7308
:10B400008091BF059091C005F3E0880F991FFA95D0
:10B41000E1F72091BD053091BE05820F931F0E9478
:10B42000108D8FEB98E00E94C8722091BF0530917B
:10B43000C00521313105D4F56091BD057091BE057F
:10B4400048E0C901E3E0880F991FEA95E1F7860F0C
:10B45000971F415058F1FC01E40FF11D5081552315
:10B46000C1F3220F331F4091B7055091B805240F47
:10B47000351FF901D182C08228E0F301DC0101907F
:10B480000D922A95E1F7DC018C91883231F480919C
:10B490008606909187060E94E7208091BF059091D3
:10B4A000C00501969093C0058093BF05F701E28027
:10B4B000F38062CF88E890E00E944BB59093BE0580
:10B4C0008093BD0569E57DE080E799E00E94BF7348
:10B4D0000E945211AB01BC0180E799E00E9496895D
:10B4E00080E799E00E94C87282E290E00E944BB52A
:10B4F0009093B8058093B7056CE47DE080E799E010
:10B500000E94BF730E945211AB01BC0180E799E019
:10B510000E94968980E799E00E94C8728091BD05DB
:10B520009091BE05892B31F08091B7059091B805B7
:10B53000892B79F464E37DE089EC98E00E94BF7385
:10B540000E945211AB01BC0189EC98E00E949689DF
:10B5500006CF82E794E49093BA058093B9051092E0
:10B560006506109264061092DB071092FD070E9498
:10B57000B514B0923E06A0923D06D0924206C0920B
:10B58000410680918606909187060E94031081E013
:10B590000E943791811130C061E27DE080E799E03F
:10B5A0000E94E3730091860610918706C8010E94ED
:10B5B000031040E060EFC8010E94F3200E94279230
:10B5C000E0918606F091870681E0808361E07DE06E
:10B5D00080E799E00E94E373809186069091870648
:10B5E0000E94A620882309F461CE65EF7CE080E705
:10B5F00099E00E94E3735ACE67EE7CE080E799E021
:10B600000E94E373B0CE1092B3051092B205E091A0
:10B610009906F0919A06309709F4F0C0E680F78019
:10B620000091990610919A060115110509F4DFC0E1
:10B63000E114F10409F4DBC0D70118968C918F70E6
:10B64000853091F7C7010E94A889823068F3B7015D
:10B65000CE0101960E94E11ACE0101960E941A12B3
:10B66000882309F462C08A859B85009759F5CE012D
:10B6700001960E94B5898C01912C812C97FF06C000
:10B6800011950195110988248394912CCE0101967E
:10B690000E94DB17C82ED12C8985853009F44EC055
:10B6A000863009F042C0B02E61E0802F0E94B99030
:10B6B00061E0892809F479C0CA94CD2809F079C0DD
:10B6C00060E077C0DC01ED91FC910484F585E02D0C
:10B6D0001995892B49F08A859B85DC01ED91FC91B8
:10B6E0000284F385E02D19958A859B85DC01ED9117
:10B6F000FC910680F781E02D1995892BB1F0CE01E0
:10B7000001960E94DB17882331F060E071E0CE01E2
:10B7100001960E9479368D819E81892B31F060E0FF
:10B7200072E0CE0101960E947936D7011296ED9013
:10B73000FC90CE0101960E94501272CFCD2829F4C0
:10B7400062E0CE0101960E94AB1760E071E0CE018D
:10B7500001960E9479368D819E81892B31F060E0BF
:10B7600072E0CE0101960E94793661E0802F0E943E
:10B77000B99060E0802F0E948B906EEA7DE080E7B8
:10B7800099E00E94BF73B80180E799E00E94A08908
:10B7900069EA7DE080E799E00E94BF7367EA7DE097
:10B7A00080E799E00E94BF73C0CFCA94CD2809F00A
:10B7B00087CFC62ED12C8B2D0E948B9062EA7DE024
:10B7C00080E799E00E94BF73B80180E799E00E948A
:10B7D000A08960EA7DE080E799E00E94BF73B6012E
:10B7E00080E799E00E94A0896EE97DE0D9CFF80159
:10B7F000868197819093B3058093B20580E799E0A5
:10B800000E94C872E091AE05F091AF05309709F43F
:10B810008AC080918D068F5F80938D060681178187
:10B820000115110509F47AC0D80118968C918F7012
:10B83000863009F069C0198F088F70E060E0CE0192
:10B8400048960E94571B8C8D9D8D892B09F45CC0F6
:10B850008091B0059091B105892B09F455C0E88C11
:10B86000F98CF70180858F70863099F56FEF73E062
:10B87000C7010E945F840097F1F0DC0118962C91BB
:10B8800018972F702530B9F41696CD90DC90C1141E
:10B89000D104F9F0DA82C982B701CE0101960E9483
:10B8A000571BED81FE811082118212821382F601F4
:10B8B000C280D380ECCFFA82E98270E060E0CE01F2
:10B8C00001960E94571B62E070E0CE0101960E9433
:10B8D000164FEC8DFD8D10821182128213828A8D9B
:10B8E000843068F462E0823008F060E08B8D0E9462
:10B8F000B990EC8DFD8D8181807F818305C080347E
:10B9000041F060E0823431F0D80112960D911C9123
:10B9100087CF62E08B8D0E94B990F6CF80918D0623
:10B92000815080938D066EEC7CE08FEB98E00E9456
:10B93000BF7366EC7CE08FEB98E00E94BF7381E000
:10B940002091990630919A06232B09F480E00E94F9
:10B95000D3146DEB7CE08FEB98E00E94BF7381E025
:10B960002091AE053091AF05232B09F480E00E94B1
:10B97000D31466EB7CE08FEB98E00E94BF7381E00C
:10B9800020918A0630918B06232B09F480E00E94D7
:10B99000D3146DEA7CE08FEB98E00E94BF7381E0E6
:10B9A00020919B0630919C06232B09F480E00E9495
:10B9B000D31464EA7CE08FEB98E00E94BF7380911F
:10B9C00019060E94D3148FEB98E00E94C8726FE9A9
:10B9D0007CE08FEB98E00E94BF730E945211AB0194
:10B9E000BC018FEB98E00E9496898FEB98E00E9453
:10B9F000C87281E080938E068FE898E00E94FF1C59
:10BA0000882351F08FE898E00E94A41D84E090E024
:10BA10009093980680939706809197069091980648
:10BA2000079731F484E090E090939806809397060E
:10BA300080918D06815080938D066D960FB6F89497
:10BA4000DEBF0FBECDBFDF91CF911F910F91FF9051
:10BA5000EF90DF90CF90BF90AF909F908F907F90AE
:10BA60006F905F900895CF93DF93EC01FB012481E9
:10BA7000358140815181628173810E94D372CE01F0
:10BA8000DF91CF910895AF92BF92CF92DF92EF9264
:10BA9000FF921F93CF93DF9300D000D0CDB7DEB7D6
:10BAA0006C017C0110E08AE0A82EB12C133061F10A
:10BAB000F701828190E0B0E0A0E089839A83AB83B4
:10BAC000BC83BE82AD82BE016F5F7F4F8FEB98E07B
:10BAD0000E94335D61E274E10E94BF731F5FFFEF5C
:10BAE000EF1AFF0A143011F726960FB6F894DEBF4E
:10BAF0000FBECDBFDF91CF911F91FF90EF90DF90F0
:10BB0000CF90BF90AF900895F601858190E0B0E0AE
:10BB1000A0E089839A83AB83BC83BE82AD82BE01E1
:10BB20006F5F7F4F8FEB98E00E94335D6FE174E1B0
:10BB3000D3CF0F931F93CF93DF9300D000D0CDB717
:10BB4000DEB70E94342966E17AE08FEB98E00E942C
:10BB5000BF73CE0101960E94998ECE0101960E947C
:10BB6000435D05EA13E01A83098380912D089091C3
:10BB70002E08A0912F08B09130088B839C83AD8351
:10BB8000BE83CE0101960E94435D1A8309831B8206
:10BB90001C821D821E8280E590E00E94968E44E009
:10BBA00050E0BE016D5F7F4F81E090E00E946178C0
:10BBB000CE0101960E94435D1A8309831B821C8279
:10BBC0001D821E8280E590E00E94968E44E050E047
:10BBD000BE016D5F7F4F85E090E00E946178CE01ED
:10BBE00001960E94435D6CE37AE08FEB98E00E943F
:10BBF000BF7388EC90E026960FB6F894DEBF0FBEB8
:10BC0000CDBFDF91CF911F910F910895CF92DF9219
:10BC1000EF92FF921F93CF93DF9300D000D0CDB768
:10BC2000DEB762EE79E08FEB98E00E94BF7384EAA2
:10BC3000E82E88E0F82E10E090E1C92ED12CF70113
:10BC400081917F01803130F463EA74E08FEB98E0FA
:10BC50000E945973153041F1F7013197808190E0CE
:10BC6000B0E0A0E089839A83AB83BC83DE82CD827F
:10BC7000BE016F5F7F4F8FEB98E00E94335D60EEF7
:10BC800079E00E94BF731F5F1630C9F626960FB683
:10BC9000F894DEBF0FBECDBFDF91CF911F91FF9013
:10BCA000EF90DF90CF9008958091A90890E0B0E0E8
:10BCB000A0E089839A83AB83BC83DE82CD82BE0100
:10BCC0006F5F7F4F8FEB98E00E94335D0E94C872D8
:10BCD000DACFEF92FF920F931F93CF93DF9300D0B1
:10BCE00000D01F92CDB7DEB77B01CE0107969F93A0
:10BCF0008F9301979F938F9301979F938F930197B2
:10BD00009F938F9301979F938F9301979F938F9307
:10BD10008E010F5F1F4F1F930F9385EA94E09F934F
:10BD20008F93DB0113968C9113978F9312968C91BE
:10BD30008F930E94CEC60FB6F894DEBF0FBECDBF64
:10BD40000697ECF46CEB7EE089EC98E00E94BF7300
:10BD5000D70112966D917C9189EC98E00E945973FD
:10BD600080E991E027960FB6F894DEBF0FBECDBFF5
:10BD7000DF91CF911F910F91FF90EF9008958091E7
:10BD80009C0890919D08892B09F44BC00E94A785BF
:10BD9000882309F446C0A0919C08B0919D08529652
:10BDA0001C921E92519754961C921E92539784E8AF
:10BDB00090E01D969C938E931C971E961C921E9746
:10BDC00080E090E350969C938E931F97ED91FC91A9
:10BDD00011970088F189E02D64E070E0CD0119959C
:10BDE00080919C0890919D08DC01ED91FC9102806E
:10BDF000F381E02D46E050E0B801199586E0F801A6
:10BE0000A4EAB8E001900D928A95E1F780919C0830
:10BE100090919D08DC01ED91FC910488F589E02D5D
:10BE200019950E94065E6EEC7EE08FEB98E00E9412
:10BE3000BF7388EC90E096CFCF93DF93CDB7DEB79A
:10BE40002E970FB6F894DEBF0FBECDBF80918D0642
:10BE500081116BC063E17EE08FEB98E00E94BF73BD
:10BE60008FEB98E00E94C8721092BC081092BB0839
:10BE700080E090E19093B7088093B60884E890E062
:10BE80009093BE088093BD0881E08093B80880E05D
:10BE900090E29093BA088093B9088AEA98E00E94E9
:10BEA000071C8B37910509F0C4C01C821B828DE7EB
:10BEB00092E09A8389838AEA98E09E838D838FEF4C
:10BEC0009FEF98878F838091B0059091B105892B62
:10BED00011F00E94EF56CE0101960E94788E909349
:10BEE000B1058093B0058AEA98E00E945E128091C5
:10BEF000B0059091B105892BD9F467E07EE089EC1B
:10BF000098E00E94BF7389EC98E00E94C8726CE1CF
:10BF100075E0CE0109960E940672CE0109960E9434
:10BF2000899ACE0109960E94C77190E080E014C002
:10BF300064EF7DE08FEB98E00E94BF738FEB98E099
:10BF40000E94C8720E94DE5880919C0890919D08C2
:10BF5000892B59F481E090E02E960FB6F894DEBF5D
:10BF60000FBECDBFDF91CF9108950E94A785882392
:10BF700089F3A0919C08B0919D0852961C921E9244
:10BF8000519754961C921E92539784E890E01D9608
:10BF90009C938E931C971E961C921E9780E090E3B4
:10BFA00050969C938E931F97ED91FC91119700886A
:10BFB000F189E02D60E670E0CD01199560919C0853
:10BFC00070919D0840E0CE0109960E944572BE0125
:10BFD000675F7F4F8EE998E00E94CD70CE01099691
:10BFE0000E94C77180919C0890919D08DC01ED91A1
:10BFF000FC910488F589E02D199566ED7DE080E7D8
:10C0000099E00E94BF736EE978E0CE0109960E9424
:10C01000FD71BE01675F7F4F80E799E00E94B173B9
:10C0200080E799E00E94C872CE0109960E94C7710C
:10C0300091CF8AEA98E00E947712892BA1F08AEAD0
:10C0400098E00E94A1126CE175E0CE0101960E9479
:10C050000672CE0101960E94899ACE0101960E9435
:10C06000C7710E94FD998AEA98E00E945E1263EE11
:10C070007DE08FEB98E00E94BF738FEB98E00E9409
:10C08000C87253CF0E941C5F892B49F486EF9FEF43
:10C09000909398068093970684EF91E0089588EC3A
:10C0A00090E00895BF92CF92DF92EF92FF920F93AC
:10C0B0001F93CF93DF9300D000D0CDB7DEB78C01B4
:10C0C0006B01FB0184819581892BD9F1E080F1809E
:10C0D0006FE370E0C7010E940EC6009791F19C01CA
:10C0E0002E193F09790137FD2CC06CE175E0CE01B6
:10C0F00001960E940672F601848195810097B9F03D
:10C100008E159F0508F47C01F60160817181FB01A9
:10C11000EE0DFF1DB0801082CE0101960E94A1712C
:10C12000F60180819181E80EF91EF701B082BE010F
:10C130006F5F7F4FC6010E94CD70CE0101960E94B5
:10C14000C77169EB74E0C6010E944870882319F139
:10C15000F801128A118A80E090E19587848784E84B
:10C1600090E0948B838B81E0868780E090E2908BD7
:10C17000878781E090E026960FB6F894DEBF0FBE69
:10C18000CDBFDF91CF911F910F91FF90EF90DF9086
:10C19000CF90BF90089566EC74E0C6010E9448708D
:10C1A000882369F0F801128A118A148A138A84E8B4
:10C1B00090E095878487168680E090E3D8CF90E062
:10C1C00080E0D9CFFF920F931F93CF93DF9300D0DE
:10C1D00000D0CDB7DEB78C01BC01CE0101960E9424
:10C1E000FD71BE016F5F7F4F80E799E00E94B173E0
:10C1F00080E799E00E94C872CE0101960E94C77143
:10C2000061E37FE0CE0101960E94CF71BE016F5FB6
:10C210007F4FC8010E942D70F82ECE0101960E941A
:10C22000C771FF2069F0B801CE0101960E94FD712F
:10C23000CE0101960E94899ACE0101960E94C77193
:10C2400026960FB6F894DEBF0FBECDBFDF91CF911B
:10C250001F910F91FF9008955F926F927F928F923E
:10C260009F92AF92BF92CF92DF92EF92FF920F9385
:10C270001F93CF93DF93CDB7DEB7C956D1090FB661
:10C28000F894DEBF0FBECDBF4C018B01F42E642F9E
:10C2900080E799E00E94998965E879E080E799E074
:10C2A0000E94BF73B801CE0101965C010E94FD712E
:10C2B000B50180E799E00E94B17380E799E00E94A0
:10C2C000C872C5010E94C77192E0F91263C263E8A7
:10C2D00079E0C5010E94CF71B501C8010E945D706F
:10C2E000F82EC5010E94C771FF2009F4C8C220E0E2
:10C2F0004DE251E0B4018DE698E00E946174E09057
:10C300008806F09089066CE779E0CE018C599F4F42
:10C310000E94CF7165E779E0CE01825A9F4F0E945B
:10C32000CF71CE018E5A9F4F0E94998E68961FAD95
:10C33000689767960FAD67976696DFAC66976596C8
:10C34000CFAC65976CE175E0CE0181960E940672D4
:10C35000BE016F5D7F4FC5010E94FD716C2DC5014F
:10C360000E94187162ED74E00E9449716D2D0E9467
:10C37000187162ED74E00E944971602F0E9418717B
:10C3800062ED74E00E944971612F0E941871BC0136
:10C39000CE01885A9F4F0E94FD71C5010E94C7714E
:10C3A000CE0181960E94C77160E779E0CE01845B7F
:10C3B0009F4F0E94CF716CE175E0CE018A5B9F4F69
:10C3C0000E9406720CE918E0D80118966C9170E092
:10C3D00084E0759567958A95E1F7C5010E947B8594
:10C3E0004D815E8169817A81CE018A5B9F4F0E9477
:10C3F0008D70C5010E94C771F80160856F7070E093
:10C40000C5010E947B854D815E8169817A81CE0163
:10C410008A5B9F4F0E948D70C5010E94C7710F5F9C
:10C420001F4FF8E0023A1F0779F66AE679E0CE017D
:10C43000805C9F4F0E94CF7169E479E0CE018196C4
:10C440000E94CF71BE016F5D7F4FCE01C8960E94E2
:10C45000FD71BE01605C7F4FCE01C8960E94637182
:10C46000BE016A5B7F4F0E946371BE01645B7F4FB8
:10C470000E946371BE01685A7F4F0E946371BE01C2
:10C48000625A7F4F0E9463718C014AE0B50180E5DA
:10C4900090E00E94FFB8F50101900020E9F7319784
:10C4A000AF014A195B09B501C8010E948D70811165
:10C4B00003C0C8010E940671BE016C597F4FC801BC
:10C4C0000E946371B7010E944971BC01C4010E94BE
:10C4D000B173C4010E94C872CE01C8960E94C77190
:10C4E000CE0181960E94C771CE01805C9F4F0E9451
:10C4F000C771CE018A5B9F4F0E94C771CE01845BDA
:10C500009F4F0E94C771CE01885A9F4F0E94C771EA
:10C51000CE01825A9F4F0E94C771CE018C599F4F06
:10C520000E94C771C4010E94C87264E670E080E096
:10C5300090E00E942A92D401ED91FC910488F58943
:10C54000E02DC401199501E010E080C022966EAD87
:10C550007FAD2297CE0181960E946A8A892B09F4C9
:10C5600048C118AE19AE1AAE1BAE1CAE1DAE1EAE43
:10C570001FAE89AD8F7089AF40E053E0BE016F5DA3
:10C580007F4FCE01C8960E941E2E00E020E033E0CF
:10C5900040E250E0B501CE01C8960E94D52ABC0108
:10C5A000C6010E94A17108EC10E125C1EE2009F43A
:10C5B000EFC046E050E070E060E0C8010E94CA6F42
:10C5C000D8016D917C91CE0181960E949D34CE015F
:10C5D00081960E941A1200E911E0882399F189A539
:10C5E000873061F4CE0181960E948F4A61E0892BE9
:10C5F00009F462E0CE0181960E94AB1718AE19AE25
:10C600001AAE1BAE1CAE1DAE1EAE1FAE89AD8F7036
:10C6100089AF40E053E0BE016F5D7F4FCE01C89609
:10C620000E941E2E00E020E033E040E250E0B50121
:10C63000CE01C8960E94D52ABC01C6010E94A171F4
:10C6400008EC10E1CE0181960E945012C801C75932
:10C65000DF4F0FB6F894DEBF0FBECDBFDF91CF9195
:10C660001F910F91FF90EF90DF90CF90BF90AF9010
:10C670009F908F907F906F905F900895F8016081F8
:10C6800071810E945F847C01892B09F040C104E91B
:10C6900011E0DCCFEE2009F47BC049E050E070E00F
:10C6A00060E0C8010E94CA6F4AE0B401C5010E945F
:10C6B000457241E050E067EC73E0C8010E948D7064
:10C6C0004D815E8169817A81C8010E948D7065E229
:10C6D00079E080E799E00E94BF73B801CE018196AE
:10C6E0000E94FD71BE016F5D7F4F80E799E00E945F
:10C6F000B17380E799E00E94C872CE0181960E94D2
:10C70000C7716DE179E0CE0181960E94CF71F80189
:10C71000848195812DA13EA182179307E1F4892B95
:10C72000A1F1E080F18069A07AA0D7018D917D010F
:10C73000882359F1082E000C990B0E949EC56C01AC
:10C74000F30181913F01082E000C990B0E949EC5B8
:10C75000C816D90651F3CE0181960E94C7715520A3
:10C7600041F021E048EC50E0B4018DE698E00E94F1
:10C770006174D8018D919C910E948F74009711F47F
:10C7800084E991E08C01C5013DC055245394E3CF69
:10C7900001E97ECFB1E0FB1270C062E479E0C5012F
:10C7A0000E94CF71B501C8010E942D70582EC5019D
:10C7B0000E94C771552049F1EE2051F346E050E048
:10C7C00070E060E0C8010E94CA6F4AE0B401CE0187
:10C7D000805C9F4F0E944572F80160817181CE019B
:10C7E00081960E949D34CE0181960E941A12811179
:10C7F000ADCE00E911E0CE0181960E945012CE012B
:10C80000805C9F4F0E94C77121CF6BE279E0C50128
:10C810000E94CF71B501C8010E942D70F82EC5018C
:10C820000E94C771F11036CF60E179E0C5010E9426
:10C83000CF71B501C8010E942D70182FC5010E944B
:10C84000C77100E0112309F401CF80E00E945A89EA
:10C8500068EE78E08FEB98E00E94BF738FEB98E072
:10C860000E94C8726CE175E0C5010E940672C501A4
:10C870000E94899AC5010E94C77100E065CE6BE3F2
:10C8800079E0C5010E94CF71B501C8010E942D70E9
:10C89000F82EC5010E94C771F11088CE65E379E0DA
:10C8A000C5010E94CF71B501C8010E942D70F82EFC
:10C8B000C5010E94C771FF2001F3EE2009F468CF83
:10C8C00045E050E070E060E0C8010E94CA6F62ED90
:10C8D00074E0C8010E944870882339F0E0909906FE
:10C8E000F0909A06E114F10491F46CE175E0C8014E
:10C8F0000E944870811107C08091990690919A0614
:10C90000009709F0BBCEE090B005F090B10520E0B3
:10C9100048EC50E2B4018DE698E00E946174C401D5
:10C920000E94C8721C821B828DE792E09A838983E1
:10C930009E828D828FEF9FEF98878F83B701C5010D
:10C940000E945675F2CDAF92BF92CF92DF92EF92D6
:10C95000FF920F931F93CF93DF93CDB7DEB7C859E4
:10C96000D1090FB6F894DEBF0FBECDBF8E010F5BAD
:10C970001F4FD8011D921C92FE01ED5BFF4F8EE10F
:10C98000DF011D928A95E9F780919C0890919D089E
:10C99000892B09F49AC10E94A785882309F495C1BF
:10C9A000A0919C08B0919D0852961C921E9251979E
:10C9B00054961C921E92539784E890E01D969C9387
:10C9C0008E931C971E961C921E9780E090E35096C3
:10C9D0009C938E931F97ED91FC9111970088F1899C
:10C9E000E02D60E270E0CD0119954FE150E0B80113
:10C9F00080919C0890919D080E94FE857C01809109
:10CA00009C0890919D08DC01ED91FC910488F589CA
:10CA1000E02D1995E114F10409F457C1F801EE0D68
:10CA2000FF1D10828091A9081F928F938091A80802
:10CA30001F928F938091A7081F928F938091A608D1
:10CA40001F928F938091A5081F928F938091A408C5
:10CA50001F928F9384ED94E09F938F931F9280E4B5
:10CA60008F93FE0131966F01FF93EF930E9461C691
:10CA700069E070E18FEB98E00E94BF73B8018FEB23
:10CA800098E00E945973B6018FEB98E00E945973A9
:10CA90008FEB98E00E94C8727E01F1E6EF0EF11C68
:10CAA000D70113961C921E92129788EE93E0A0E095
:10CAB000B0E0F70184839583A683B78384E08487FD
:10CAC0008DE293E09183808316861586108B07870D
:10CAD000128A118A80E590E0948B838B178A68E331
:10CAE0007FE080E799E00E94BF736EE978E0CE01B5
:10CAF00087589F4F0E94FD71BE0167587F4F80E7A6
:10CB000099E00E94B17380E799E00E94C872CE015B
:10CB100087589F4F0E94C77163E075E0CE0185572B
:10CB20009F4F0E94067263E075E0CE0187589F4FC9
:10CB30000E940672BE0167587F4FCE018D579F4FEE
:10CB40000E94FD716EE978E0CE018D579F4F0E94E3
:10CB50006371BE0165577F4F0E946371BC01CE01B6
:10CB60008F569F4F0E94FD71CE018D579F4F0E949F
:10CB7000C771CE0187589F4F0E94C771CE0185575C
:10CB80009F4F0E94C77185E095E0CD57DF4F998395
:10CB90008883C358D040C957DF4F19821882C758BD
:10CBA000D040C757DF4F19821882C958D040CF569E
:10CBB000DF4F88819981C159D040CB57DF4F99838E
:10CBC0008883C558D04063E070E180E799E00E9417
:10CBD000BF730E945211AB01BC0180E799E00E9433
:10CBE000968980E799E00E94C87264E670E080E070
:10CBF00090E00E942A9282EE90E6D7011E969C93C6
:10CC00008E931D9765EC7CE68DE897E70E946BB9E3
:10CC10008C010FB6F894DEBF0FBECDBF892BA1F1FA
:10CC200083E090E00E944BB5D8011D969C938E93B3
:10CC30001C97FC01F182E0821282C7010E94FF1C56
:10CC4000882319F0C7010E94A41DD70151966D9148
:10CC50007C9152975396AD90BC906115710509F483
:10CC60004BC0CE0187589F4F0E94F573A501BE01AE
:10CC700067587F4FC7010E942458181619060CF4F4
:10CC800087C1C8010E9466776AE97FE080E799E082
:10CC90000E94BF73EE24EA94FE2CCE018F569F4F64
:10CCA0000E94C771C701C856DF4F0FB6F894DEBFA8
:10CCB0000FBECDBFDF91CF911F910F91FF90EF90ED
:10CCC000DF90CF90BF90AF90089540E250E06BE3CB
:10CCD00070E1C8010E94BAB86DE170E18FEB98E095
:10CCE0000E94BF73B8018FEB98E00E9459738FEBDD
:10CCF00098E00E94C87296CEF70167857089A501F9
:10CD0000C7010E948F13B9CF83E99FE09F938F9350
:10CD10001F930F930E94F2B9D70156961C921E9250
:10CD20005597D8011C96ED91FC91A080B1800F9091
:10CD30000F900F900F9093E3C92ED12CD501ED9158
:10CD4000FC910084F185E02DC501199541975CF4B3
:10CD5000B1E0CB1AD10839F064E170E080E090E0F6
:10CD60000E942A92EBCF6E01E7E9CE0ED11CDF9232
:10CD7000CF9283E49FE09F938F931F930F930E9422
:10CD80000FBA0F900F900F900F900F900F90019788
:10CD9000D1F4D6018D919C91F701968B858B6CE136
:10CDA00075E0CE0185579F4F0E94067280E0C12C2E
:10CDB000FAE0CF1270C08A3009F071C0CE018557F9
:10CDC0009F4F0E94C771D7015596ED90FC90B8EC2B
:10CDD000EB16F10409F0BAC067EF7FE08FEB98E043
:10CDE0000E94BF7364EF71E080E090E00E942A929D
:10CDF000ED961FAE1EAEED97EF961FAE1EAEEF97EF
:10CE00008FEF9FEFC158DF4F99838883CF57D04072
:10CE100087E692E0EB969FAF8EAFEB97CF57DF4F51
:10CE200019830883C158D040F8948091B00590913F
:10CE3000B105892B11F00E94EF56CE0187589F4F04
:10CE40000E94788E9093B1058093B0057894C801C4
:10CE50000E9466778091B0059091B105892B09F009
:10CE600063C06CE175E0CE0185579F4F0E9406724A
:10CE7000CE0185579F4F0E94899ACE0185579F4FBB
:10CE80000E94C77160EE7FE089EC98E00E94BF735A
:10CE9000F12CE12C02CF9DE0C91201C0C82EC801BF
:10CEA0000E94B6B9D82ED7011D96AD90BC90A114A2
:10CEB000B10499F1BAE08B1779F0EDE08E1761F0CB
:10CEC000FFEF8F1749F0682FCE0185579F4F0E94C3
:10CED000B9708C2DCD2C6CCFC157DF4F88819981D3
:10CEE000CF58D040892B91F0BE0165577F4FCE01BE
:10CEF00087589F4F0E94FD71CE0187589F4FF501C3
:10CF00001995CE0187589F4F0E94C7716CE175E05B
:10CF1000CE0185579F4F0E949771FFEFDF12D9CF47
:10CF2000C8010E9466774ACF0E94DE5880918E0623
:10CF3000882329F00E949A8867FF0E94281769EDCC
:10CF40007FE08FEB98E00E94BF73A7CEE0E3EE1680
:10CF5000E1E0FE0651F465EC7FE08FEB98E00E9483
:10CF6000BF73C8010E94667798CE6DEA7FE089ECB6
:10CF700098E00E94BF73C8010E946677B70189ECF0
:10CF800098E00E94A08989EC98E00E94C87285CE42
:10CF9000D7011F96BC901F975096AC90DF92CF920E
:10CFA00086E99FE09F938F931F930F930E94F2B99E
:10CFB000DF92CF9281E99FE09F938F931F930F930E
:10CFC0000E94F2B9D8011C96ED91FC9181E0828318
:10CFD000DF92CF928EE89FE09F938F931F930F93E2
:10CFE0000E94F2B9D8011C96ED91FC911282AF9289
:10CFF000BF9288E59FE09F938F931F930F930E94AA
:10D00000F2B90FB6F894DEBF0FBECDBFB12C8FE4DE
:10D01000C82E8FE0D82E8B2D94E08902F0011124C8
:10D02000A3E8B0E0AC0FBD1FEA0FFB1F8081918128
:10D03000009709F469CE2281338121153105C1F3AE
:10D040003F932F939F938F93DF92CF921F930F93D2
:10D050000E94F2B9B3940FB6F894DEBF0FBECDBFF5
:10D06000DACF0F931F93CF93DF93EB0102970CF46A
:10D070009DC00A811B816AE27FE0C8010E9465B8F9
:10D08000892B51F481E00E945A8988EC90E0DF916D
:10D09000CF911F910F91089566E27FE0C8010E9431
:10D0A00065B8892B11F480E0EECF66E07FE08FEB6E
:10D0B00098E00E94BF730E949A8863FB662760F91C
:10D0C00081E0682770E08FEB98E00E94A0898FEBE9
:10D0D00098E00E94C87280919C0890919D08892BCD
:10D0E00009F454C00A811B810E94A785882309F492
:10D0F0004DC0F80101900020E9F73197E01BF10BDA
:10D10000B09708F043C0A0919C08B0919D0852963A
:10D110001C921E92519754961C921E92539784E82B
:10D1200090E01D969C938E931C971E961C921E97C2
:10D1300080E090E350969C938E931F97ED91FC9125
:10D1400011970088F189E02D60E270E0CD0119951A
:10D15000B80180919C0890919D080E94597380911C
:10D160009C0890919D08DC01ED91FC910190F0816B
:10D17000E02D60E0199580919C0890919D08DC015C
:10D18000ED91FC910488F589E02D19956A817B81E8
:10D190008FEB98E00E9459736FEF7EE08FEB98E081
:10D1A0000E94BF738FEB98E00E94C872809197062F
:10D1B0009091980602977CF10E94A364883C9105A7
:10D1C00039F424E030E030939806209397065FCF3F
:10D1D0008F3F9807C9F464EE7EE080E799E00E94F3
:10D1E000BF7380E799E00E94C87210928C0683E0BA
:10D1F00090E090939806809397068FE898E00E94BD
:10D20000A41D89EC90E043CF20918E062111D9CF47
:10D210002FE030E0D8CF67ED7EE089EC98E00E9407
:10D22000BF7389EC98E00E94C87284EF91E02FCF21
:10D230000895FC01248135816217730748F48081C9
:10D240009181009729F0860F971FFC018081089536
:10D2500080E008950895AF92BF92CF92DF92EF924F
:10D26000FF920F931F93CF93DF936C017B018B0190
:10D27000040F151FEB015E01AE18BF08C017D107E0
:10D2800059F06991D601ED91FC910190F081E02D6A
:10D29000C6011995892B79F7C501DF91CF911F91AF
:10D2A0000F91FF90EF90DF90CF90BF90AF900895D7
:10D2B000FC01538D448D252F30E0842F90E0821B9C
:10D2C000930B541710F0CF96089501970895FC0121
:10D2D000918D828D981761F0A28DAE0FBF2FB11D79
:10D2E0005D968C91928D9F5F9F73928F90E00895D1
:10D2F0008FEF9FEF0895FC01918D828D981731F08B
:10D30000828DE80FF11D858D90E008958FEF9FEFDE
:10D310000895FC01918D228D892F90E0805C9F4FB4
:10D32000821B91098F739927089583ED98E00E94DD
:10D33000896921E0892B09F420E0822F0895FC01FE
:10D34000A48DA80FB92FB11DA35ABF4F2C91848D66
:10D3500090E001968F739927848FA689B7892C93C3
:10D36000A089B1898C91837080648C93938D848D16
:10D37000981306C00288F389E02D80818F7D808319
:10D380000895EF92FF920F931F93CF93DF93EC01D9
:10D3900081E0888F9B8D8C8D98131AC0E889F9895C
:10D3A000808185FF15C09FB7F894EE89FF8960835F
:10D3B000E889F98980818370806480839FBF81E0E0
:10D3C00090E0DF91CF911F910F91FF90EF90089522
:10D3D000F62E0B8D10E00F5F1F4F0F731127E02EFD
:10D3E0008C8D8E110CC00FB607FCFACFE889F98935
:10D3F000808185FFF5CFCE010E949F69F1CFEB8D33
:10D40000EC0FFD2FF11DE35AFF4FF0829FB7F89408
:10D410000B8FEA89FB8980818062CFCFCF93DF9326
:10D42000EC01888D8823B9F0AA89BB89E889F9893C
:10D430008C9185FD03C0808186FD0DC00FB607FC71
:10D44000F7CF8C9185FFF2CF808185FFEDCFCE01A4
:10D450000E949F69E9CFDF91CF91089580E090E02D
:10D46000892B29F00E94956981110E94000080E0BB
:10D4700090E0892B49F080E090E0892B29F00E9410
:10D48000000081110E94000080E090E0892B49F0AB
:10D4900080E090E0892B29F00E94000081110E9419
:10D4A000000080E090E0892B49F080E090E0892B3B
:10D4B00029F00E94000081110C94000008950F9340
:10D4C0001F93FC0162857385848595850281138194
:10D4D00024813581601B710B820B930B06851785A8
:10D4E00020893189601B710B820B930B1F910F9167
:10D4F0000895DC01ED91FC910190F081E02D1994EB
:10D500008FEF9FEF0895FC01628973898489958963
:10D510000895EF920F931F93CF93DF93FC01248D17
:10D52000222341F0213051F1DF91CF911F910F91D2
:10D53000EF9008952289338944895589868997898E
:10D54000A08DB18D821B930BA40BB50B892F9A2F45
:10D55000AB2FBB278C010F5F1F4F628173818481CA
:10D560009581CFB7F894DCB7E1E0ECBFEE24E3940B
:10D57000E2E0FEEF1995DCBFCFBFD6CFF0E0E0E0F0
:10D58000DF91CF911F910F91EF901994FC01138EB1
:10D59000128E41110CC082899389A489B589868B2A
:10D5A000978BA08FB18F148E81E090E0089590E06A
:10D5B00080E00895CF92DF92EF92FF92CF93DF93B6
:10D5C000DC01CB01642FCFB7F8946D01EE24FF246A
:10D5D000CBBEDCB741E04CBFA901E1E0FEEF1995FD
:10D5E000DCBFCFBFDF91CF91FF90EF90DF90CF9066
:10D5F0000895CF93DF93FC01248D211110C0EC011D
:10D60000828D938D892B49F066897789808D918DE4
:10D6100030E020E045E00E94DA6A1B8E1A8EDF912E
:10D62000CF9108951F93CF93DF93FC01248D211197
:10D6300045C0162FEC01828D938D892B49F46689A4
:10D640007789808D918D30E020E043E00E94DA6A96
:10D650004A8D5B8DCA0181709927FE01E80FF91F81
:10D66000158F892B69F02D8D3E8D6E897F89888D70
:10D67000998D640F751F811D911D41E00E94DA6A2A
:10D680008A8D9B8D01969B8F8A8F81159140B1F475
:10D690006E897F89888D998D30E020E045E00E9479
:10D6A000DA6A1B8E1A8E8E899F89A88DB98D9F5F2D
:10D6B000AF4FBF4F8E8B9F8BA88FB98F81E090E0CB
:10D6C000DF91CF911F910895DC01ED91FC910280D3
:10D6D000F381E02D40E01994FB01248135814281E2
:10D6E00053812417350750F4A081B181A20FB31FD5
:10D6F0008C938481958101969583848380E008953D
:10D70000CF93DF93EC01E881F9810284F385E02D6A
:10D71000CE0119950196B9F7DF91CF910895CF9277
:10D72000DF92EF92FF920F931F93CF93DF937C01D1
:10D730006A018B01D0E0C0E0CC15DD0581F0D70196
:10D74000ED91FC910284F385E02DC70119958F3F7F
:10D75000980729F0F80181938F012196EDCFCE0132
:10D76000DF91CF911F910F91FF90EF90DF90CF90BD
:10D770000895CF93C62FDC01ED91FC910088F189CB
:10D78000E02D1995DC01ED91FC910190F081E02DE7
:10D790006C2FCF911994062E000C770BFC01778328
:10D7A00066830895CF93DF93EC018E819F8101966C
:10D7B00011F5E881F9810088F189E02DCE011995F4
:10D7C000DC01ED91FC910084F185E02D1995892B08
:10D7D000B1F0E881F9810284F385E02DCE0119953D
:10D7E0008132910534F3E881F9810684F785E02DD3
:10D7F000682FCE01199581E0DF91CF91089580E0E7
:10D80000FBCFCF93DF931F92CDB7DEB76983DC01E7
:10D81000ED91FC910280F381E02D41E050E0BE01EA
:10D820006F5F7F4F19950F90DF91CF910895EF9221
:10D83000FF920F931F93CF93DF93EC018B017A013B
:10D840000E946F94688B798B8A8B9B8B8C819D81D6
:10D85000DC01ED91FC910280F381E02DA701B8017C
:10D86000DF91CF911F910F91FF90EF9019941F932B
:10D87000CF93DF93EC01162F0E946F94688B798B06
:10D880008A8B9B8B8C819D81DC01ED91FC910190B9
:10D89000F081E02D612FDF91CF911F911994CF92EC
:10D8A000DF92EF92FF92CF93DF93EC018E819F8105
:10D8B0008F3F980759F02FEF3FEF3F832E83DF9183
:10D8C000CF91FF90EF90DF90CF9008950E946F94DA
:10D8D0006B017C01A4EFCA0EA1E0DA1EE11CF11C71
:10D8E000E881F9810088F189E02DCE011995DC01EC
:10D8F000ED91FC910084F185E02D1995892B39F487
:10D900000E946F946C157D058E059F0548F3E88194
:10D91000F9810088F189E02DCE011995DC01ED91A6
:10D92000FC910284F385E02DDF91CF91FF90EF9081
:10D93000DF90CF9019940E9499C50F931F93CF93B6
:10D94000DF93EC0188819981009759F02A813B810E
:10D950002617370730F081E0DF91CF911F910F91AB
:10D9600008958B016F5F7F4F0E94B8C4009759F0F4
:10D97000998388831B830A832C813D81232B59F74C
:10D98000FC011082E8CF80E0E7CFEF92FF920F9387
:10D990001F93CF93DF93009751F4CFEFDFEFCE01CA
:10D9A000DF91CF911F910F91FF90EF900895DC01CF
:10D9B0001C96ED90FC90F70100811181D801ED914A
:10D9C000FC910688F789E02DC8011995882329F371
:10D9D000D801ED91FC910084F185E02DC8011995E5
:10D9E000D801ED91FC91892B61F30284F385E02D40
:10D9F000C8011995EC01019681F2F8018789882305
:10DA000029F06C2F83ED98E00E949989D701129636
:10DA10008C91882321F2C532D10509F6D801ED9108
:10DA2000FC910084F185E02DC801199502975CF006
:10DA3000D801ED91FC910688F789E02DC801199570
:10DA40008111ECCFAACFD1E0C0E0D801ED91FC91DB
:10DA50000284F385E02DC80119958F3F980709F4DA
:10DA60009CCF9C01215431092A31310570F48D2F4E
:10DA70008295807F829FC00D1124D11104C00C2E8D
:10DA8000000CDD0B8CCFD0E0E0CF9C01215631099A
:10DA90002A31310560F3C0978A30910570F79D2FC8
:10DAA0009295907F989FC00D1124E7CFCF92DF927F
:10DAB000EF92FF920F931F93CF93DF936C018B0133
:10DAC00086E090E00E944BB5EC0190931D07809397
:10DAD0001C07F60101900020E9F7CF018C199D0980
:10DAE0000E944BB57C01B6010E9422C6F60101904E
:10DAF0000020E9F73197EC19FD09EE0DFF1D1082AA
:10DB0000F982E8821B830A8380911E0790911F0788
:10DB10009D838C83D0931F07C0931E07DF91CF9105
:10DB20001F910F91FF90EF90DF90CF900895FC012F
:10DB3000868197818F3F980729F02FEF3FEF37833A
:10DB400026830895808591850C94B6B91F93CF9351
:10DB5000DF93182F66E270E00E94BF1CC82F67E2B7
:10DB600070E0812F0E94BF1C9C2FDF91CF911F91ED
:10DB70000895CF93FC01C08D80E590E00E94968EC1
:10DB800060E270E08C2F0E94F58E62E070E08C2FD6
:10DB90000E94BF1C84FD1AC062E070E08C2F0E94BE
:10DBA000BF1C83FF0CC048E162E070E08C2F0E9434
:10DBB000B51C0E94371D90E080E0CF9108950E942F
:10DBC000371D80E590E00E94968EDFCF40E162E055
:10DBD00070E08C2F0E94B51C0E94371D81E090E000
:10DBE000ECCFFF920F931F93CF93DF93EB01FC01D8
:10DBF000178A168A2A81211109C02B81211106C09A
:10DC00002C81211103C02D812223F1F041155105F2
:10DC1000D9F08A01FC01F08C80E590E00E94968E9C
:10DC2000BE016E5F7F4F8F2D0E94EE1CB8018F2DBD
:10DC30000E94DD1C0E94371D81E090E0DF91CF91B2
:10DC40001F910F91FF90089590E080E0F7CFAF9281
:10DC5000BF92CF92DF92FF920F931F93CF93DF93E8
:10DC60008C015B01EA01FC01C688D788F08C80E555
:10DC700090E00E94968E8F2D0E94AD8F8C179D078D
:10DC800020F48F2D0E94AD8FEC019E01A501B601FD
:10DC90008F2D0E944D8F0E94371DF801868997892C
:10DCA0008C0F9D1F978B868BCE01DF91CF911F919B
:10DCB0000F91FF90DF90CF90BF90AF9008957F922B
:10DCC0008F929F92AF92BF92CF92DF92EF92FF928C
:10DCD0000F931F93CF93DF93CDB7DEB7A6970FB601
:10DCE000F894DEBF0FBECDBF8C01762E942E852E0C
:10DCF00020E2A22ECE0101967C01DC01EA2D1D92CC
:10DD0000EA95E9F76801F3E4CF0ED11C85EA93E0C8
:10DD10009AA389A38FEF8BA38CA38DA38EA343E437
:10DD200050E0BE016F5D7F4FC6010E94F16D01960C
:10DD300009F4BFC081E089838A8386E0B82EBB8264
:10DD40001C82D80114966D917D918D919C911797AD
:10DD50000E94C0C16D837E838F83988789869A864F
:10DD600080E890E09C878B874CE150E0B701C601CA
:10DD70000E94276EFE0137968AE1DF011D928A9587
:10DD8000E9F74801B8E08B0E911CF401D70101902E
:10DD90000D92BA94E1F740E150E0B701C6010E944C
:10DDA000276EF7011192AA94E9F796E0A92EB12CFB
:10DDB00040E250E0B701C6010E94276EF1E0AF1AC1
:10DDC000B108B1F783E6898392E89A8393E59B8350
:10DDD0008C8385E38D8381E08E837F829DE39887AA
:10DDE00097E099878A8786E0F401DE011B9601900F
:10DDF0000D928A95E1F78CE0898B8A8B63E175E05F
:10DE0000CE0143960E9422C6D8011B966C91CE018A
:10DE100049960E94C98FF8016485CE014B960E94F5
:10DE2000C98FD8011D966C91CE014D960E94C98F65
:10DE30004EE150E0B701C6010E94276EB3E07B12AD
:10DE40001EC082E3898384E08A83F80196859B83E0
:10DE500097859C8390899D8391899E8396E39F8378
:10DE60008887828D8987838D8A87848D8B87858D2E
:10DE70008C874CE050E0B701C6010E94276E87E313
:10DE8000898386E08A8391E09B8393E09C838D83E2
:10DE90008FE08E838AE38F838BE388878FEF898778
:10DEA00049E050E0B701C6010E94276EC6010E94FA
:10DEB000B96DA6960FB6F894DEBF0FBECDBFDF9149
:10DEC000CF911F910F91FF90EF90DF90CF90BF9077
:10DED000AF909F908F907F900895AF92BF92CF9216
:10DEE000DF92EF92FF920F931F93CF93DF93DC01AA
:10DEF000CD90DC901197C114D10439F01496CD91D6
:10DF0000DC918C017601209761F4DF91CF911F9114
:10DF10000F91FF90EF90DF90CF90BF90AF9008955A
:10DF200075015701BFEFAB1ABB0AF7018081082EBC
:10DF3000000C990B0E945CB8892B91F72197CC0DAE
:10DF4000DD1D8881082E000C990B0E945CB8892B7E
:10DF500029F0CE15DF0510F02197F3CFAE014F5F0A
:10DF60005F4F4E195F09D80115965C934E93149735
:10DF7000CE14DF0420F4B701C6010E94D5C5D80134
:10DF8000ED91FC91119714968D919C91E80FF91FDA
:10DF90001082BBCFCF93DF93DC011496ED91FC91FF
:10DFA0006E177F0728F54115510511F19F01261BBA
:10DFB000370B4217530708F49A01DB01EC01888103
:10DFC0009981E21BF30BFD83EC83AF01461B570BDA
:10DFD000260F371FBC01620F731F8A0F9B1F0E9401
:10DFE00047C6E881F9818C819D81E80FF91F108275
:10DFF000DF91CF910895DF92EF92FF920F931F93DD
:10E00000CF93DF93FC01E480F580E114F10451F437
:10E010008FEF9FEFDF91CF911F910F91FF90EF90C6
:10E02000DF900895EC010190F081E02DEE0DFF1DD1
:10E03000D080108208811981062E000C770BC80150
:10E040000E9456C60E0D1F1DF801D082009701F3E5
:10E0500028813981821B930BDDCFFB0144815581DF
:10E06000FC01248135812417350778F08081918166
:10E07000009759F0FB01608171816115710529F0EC
:10E080000E9439C621E0892B09F020E0822F0895F3
:10E09000FC0124813581232B39F421E0FB018081AF
:10E0A000882349F020E007C0808191810E9419C631
:10E0B00021E0892BB9F7822F0895FC012481358155
:10E0C000FB014481558124173507E1F4FC0180816F
:10E0D0009181FB01608171810097D1F0611571051B
:10E0E000A1F4232BC1F0FC01808190E008C0232B18
:10E0F00091F0FB01808190E091958195910921E05B
:10E10000892B09F020E0822F08950E9419C6F7CFCD
:10E110006115710561F721E0F6CFEF92FF920F9341
:10E120001F93CF93DF936115710541F480E0DF9178
:10E13000CF911F910F91FF90EF90089541155105D8
:10E14000B1F07B01EC010C811D81040F151FB8019A
:10E150000E949D6C882351F3288139818C819D8197
:10E16000B701820F931F0E9422C61D830C8381E09A
:10E17000DECFCF93DF931F921F92CDB7DEB76983B7
:10E180001A8241E050E0BE016F5F7F4F0E948D70A8
:10E190000F900F90DF91CF9108950F931F93CF931E
:10E1A000DF938C01EB01FC01808191810097E1F00C
:10E1B0006881798161157105A9F0428153812C81B3
:10E1C0003D814217530770F00E9422C68C819D81C9
:10E1D000F801958384831D821C82DF91CF911F916A
:10E1E0000F9108950E94E7B588819981F801918384
:10E1F00080838A819B81938382838C819D81958397
:10E200008483198218821B821A82E5CFCF93DF9311
:10E21000EC0188819981009711F00E94E7B519827D
:10E2200018821D821C821B821A82DF91CF91089571
:10E23000EF92FF920F931F93CF93DF9300D01F9223
:10E24000CDB7DEB77C01862F4AE08E010F5F1F4FEE
:10E25000B80190E00E94FFB8F80101900020E9F7B2
:10E260003197AF01401B510BB801C7010E948D705F
:10E27000811103C0C7010E940671C7010F900F9062
:10E280000F900F90DF91CF911F910F91FF90EF9022
:10E290000895CF93DF93EC016115710539F4CE0138
:10E2A0000E940671CE01DF91CF910895FB0101908C
:10E2B0000020E9F73197AF01461B570B0E948D7084
:10E2C000882369F3EFCFCF93DF93EC01FB01448107
:10E2D0005581608171810E948D70811103C0CE01D2
:10E2E0000E940671CE01DF91CF910895EF92FF92C7
:10E2F0000F931F93CF93DF93EC017B018A01BA0147
:10E300000E949D6C81110BC0CE010E940671CE014E
:10E31000DF91CF911F910F91FF90EF9008951D8392
:10E320000C83B701888199810E9422C6F0CFFB013E
:10E3300001900020E9F73197AF01461B570B0C9471
:10E340007671CF93DF93EC016115710531F00E9476
:10E350009771CE01DF91CF9108950E940671F9CF98
:10E36000CF93DF93EC01FB018617970749F060819B
:10E3700071816115710541F0448155810E9476716A
:10E38000CE01DF91CF9108950E940671F9CFFC0173
:10E3900080819181009711F00C94E7B50895EF9278
:10E3A000FF920F931F93CF93DF93EC018B011982A0
:10E3B00018821B821A821D821C82CB010E9493B894
:10E3C0007C01BC01CE010E949D6C811109C0CE016F
:10E3D000DF91CF911F910F91FF90EF900C940671F8
:10E3E000FD82EC82B80188819981DF91CF911F91E4
:10E3F0000F91FF90EF900C948CB8FC011182108269
:10E4000013821282158214820C94B071FC01118265
:10E4100010821382128215821482FB010190002067
:10E42000E9F73197AF01461B570B0C9476710F93A8
:10E430001F93CF93DF93EC010E946F9468877987D5
:10E440008A879B87E881F9810284F385E02DCE01DC
:10E45000199597FF15C00E946F94088519852A8524
:10E460003B85601B710B820B930B0C811D812E81F0
:10E470003F81601771078207930720F38FEF9FEFAB
:10E48000DF91CF911F910F910895EF92FF920F931B
:10E490001F93CF93DF93EC017B01042F6CE175E0B8
:10E4A0000E940672C7010E941772002E000C110B09
:10E4B00097FD0BC00817190741F0682FCE010E9485
:10E4C000B970C7010E941772F3CFCE01DF91CF91CF
:10E4D0001F910F91FF90EF900895FB010190002094
:10E4E000E9F73197AF01461B570BDC01ED91FC9129
:10E4F0000280F381E02D19948F929F92AF92BF9288
:10E50000EF92FF920F931F93CF93DF93CDB7DEB7B8
:10E51000A1970FB6F894DEBF0FBECDBF7C01FA0104
:10E52000CB0119A2223008F42AE08E010F5D1F4FA3
:10E53000822E912CB12CA12CBF01A50194010E9427
:10E540002DC1F901CA016A300CF5605DD8016E93E6
:10E550008D01232B242B252B79F790E080E0109759
:10E5600021F0BD01C7010E946D72A1960FB6F8940B
:10E57000DEBF0FBECDBFDF91CF911F910F91FF90F6
:10E58000EF90BF90AF909F908F900895695CDECF21
:10E590006AE175E00C946D72DC01ED91FC910190E3
:10E5A000F081E02D1994CF92DF92EF92FF920F93BA
:10E5B0001F93CF93DF932115310581F4DC01ED9199
:10E5C000FC910190F081E02D642FDF91CF911F919C
:10E5D0000F91FF90EF90DF90CF9019942A30310582
:10E5E00001F52AE077FF1DC06A017B01EC016DE2B5
:10E5F0000E94CC728C0144275527BA014C195D0941
:10E600006E097F092AE0CE010E947C72800F911F63
:10E61000DF91CF911F910F91FF90EF90DF90CF90FE
:10E620000895DF91CF911F910F91FF90EF90DF90B0
:10E63000CF900C947C728F929F92AF92BF92CF92A8
:10E64000DF92EF92FF920F931F93CF93DF937C01A2
:10E650008B014C0182E0880E911C5701E5E0AE0E63
:10E66000B11CD0E0C0E0F40161914F01C8010E94EB
:10E6700099896C016EE2C8010E94CC728C0D9D1DBF
:10E68000C80FD91F8A149B0471F7F7016581C8016F
:10E690000E9499898C0F9D1FDF91CF911F910F913F
:10E6A000FF90EF90DF90CF90BF90AF909F908F90B2
:10E6B00008956115710511F00C946D7290E080E081
:10E6C00008950F931F93CF93DF93EC018B0163E0C9
:10E6D00075E00E94597301151105C1F1F8016191AE
:10E6E0008F01662399F1603240F0623231F06C356F
:10E6F00021F0CE010E94CC72F1CF6CE5CE010E94D8
:10E70000CC72F801319780818C30D1F044F489309B
:10E71000D9F08A30B9F0883009F762E6EACF823260
:10E7200059F024F462E78D3021F3D8CF8F3231F0E5
:10E730006CE58C35F1F2D2CF62E2DBCF6FE2D9CF5C
:10E7400066E6D7CF6EE6D5CF64E7D3CF62E2CE01DF
:10E750000E94CC7290E080E0DF91CF911F910F91E9
:10E760000895DB0114964D915C9115976D917C9104
:10E77000DC01ED91FC910280F381E02D1994EF9280
:10E78000FF920F931F93CF93DF938C017B01D0E017
:10E79000C0E0F701EC0FFD1F6491662361F0D80122
:10E7A000ED91FC910190F081E02DC8011995892B24
:10E7B00011F02196EECFCE01DF91CF911F910F91F5
:10E7C000FF90EF9008950F931F93CF93DF93EC0189
:10E7D0000E94BF738C01CE010E94C872800F911FEE
:10E7E000DF91CF911F910F910895DC0185EA93E0AD
:10E7F0008D939D9384E0FB0101900D928A95E1F742
:10E8000008951F920F920FB60F9211240BB60F921C
:10E810002F933F934F935F936F937F938F939F9328
:10E82000AF93BF93EF93FF9383ED98E00E949F69AE
:10E83000FF91EF91BF91AF919F918F917F916F91D8
:10E840005F914F913F912F910F900BBE0F900FBE94
:10E850000F901F9018951F920F920FB60F921124D0
:10E860000BB60F922F938F939F93EF93FF93E091AB
:10E87000E308F091E4088081E091E908F091EA086A
:10E8800082FD1DC090818091EC088F5F8F73209175
:10E89000ED08821741F0E091EC08F0E0ED52F74FFF
:10E8A000958F8093EC08FF91EF919F918F912F911D
:10E8B0000F900BBE0F900FBE0F901F901895808188
:10E8C000F2CFDF92EF92FF920F931F93CF93DF93DC
:10E8D00000D000D0CDB7DEB78B017A01D22E6CE12B
:10E8E00075E0CE0101960E9406729E012F5F3F4F98
:10E8F0004D2DB701C8010E94B39BCE0101960E9425
:10E90000C77126960FB6F894DEBF0FBECDBFDF915C
:10E91000CF911F910F91FF90EF90DF900895CF92CC
:10E92000DF92EF92FF920F931F93CF93DF93CDB7B8
:10E93000DEB7EC970FB6F894DEBF0FBECDBFDC019B
:10E940002C91222309F469C067EC73E00E94C9B8D6
:10E950009A8389837E01B3E0EB0EF11C01E010E0A5
:10E96000D02EC12E67EC73E090E080E00E94C9B821
:10E97000F701819391937F010E31110521F00F5F13
:10E980001F4F892B69F700911C0710911D07E98023
:10E99000FA800115110589F1D8016D917C91C701AB
:10E9A0000E9419C6892B29F5D8011296ED91FC9188
:10E9B000BE016F5F7F4F8D2D9C2D19958C0183EDCE
:10E9C00098E00E94C87263E775E183ED98E00E94C9
:10E9D000BF73C801EC960FB6F894DEBF0FBECDBF73
:10E9E000DF91CF911F910F91FF90EF90DF90CF902B
:10E9F0000895F80104811581CCCF67E775E183EDB7
:10EA000098E00E94E37383ED98E00E94C87263E788
:10EA100075E183ED98E00E94BF7310E000E0D9CF6C
:10EA2000CF9383ED98E00E948969892BE9F183ED0A
:10EA300098E00E946769C82F8A3089F08D3079F09C
:10EA4000883001F568E083ED98E00E94CC728091F7
:10EA50002007882331F3815080932007E2CFE09193
:10EA60002007F0E0E052F94F10826AE175E083ED93
:10EA700098E00E94597380EE96E00E948F74109285
:10EA80002007CFCF682F83ED98E00E94CC72E091F1
:10EA90002007EB3330F681E08E0F80932007F0E003
:10EAA000E052F94FC083BDCFCF9108958F929F92CE
:10EAB000AF92BF92CF92DF92EF92FF920F931F938C
:10EAC000CF93DF936115710509F496C0DB011896A9
:10EAD000EC911897E295E07FE595E595E595E5954C
:10EAE000E73008F089C0EC010E2E000CFF0B8827E0
:10EAF000E358FA488F4F0C94B8C1847595759E758C
:10EB0000B575FF7511764A766DE175E0CE01DF913E
:10EB1000CF911F910F91FF90EF90DF90CF90BF901A
:10EB2000AF909F908F900C946D7219968C9167E2C4
:10EB300075E0882359F362E275E0E8CF19964D91AC
:10EB40005D916D917C911C972AE030E0CE01DF91C0
:10EB5000CF911F910F91FF90EF90DF90CF90BF90DA
:10EB6000AF909F908F900C94D3721996CD90DD90BA
:10EB7000ED90FC901C9720E030E0A901C701B601A0
:10EB80000E94E3BF87FF09C06CEB73E0CE010E94D7
:10EB90005973F7FAF094F7F8F094C701B6010E94A0
:10EBA000BCC24B015C01BC01A401CE010E9496894C
:10EBB00062ED74E0CE010E945973C501B4010E9458
:10EBC000E8BF9B01AC01C701B6010E94D6C12DEC84
:10EBD0003CEC4CE45DE30E94D7C120E030E040E231
:10EBE00051E40E9449C00E94BCC2AB0170E060E0E9
:10EBF0002AE0CE010E947C7290E080E01DC0199650
:10EC00006D917C91CE01DF91CF911F910F91FF907B
:10EC1000EF90DF90CF90BF90AF909F908F900C942B
:10EC2000617316960D911C916BE5CE010E94CC721A
:10EC3000019679F48FEF9FEFDF91CF911F910F91A4
:10EC4000FF90EF90DF90CF90BF90AF909F908F900C
:10EC500008950115110579F0B801CE010E9456758D
:10EC6000019641F3D80112960D911C9101151105E1
:10EC700011F06CE2DACF6DE5CE010E94CC7221E09A
:10EC800030E0019611F030E020E088279927821BC0
:10EC9000930BD2CF16960D911C916BE7CE010E947B
:10ECA000CC72019639F20115110529F1D8016D9147
:10ECB0007C91CE010E946173019609F4BBCF6AE397
:10ECC000CE010E94CC72019609F4B4CFB801CE01F6
:10ECD0000E945675019609F4ADCFD80112960D9198
:10ECE0001C910115110539F06CE2CE010E94CC7225
:10ECF0000196C9F69FCF6DE7BFCFCF93DF93EC01AD
:10ED0000E881F9810284F385E02DCE0119958F3FCA
:10ED1000980769F0E881F981813291059CF30684B6
:10ED2000F785E02D682FCE01199590E080E0DF9106
:10ED3000CF910895CF92DF92EF92FF920F931F939E
:10ED4000CF93DF937C016B01DC01ED91FC91028498
:10ED5000F385E02D1995829761F0CFEFDFEFCE01BB
:10ED6000DF91CF911F910F91FF90EF90DF90CF90A7
:10ED70000895F6018085807F8460808786E090E03A
:10ED80000E944BB58C01009741F3E0EAF6E0DC010C
:10ED9000ED93FC9380E4DF011D928A95E9F780E40E
:10EDA00090E0F8019383828315821482D701ED915C
:10EDB000FC910284F385E02DC7011995EC010196C1
:10EDC000C9F0C232D10509F44DC0C032D1050CF4EE
:10EDD00049C0B8018C2FCC35D10549F5D701ED914B
:10EDE000FC910284F385E02DC7011995EC018F3F5A
:10EDF000980721F4C8010E94E7B5B1CF823691058A
:10EE000041F15CF48F32910509F18C359105D9F00F
:10EE1000829761F6B80182E20AC08E369105E1F070
:10EE20004CF4B8018CE0C636D10509F0BFCF0E9482
:10EE30006C6BBCCF8237910591F0B80189E0C43783
:10EE4000D105A9F3B3CFB8018CE5F1CFB8018FE2BA
:10EE5000EECFB80188E0EBCFB8018AE0E8CFB80187
:10EE60008DE0E5CFF80184819581009749F001900C
:10EE7000F081E02DE80FF91F31978081882321F080
:10EE8000B80180E00E946C6BD80114968D919C9122
:10EE90000E944BB5EC01009739F060EA76E00E94E1
:10EEA00022C6C8010E94E7B5F601D287C187D0E02B
:10EEB000C0E055CF8DE090E00E944BB5009729F05F
:10EEC0002DE0FC0111922A95E9F708950F931F9305
:10EED000CF93DF930097E1F0EC010C851D850115C0
:10EEE000110579F0D8018D919C91009739F0DC01E2
:10EEF000ED91FC910488F589E02D1995C8010E94D7
:10EF0000E7B5CE01DF91CF911F910F910C9441B9DC
:10EF1000DF91CF911F910F910895AF92BF92CF9241
:10EF2000DF92EF92FF920F931F93CF93DF9300D066
:10EF30001F92CDB7DEB761157105B1F06B01182FC7
:10EF4000DB011C96AD90BC90F501E080F180D7010B
:10EF5000ED91FC910688F789E02DC7011995811183
:10EF600006C0C6010E9466778FEF9FEF13C0F501C0
:10EF70009281911124C0D701ED91FC910190F08113
:10EF8000E02D612FC7011995F7018789811111C003
:10EF900090E080E00F900F900F900F90DF91CF9155
:10EFA0001F910F91FF90EF90DF90CF90BF90AF90A7
:10EFB0000895612F83ED98E00E94CC72E9CF812FF4
:10EFC0008F7D81548A31B8F280ED810F8A3098F2BA
:10EFD00083ED810F823078F21F3569F21E3759F2C6
:10EFE0001132B1F086EC810F823090F08AED810F02
:10EFF000873070F01D3361F0812F8F7E8F3241F0AA
:10F000008DED810F823020F01B3511F01D3511F48C
:10F0100091FFB1CF19821A821B821C82812F012E8F
:10F02000000C990B9F931F938DE295E09F938F9314
:10F030008E010F5F1F4F1F930F930E949EC66E019C
:10F04000F4E0CF0ED11C0F900F900F900F900F9007
:10F050000F90D8016D918D01D701ED91FC91019038
:10F06000F081E02DC7011995F7018789882339F0D0
:10F07000F8013197608183ED98E00E94CC720C1505
:10F080001D0539F785CF2C9A08952C9808951F9364
:10F09000CF93DF93182F60E270E00E94BF1CC82F4F
:10F0A00061E270E0812F0E94BF1C9C2FDF91CF9105
:10F0B0001F9108958EBD00000DB407FEFDCF8EB5E3
:10F0C0000895CF92DF92EF92FF920F931F93CF9309
:10F0D000DF93EC017A018B016C01C40ED51ECC15B7
:10F0E000DD05A9F00E9445788FE00E945A788D2FA7
:10F0F0000E945A788C2F0E945A78219680E00E94B4
:10F100005A78F80181938F010E944378E8CFC701B4
:10F11000DF91CF911F910F91FF90EF90DF90CF90F3
:10F120000895CF92DF92EF92FF920F931F93CF93A8
:10F13000DF93EC017A018B016C01C40ED51ECC1556
:10F14000DD05A1F00E94457880EF0E945A788D2F4E
:10F150000E945A788C2F0E945A782196F80181914A
:10F160008F010E945A780E944378E9CFC701DF914E
:10F17000CF911F910F91FF90EF90DF90CF90089566
:10F180001F93CF93DF93D82F192FC62F0E94457856
:10F1900080EF0E945A78812F0E945A788D2F0E940A
:10F1A0005A788C2F0E945A780E94437881E0DF9130
:10F1B000CF911F910895EF92FF920F931F93CF93DA
:10F1C000C82F7B0180E590E00E94968E68E270E097
:10F1D0008C2F0E94BF1C082F69E270E08C2F0E94C8
:10F1E000BF1C282F302FB90121E030E0A7018C2F60
:10F1F0000E94058F0E94371D81E090E0CF911F9102
:10F200000F91FF90EF900895CF93DF931F92CDB7AA
:10F21000DEB7FC01218D328D8FEF9FEF232B41F064
:10F22000BE016F5F7F4F808D0E94DB78898190E007
:10F230000F90DF91CF910895FF920F931F93CF937B
:10F24000DF93F82E80E590E00E94968E10E000E0BB
:10F250008F2D0E94A66DEC01892B21F08F2D0E942D
:10F26000A66D8C01C017D10799F70E94371DCE01FA
:10F27000DF91CF911F910F91FF900895AF92BF92B0
:10F28000CF92DF92EF92FF921F93CF93DF93182FCD
:10F290006B017A0180E590E00E94968EB12CA12C42
:10F2A000812F0E94A66DEC01892B21F0812F0E94F5
:10F2B000A66D5C01CA15DB0599F72097F9F463E0A8
:10F2C00070E0812F0E94BF1C843159F0882349F0DF
:10F2D000C1E0D0E08C3111F4D0E0C0E0D195C1950F
:10F2E000D1090E94371DCE01DF91CF911F91FF9070
:10F2F000EF90DF90CF90BF90AF900895EC16FD0691
:10F300000CF4E7011C161D0664F768E270E0812F1B
:10F310000E94BF1CE82E69E270E0812F0E94BF1C92
:10F32000282F3E2D79019E01A601B701812F0E9451
:10F33000058FEC0EFD1E4F2D68E270E0812F0E94BC
:10F34000B51C4E2D69E270E0812F0E94B51C60E46F
:10F3500070E0812F0E94F58EC4CFCF93DF93FC0124
:10F36000218D328D2115310529F48FEF9FEFDF912B
:10F37000CF910895EC01808D4217530708F0A90141
:10F380000E943E791816190684F7298D3A8D281B9C
:10F39000390B3A8F298FEBCF0F931F93CF93DF93C6
:10F3A0001F92CDB7DEB7FC01218D328D232B41F4A6
:10F3B0008FEF9FEF0F90DF91CF911F910F910895E5
:10F3C0008C0141E050E0BE016F5F7F4FFC01808DFA
:10F3D0000E943E79181619065CF7F801818D928D0E
:10F3E0000197928F818F898190E0E4CF0F931F93D3
:10F3F000CF93DF9300D000D01F921F92CDB7DEB71E
:10F400008C01D80159968D919C915A97892B41F086
:10F41000ED91FC910284F385E02DC8011995F1CF9F
:10F42000F801808D0E941C7918161906B4F548E081
:10F4300050E0BE016F5F7F4FD80158968C910E94BB
:10F440003E7918161906F4F4D801509684E0FE01AE
:10F45000319601900D928A95E1F78D8190E0982F79
:10F4600088272E81820F911DF801958B848B8F81C7
:10F47000282F30E0322F22278885820F932F911D6D
:10F48000928F818F28960FB6F894DEBF0FBECDBF46
:10F49000DF91CF911F910F91089590E080E0F2CF1E
:10F4A0004F925F926F927F928F929F92AF92BF9294
:10F4B000CF92DF92EF92FF920F931F93CF93DF9340
:10F4C000CDB7DEB763970FB6F894DEBF0FBECDBFE2
:10F4D0007C016B013A01FB0120E090E080E06AE0F2
:10F4E0003191332309F461C040ED430F4A3008F0F5
:10F4F0004DC0689FA001699F500D1124CA01C0979B
:10F50000830F911D37FD9A958F3F910549F340F385
:10F51000F701428153816481758180912708909120
:10F520002808A0912908B0912A08481759076A07A6
:10F530007B0709F42EC28701085F1F4F0E946F945A
:10F540006F7077277C5FC8010E941714813009F023
:10F5500025C285EA93E09A838983F70182819381AA
:10F56000A481B5818B839C83AD83BE8345E350E04A
:10F57000BE016F5F7F4FC8010E94F16D892BA9F515
:10F58000D12CC12CC8010E94021417C03E3209F0D0
:10F59000BFCF233009F4BCCFD301A20FB11D129607
:10F5A0008C932F5F90E080E09BCF233009F0B0CFA9
:10F5B000F3018583CC24C394D12CC60163960FB686
:10F5C000F894DEBF0FBECDBFDF91CF911F910F9199
:10F5D000FF90EF90DF90CF90BF90AF909F908F9073
:10F5E0007F906F905F904F9008950E946F94F70105
:10F5F000778366837627672776277A83698342E055
:10F6000050E0BE016F5F7F4FC8010E94276E81E00E
:10F6100090E09E878D8742E050E0BE01635F7F4FA0
:10F62000C8010E94276E80E091E09E878D8742E0AE
:10F6300050E0BE01635F7F4FC8010E94276E1E86A7
:10F640001D8642E050E0BE01635F7F4FC8010E940B
:10F65000276E42E050E0BE01635F7F4FC8010E9409
:10F66000276E42E050E0BE01635F7F4FC8010E94F9
:10F67000276E5601F6018081882301F16501F601AC
:10F6800081912F01882311F08E32B1F446018A183E
:10F690009B081814190474F48F8641E050E0BE01F1
:10F6A000615F7F4FC8010E94276EA401B501C801A8
:10F6B0000E94276E5201DECF6201E1CF1F8641E03A
:10F6C00050E0BE01615F7F4FC8010E94276EC12CD0
:10F6D000DD24D394DE86CD8642E050E0BE01635F38
:10F6E0007F4FC8010E94276EDE86CD8642E050E043
:10F6F000BE01635F7F4FC8010E94276EC8010E9450
:10F70000B96D892B09F43CCFF3E0AF2EB12C230166
:10F7100022E0420E511CEEC0F70142815381648108
:10F720007581808D918DA28DB38D481759076A0719
:10F730007B0709F024C1848D958DC59709F01FC101
:10F7400081A192A15DEFC52EDD24DA940C970CF413
:10F75000C5C04CE050E0BE016F5F7F4FC8010E9402
:10F76000AD798B819C819827892798279A8B898BE3
:10F7700029813A81322723273227F7014681578191
:10F780004217530709F000C197FFFEC08F709270B7
:10F790003BEFC32EDD24DA94892B09F09FC06F80E4
:10F7A00078847624672476242AEFC22EDD24DA9426
:10F7B0006114710409F492C0D12CC12C8D819E81F9
:10F7C000982789279827C816D90640F541E050E0C8
:10F7D000BE01635F7F4FC8010E94AD798D8588238C
:10F7E00051F08D859FEF980F9D87882321F0C801E8
:10F7F0000E94CC79F6CF8D858111E8CFC8010E9497
:10F80000CC79C8010E94CC79C8010E94CC79C8018A
:10F810000E94CC79FFEFCF1ADF0AD0CF912C812C38
:10F8200041E050E0BE016D5E7F4FC8010E94AD799E
:10F830008B89982F907C61F4882389F08B899FEFC6
:10F84000980F9B8B882341F0C8010E94CC79F6CF9A
:10F85000C8010E94CC791B8A8B898111E1CF42E0DB
:10F8600050E0BE01615F7F4FC8010E94AD7942E068
:10F8700050E0BE01635F7F4FC8010E94AD79C801AF
:10F880000E94CC79C8010E94CC79C8010E94CC7931
:10F89000C8010E94CC7942E050E0BE016F5E7F4F0C
:10F8A000C8010E94AD798F8598898115914009F032
:10F8B00040C0CD84DE84DC24CD24DC2481E0C81665
:10F8C000D104B9F589899A898115944009F04EC00F
:10F8D00044E050E0B201C8010E94AD790E94125884
:10F8E00081E0A81AB10809F44DCEFFEFCF16DF066C
:10F8F00009F048CE0E946F943B014C01C8010E9460
:10F90000F679181619060CF407CF0E946F94661941
:10F91000770988099909613A7F408105910558F571
:10F920000E94125861E070E080E090E00E942A920C
:10F93000E5CFD12CC12C89899A89982789279827C6
:10F94000C816D90638F4C8010E94CC79FFEFCF1A47
:10F95000DF0AF1CF2FEF821A920A6814790409F0B6
:10F960005FCF96EFC92EDD24DA94B8CFE7EFCE2E25
:10F97000DD24DA94B3CFCC24CA94DC2CAFCF6EEF65
:10F98000C62EDD24DA94AACF4CEFC42EDD24DA94FF
:10F99000A5CF8EEFC82EDD24DA940FCED12CC12C4A
:10F9A0000CCE2F923F924F925F926F927F928F92E6
:10F9B0009F92AF92BF92DF92EF92FF920F931F93AD
:10F9C000CF93DF93CDB7DEB7E4970FB6F894DEBFE1
:10F9D0000FBECDBF7C014A015B0119010E946F94EB
:10F9E0002B013C0187010D5B1F4FC8010E94F67976
:10F9F000181619069CF00E946F94641975098609FF
:10FA0000970986169706A806B90608F488C162E326
:10FA100070E080E090E00E942A92E7CF42E250E05E
:10FA2000BE016F5F7F4FC8010E94AD79898182302E
:10FA3000D1F0D12C8D2DE4960FB6F894DEBF0FBE19
:10FA4000CDBFDF91CF911F910F91FF90EF90DF908D
:10FA5000BF90AF909F908F907F906F905F904F90EE
:10FA60003F902F900895F8018489958983349105FA
:10FA700001F76D817E818F8198850E94C0C12B0125
:10FA80003C01F101408251826282738246E050E083
:10FA9000B701685F7F4FCE014D960E94C8C5892B84
:10FAA00041F6F70180819181A281B3814816590600
:10FAB0006A067B0608F4BDCF84819581A681B78153
:10FAC00084159505A605B70508F4B3CF89899A89E9
:10FAD000AB89BC8986879787A08BB18B8EECA82ECB
:10FAE000B12CC8010E94CC79F1E0AF1AB108C9F776
:10FAF000D12CC70182969AA789A7F701B696FCA7D1
:10FB0000EBA708969EA78DA73C974F01899698ABC7
:10FB10008FA73897FAABE9AB1701F6E12F0E311C2E
:10FB2000C5979CAB8BABF801818D928D1816190689
:10FB30000CF080CFC8010E94CC798333910509F481
:10FB4000D4C0A4F58130910509F474C074F4892BF4
:10FB500051F3C8010E94CC79B82EBA94FFEFBF16BA
:10FB600011F3C8010E94CC79F8CF8330910509F4D4
:10FB70006CC0069771F7C8010E94CC79A82E44E0AA
:10FB800050E06BA97CA9C8010E94AD79712C612C51
:10FB9000EA2DE450FF0B5F016A147B0424F6C801D0
:10FBA0000E94CC79FFEF6F1A7F0AF6CF8A33910556
:10FBB00009F46FC074F585339105A1F1C69749F634
:10FBC000C8010E94CC79B82EF701828D811109C03D
:10FBD000838D811106C0848D811103C0858D88239A
:10FBE000A1F0EFA5F8A94080518062807380B40134
:10FBF000CE0183960E94F5738DA19EA1AFA1B8A5F9
:10FC000084159505A605B705D9F544E050E0B40183
:10FC100018C08B33910509F452C08F3F910509F448
:10FC200082CF97CFC8010E94CC79C8010E94CC79BD
:10FC3000D82E79CFC8010E94CC7944E050E069A960
:10FC40007AA9C8010E94AD796ECFC8010E94CC7913
:10FC5000A82E44E050E0B101C8010E94AD79712C9A
:10FC6000612C8A2D8450990B5C016A147B040CF082
:10FC70005ACFC8010E94CC799FEF691A790AF5CF53
:10FC8000BA94FFEFBF1609F44ECFC8010E94CC7999
:10FC9000F7CFC8010E94CC7944E050E06BA57CA569
:10FCA000C8010E94AD79F70166A177A180A591A551
:10FCB0000E94C0C166A377A380A791A734CFC801D3
:10FCC0000E94CC7944E050E06DA57EA5C8010E9459
:10FCD000AD79F70162A573A584A595A50E94C0C161
:10FCE00062A773A784A795A71ECFC8010E94CC79ED
:10FCF00044E050E069A57AA5C8010E94AD79F701FA
:10FD000062A173A184A195A10E94C0C162A373A343
:10FD100084A395A366A777A780AB91AB04CFDD241E
:10FD2000DA9488CE2F923F924F925F926F927F9299
:10FD30008F929F92AF92BF92CF92DF92EF92FF92FB
:10FD40000F931F93CF93DF9300D000D0CDB7DEB7D2
:10FD50008C010E94BCB62FEC37E040E050E00E94DE
:10FD60004FC1DC01CB010196A11DB11DF8018483B7
:10FD70009583A683B78380839183A283B38358013D
:10FD8000F3E4AF0EB11CC5010E94021464E470E0FC
:10FD9000C5010E941714882309F445C10E946F947D
:10FDA0002B013C01480182E4880E911C48EEC42ED0
:10FDB00043E0D42EE12CF12C52E0252E1E821D8230
:10FDC000D4018C918330B1F1811166C0F801848136
:10FDD0009581A681B7810196A11DB11D848395836C
:10FDE000A683B7830E946F946419750986099709E1
:10FDF000A70196010E942DC1A90161E0C8010E94DE
:10FE00005F6E81E0D4018C938D819E810197C1F258
:10FE10000E946F946419750986099709D801D696CE
:10FE20002D913D914D915C91D99726173707480741
:10FE3000590720F6C5010E940214F80184819581BA
:10FE4000A681B7810196A11DB11D84839583A683E8
:10FE5000B7830E946F94F801FE966083718382835A
:10FE600093838D819E8126960FB6F894DEBF0FBED8
:10FE7000CDBFDF91CF911F910F91FF90EF90DF9059
:10FE8000CF90BF90AF909F908F907F906F905F903A
:10FE90004F903F902F9008958430F1F4F8018481C1
:10FEA0009581A681B7810196A11DB11D848395839B
:10FEB000A683B7830E946F94641975098609970910
:10FEC000A70196010E942DC1A90163E0C8010E940B
:10FED0005F6ED4012C9298CF813051F5F80142AD7C
:10FEE00053AD64AD75AD9E012F5F3F4FC8010E94B9
:10FEF000D17C382EF2E08F1390C089819A81AB813A
:10FF0000BC81F80184839583A683B7830E946F9494
:10FF10006419750986099709A70196010E942DC1E8
:10FF2000A90163E0C8010E945F6ED4013C926CCFCE
:10FF3000823009F069CFF80142AD53AD64AD75ADC3
:10FF40009E012F5F3F4FC8010E94D17C382EF5E003
:10FF50008F135DC0E3E0D401EC93F80182A193A17B
:10FF6000A4A1B5A1892B8A2B8B2B41F484E893E0C3
:10FF7000A0E0B0E082A393A3A4A3B5A3F80186A157
:10FF800097A1A0A5B1A5892B8A2B8B2B61F482A107
:10FF900093A1A4A1B5A1B695A7959795879586A39A
:10FFA00097A3A0A7B1A7F80182A593A5A4A5B5A57D
:10FFB000892B8A2B8B2BA9F482A193A1A4A1B5A193
:10FFC000AC01BD0123E076956795579547952A9535
:10FFD000D1F7841B950BA60BB70B82A793A7A4A7F9
:10FFE000B5A7F80186A197A1A0A5B1A586A797A757
:10FFF000A0ABB1AB82A593A5A4A5B5A582AB93ABED
:020000021000EC
:10000000A4ABB5AB81E090E09E838D83FDCE96E0FE
:10001000891303C0D4011C92F7CEBFEF3B12F4CE7C
:10002000F4011082F1CE1E821D821BCFCF93C82F08
:1000300080E590E00E94968E60E170E08C2F0E9437
:10004000F58E4FEF62E070E08C2F0E94B51CCF91CF
:100050000C94371DFF920F931F93CF93DF93C82FFC
:10006000D62F8A01F22E0E94168080E590E00E9431
:10007000968E4D2F4F2970E060E08C2F0E94B51CAA
:1000800001151105D1F0412F64E070E08C2F0E9422
:10009000B51C402F65E070E08C2F0E94B51C61E01C
:1000A00070E08C2F0E94F58E0E94371D81E0DF9159
:1000B000CF911F910F91FF90089500919E0610918E
:1000C0009F060F5F1F4F10939F0600939E06DBCF86
:1000D000BF92CF92DF92EF92FF920F931F93CF9335
:1000E000DF9300D000D0CDB7DEB7FC01208D2430E7
:1000F00009F05DC06A017B018C01B12C63E070E006
:100100008B2D0E94BF1C81114AC0F801B08EF801EE
:10011000808D843009F44BC096E0ECE9F2E0DE011A
:10012000119601900D929A95E1F7F70193819F77CF
:100130009C8394819D8395819E83B7016E5F7F4FE1
:100140000E94EE1CB601F801808D0E94DD1CF801B2
:10015000808D90E0982F882746E050E0BE016F5FC9
:100160007F4F8A5F9B4F0E949178F801128E118E0B
:1001700020E8A60162E0808D0E942A8081E0269618
:100180000FB6F894DEBF0FBECDBFDF91CF911F91A8
:100190000F91FF90EF90DF90CF90BF90089588313E
:1001A00009F4B3CFB394F4E0BF12A8CFB0CF80E08E
:1001B000E6CFCF93C82F80E590E00E94968E63E053
:1001C00070E08C2F0E94BF1CC82F0E94371D8C2FFF
:1001D000CF9108958F7099278230910518F002977A
:1001E00061F008958091790890917A08DC01ED9191
:1001F000FC910680F781E02D199480917B08909105
:100200007C08DC01ED91FC91008CF18DE02D1995BD
:1002100080917B0890917C08DC01ED91FC91048831
:10022000F589E02DE9CF8F929F92AF92BF92CF9246
:10023000DF92EF92FF92CF93DF93EC014A015B01D3
:10024000C12CD12C7601CE010E94FF1C882399F08D
:10025000C814D904EA04FB0474F4CE010E949B1470
:10026000892B89F38FEFC81AD80AE80AF80ACE0159
:100270000E948114E8CFDF91CF91FF90EF90DF9043
:10028000CF90BF90AF909F908F9008952F923F9204
:100290004F925F926F927F928F929F92AF92BF9296
:1002A000CF92DF92EF92FF920F931F93CF93DF9342
:1002B00000D000D01F921F92CDB7DEB78C016B012A
:1002C0000E947D76019619F48FEF9FEF1DC0D80133
:1002D000ED91FC910284F385E02DC80119957C0114
:1002E0008F3F980789F3D801ED91FC910684F7853B
:1002F000E02D682FC8011995B2E2EB16F104E9F47C
:10030000B601C8010E949A7628960FB6F894DEBF0F
:100310000FBECDBFDF91CF911F910F91FF90EF9056
:10032000DF90CF90BF90AF909F908F907F906F9015
:100330005F904F903F902F900895EDE2EE16F104FC
:1003400029F0C701C0970A9708F043C1D801ED9181
:10035000FC910284F385E02DC80119957C018F3F43
:10036000980709F4B1CF8D9799F5D801ED91FC91DB
:100370000284F385E02DC80119957C01019609F4EA
:10038000A3CFEFEFFFEFF887EF83C701C097812C72
:10039000912C54010A9708F5AAE0B0E0A501940158
:1003A0000E946EC130E3E31AF1084701FF0CAA086E
:1003B000BB08860E971EA81EB91ED801ED91FC91B0
:1003C0000284F385E02DC80119957C01C097E2CF26
:1003D00021E030E038872F83D8CFBEE2EB16F1045E
:1003E00001F1C7018F7D85349105D9F0AF81B885C2
:1003F000A50194010E9479C1F60161877287838704
:1004000094878085807F82608087D801ED91FC9100
:100410000684F785E02D6E2DC801199590E080E0E7
:1004200073CFC501B4010E94EABF2B013C01312CFE
:10043000212CFEE2EF16F10499F5D801ED91FC9123
:100440000284F385E02DC80119957C01312C212C03
:1004500020E030E040E251E4C301B2010E9449C013
:100460004B015C01B70160537109072E000C880B2A
:10047000990B0E94EABFA50194010E94D7C12B01EC
:100480003C01B1E02B1A3108D801ED91FC910284B6
:10049000F385E02DC80119957C01C0970A97C0F239
:1004A000C7018F7D8534910509F040C0D801ED91D9
:1004B000FC910284F385E02DC80119957C01D801D7
:1004C000ED91FC918B32910519F50284F385E02DB5
:1004D000C80119957C01E1E0EE83B12CA12C8AE0E2
:1004E000982ED801ED91FC91C701C0978A309105F3
:1004F00008F59A9C90019B9C300D11245C01A20E82
:10050000B31E0284F385E02DC80119957C01E9CF63
:100510008D9749F40284F385E02DC80119957C017B
:100520003FEF3E83DACF81E08E83D7CFB1E0BE8349
:10053000B12CA12CEF81F885BF01FF0F880B990B1F
:100540000E94EABFA30192010E9449C02B013C0115
:10055000B501BB0C880B990B0E94EABF4B015C01F3
:10056000FE816F2FFF0F770B880B990B0E94EABF5C
:100570009B01AC01C501B4010E9449C04B015C0163
:10058000B101330C880B990B0E94EABF9B01AC01AF
:10059000C501B4010E94D7C19B01AC0160E070E0CD
:1005A00080E291E40E94F0C29B01AC01C301B20160
:1005B0000E9449C0D60119966D937D938D939C93AB
:1005C0001C9718968C911897807F836018968C934F
:1005D0001CCFBBE5EB16F10409F062C0D801ED9128
:1005E000FC910284F385E02DC80119958B359105A6
:1005F00009F06ACEF6018085807F85608087C8011A
:100600000E947D76D801ED91FC910284F385E02D66
:10061000C80119958D35910509F400CFD801ED91E8
:10062000FC910684F785E02D682FC8011995BB243D
:10063000BA940E945A777C01009709F445CEBB20FA
:1006400031F1F60197838683C8010E947D76B70158
:10065000C8010E944681892B09F036CEC8010E944C
:100660007D76D801ED91FC910284F385E02DC801DF
:100670001995B12C47018C329105D9F221E030E077
:100680008D35910509F08DC030E020E08AC0D4019D
:1006900013969C938E931297FC0195828482D4CFFB
:1006A000BBE7EB16F10409F08AC0D801ED91FC918B
:1006B0000284F385E02DC80119958B37910509F067
:1006C00003CEF6018085807F86608087C8010E9406
:1006D0007D76D801ED91FC910284F385E02DC8016F
:1006E00019958D37910509F499CED801ED91FC91BA
:1006F0000684F785E02D682FC801199599249A94EE
:100700000E945A777C01009709F4DECD992009F404
:100710004DC0F60197838683C8010E947D76B7019C
:10072000C8010E949A76019609F4CECDC8010E94B4
:100730007D76D70119968D919C911A9711969C936D
:100740008E931A961C921E921997D801ED91FC91E6
:100750000284F385E02DC8011995CA9709F0B4CD3C
:10076000C8010E947D76B701C8010E9446810196AA
:1007700009F4AACDC8010E947D76D801ED91FC91C3
:100780000284F385E02DC8011995912C57018C3214
:10079000910509F4B5CF21E030E08D37910509F4DA
:1007A00073CF88279927821B930BAECDD501139663
:1007B0009C938E931297FC01B582A482ADCFBEE6C6
:1007C000EB16F10421F519821A821B821C82D801D2
:1007D000ED91FC910484F585E02D44E050E0BE01EC
:1007E0006F5F7F4FC8011995049709F06DCD44E004
:1007F00050E06DE175E0CE0101960E9439C6009788
:1008000009F062CDF6012085207F20877DCDF6E6B8
:10081000EF16F10441F59E012F5F3F4F790185E00E
:10082000D9011D928A95E9F7D801ED91FC910484D4
:10083000F585E02D45E050E0B901C801199505970F
:1008400009F042CD45E050E067E275E0C7010E9443
:1008500039C6009709F038CDF6012085207F216048
:100860002087118651CDF4E7EF16F10409F02CCD65
:1008700019821A821B821C82D801ED91FC9104849A
:10088000F585E02D44E050E0BE016F5F7F4FC80169
:100890001995049709F018CD44E050E062E275E044
:1008A000CE0101960E9439C6009709F00DCDF601E0
:1008B0002085207F2160208721E0218725CD0F938F
:1008C0001F93CF93DF938B01FC01C681D7812097C3
:1008D00059F0B801888199810E94F0C5892B21F0D7
:1008E0000A80DB81C02DF3CFCE01DF91CF911F9124
:1008F0000F9108958091430890914408009711F456
:1009000080E02FC0DC01ED91FC910688F789E02D95
:100910001995209166083091670881111FC0232B1B
:1009200079F78DEF9FEF9093670880936608809129
:10093000430890914408DC01ED91FC910680F78119
:10094000E02D19958091430890914408DC01ED91C8
:10095000FC910488F589E02D1995D2CF81E0232BF5
:1009600079F60895CF93DF93EC01FA013296E60F02
:10097000F71FDC019D012C1B3D0BCF01861B970B44
:100980004D91442311F04193F5CFAC01421B530B21
:10099000640F751FFB013297308361507109FB01B1
:1009A0002083DF91CF910895FC0186819781009784
:1009B00039F0662329F06150FC0182819381F7CFE1
:1009C0000895CF92DF92EF92FF92DC011196EC91A5
:1009D0001197E295EF70EC3098F4F0E08827EC5036
:1009E000FB478F4F0C94B8C157851A851A8500852F
:1009F000008500853D851E85008500850785078566
:100A00008FEF9FEFFF90EF90DF90CF9008951496B7
:100A10008D919D910D90BC91A02DB7FD48C08F3F49
:100A20009105A105B10571F36CF38FEF90E0A0E0A3
:100A3000B0E0E8CF14968C9190E0E4CF1496CD907E
:100A4000DD90ED90FC90179720E030E0A901C70100
:100A5000B6010E94E3BF87FD2AC020E030E04FE7E7
:100A600053E4C701B6010E94EBC218161CF1C7017E
:100A7000B6010E94B5C2CB01C5CF14966D917D9190
:100A80008D919C911797673F2FEF7207820792070E
:100A900074F061152AE07207810591055CF42AE083
:100AA00030E040E050E00E944FC1C901ABCF90E080
:100AB00080E0A8CF8FEF90E0A5CFEF92FF920F9349
:100AC0001F93CF93DF937C018B01D0E0C0E0C7017F
:100AD0000E94177297FD07C0F80181938F0121963C
:100AE000C430D105A1F7CE01DF91CF911F910F91B5
:100AF000FF90EF9008950F931F93CF93DF93CDB79F
:100B0000DEB762970FB6F894DEBF0FBECDBF8C0183
:100B1000CB01F80111821082138212821582148295
:100B200040E1BE016F5F7F4F0E94FFB8BE016F5F63
:100B30007F4FC8010E94977162960FB6F894DEBF8E
:100B40000FBECDBFDF91CF911F910F910895CF932D
:100B5000DF93A0919C08B0919D08109709F444C0C0
:100B600052961C921E92519754961C921E92539725
:100B700084E890E01D969C938E931C971E961C9281
:100B80001E9780E090E350969C938E931F97ED9173
:100B9000FC9111970088F189E02D70E060E0CD01B3
:100BA0001995CEEBD2E080919C0890919D08DC01D4
:100BB000ED91FC91B2E0C23CDB07C1F00284F38509
:100BC000E02D19952991022E000C330B8217930703
:100BD00051F380919C0890919D08DC01ED91FC916E
:100BE0000488F589E02D199580E005C00488F58911
:100BF000E02D199581E0DF91CF910895AF92BF92DA
:100C0000CF92DF92EF92FF920F931F93CF93DF93D8
:100C10005C017B018B01040F151FEB016E01CE18E7
:100C2000DF08C017D10741F0C5010E9417721816DE
:100C3000190614F48993F2CFC601DF91CF911F9169
:100C40000F91FF90EF90DF90CF90BF90AF900895FD
:100C5000CF93DF9320919C0830919D08232B11F4B2
:100C600080E056C0EC010E94A7858823C9F3FE01ED
:100C700001900020E9F73197EC1BFD0B709780F78E
:100C8000A0919C08B0919D0852961C921E9251977B
:100C900054961C921E92539784E890E01D969C9364
:100CA0008E931C971E961C921E9780E090E35096A0
:100CB0009C938E931F97ED91FC9111970088F18979
:100CC000E02D60E470E0CD011995BE0180919C0893
:100CD00090919D080E94597380919C0890919D0865
:100CE000DC01ED91FC910190F081E02D60E019951F
:100CF000EC0180919C0890919D08DC01ED91FC91A4
:100D00000488F589E02D199581E0CD2B09F4A8CF51
:100D1000DF91CF910895CF93DF9320919C0830917C
:100D20009D08232B11F480E056C0EC010E94A7859A
:100D30008823C9F3FE0101900020E9F73197EC1BED
:100D4000FD0B709780F7A0919C08B0919D0852967A
:100D50001C921E92519754961C921E92539784E8AF
:100D600090E01D969C938E931C971E961C921E9746
:100D700080E090E350969C938E931F97ED91FC91A9
:100D800011970088F189E02D60E570E0CD0119959B
:100D9000BE0180919C0890919D080E94597380919A
:100DA0009C0890919D08DC01ED91FC910190F081EF
:100DB000E02D60E01995EC0180919C0890919D08D0
:100DC000DC01ED91FC910488F589E02D199581E015
:100DD000CD2B09F4A8CFDF91CF9108950F931F93E6
:100DE000CF93DF9300D01F92CDB7DEB7FC01828195
:100DF0009381A481B58189839A83AB83BC838091DD
:100E00009C0890919D08892B11F480E049C00E94B4
:100E1000A7858823D1F3A0919C08B0919D08529694
:100E20001C921E92519754961C921E92539784E8DE
:100E300090E01D969C938E931C971E961C921E9775
:100E400080E090E350969C938E931F97ED91FC91D8
:100E500011970088F189E02D60E170E0CD011995CE
:100E600080919C0890919D08DC01ED91FC9102809D
:100E7000F381E02D44E050E0BE016F5F7F4F199594
:100E80008C0180919C0890919D08DC01ED91FC9172
:100E90000488F589E02D199581E0012B09F4B5CF7F
:100EA0000F900F900F900F90DF91CF911F910F91A6
:100EB00008950F931F93CF93DF9300D01F92CDB768
:100EC000DEB7FC0182819381A481B58189839A83F5
:100ED000AB83BC8380919C0890919D08892B11F471
:100EE00080E049C00E94A7858823D1F3A0919C0887
:100EF000B0919D0852961C921E92519754961C9246
:100F00001E92539784E890E01D969C938E931C97B5
:100F10001E961C921E9780E090E350969C938E93B1
:100F20001F97ED91FC9111970088F189E02D6CE1FC
:100F300070E0CD01199580919C0890919D08DC018D
:100F4000ED91FC910280F381E02D44E050E0BE0180
:100F50006F5F7F4F19958C0180919C0890919D083F
:100F6000DC01ED91FC910488F589E02D199581E073
:100F7000012B09F4B5CF0F900F900F900F90DF91D8
:100F8000CF911F910F9108950F931F93CF93DF93EC
:100F900000D01F92CDB7DEB7FC0182819381A4817E
:100FA000B58189839A83AB83BC8380919C0890919F
:100FB0009D08892B11F480E049C00E94A7858823F1
:100FC000D1F3A0919C08B0919D0852961C921E925C
:100FD000519754961C921E92539784E890E01D9668
:100FE0009C938E931C971E961C921E9780E090E314
:100FF00050969C938E931F97ED91FC9111970088CA
:10100000F189E02D64E170E0CD01199580919C0893
:1010100090919D08DC01ED91FC910280F381E02D1F
:1010200044E050E0BE016F5F7F4F19958C018091C5
:101030009C0890919D08DC01ED91FC910488F58954
:10104000E02D199581E0012B09F4B5CF0F900F9099
:101050000F900F90DF91CF911F910F9108950F93F3
:101060001F93CF93DF9300D01F92CDB7DEB7FC0163
:1010700082819381A481B58189839A83AB83BC8368
:1010800080919C0890919D08892B11F480E049C0C3
:101090000E94A7858823D1F3A0919C08B0919D0858
:1010A00052961C921E92519754961C921E925397E0
:1010B00084E890E01D969C938E931C971E961C923C
:1010C0001E9780E090E350969C938E931F97ED912E
:1010D000FC9111970088F189E02D68E170E0CD0165
:1010E000199580919C0890919D08DC01ED91FC91EF
:1010F0000280F381E02D44E050E0BE016F5F7F4F3E
:1011000019958C0180919C0890919D08DC01ED91CE
:10111000FC910488F589E02D199581E0012B09F4F3
:10112000B5CF0F900F900F900F90DF91CF911F913F
:101130000F910895CF93DF9300D01F92CDB7DEB704
:1011400019821A821B821C8287E7898380919C08FE
:1011500090919D08892BE9F10E94A7858823C9F108
:10116000A0919C08B0919D0852961C921E92519796
:1011700054961C921E92539784E890E01D969C937F
:101180008E931C971E961C921E9780E090E35096BB
:101190009C938E931F97ED91FC9111970088F18994
:1011A000E02D6CE070E0CD011995BE016F5F7F4FBF
:1011B00080919C0890919D080E945D8580919C087B
:1011C00090919D08DC01ED91FC910488F589E02D5A
:1011D000199569817A818B819C810F900F900F9076
:1011E0000F90DF91CF9108950F931F93CF93DF93CB
:1011F00000D01F92CDB7DEB769837A838B839C833F
:1012000080919C0890919D08892B11F480E049C041
:101210000E94A7858823D1F3A0919C08B0919D08D6
:1012200052961C921E92519754961C921E9253975E
:1012300084E890E01D969C938E931C971E961C92BA
:101240001E9780E090E350969C938E931F97ED91AC
:10125000FC9111970088F189E02D6CE070E0CD01E0
:10126000199580919C0890919D08DC01ED91FC916D
:101270000280F381E02D44E050E0BE016F5F7F4FBC
:1012800019958C0180919C0890919D08DC01ED914D
:10129000FC910488F589E02D199581E0012B09F472
:1012A000B5CF0F900F900F900F90DF91CF911F91BE
:1012B0000F910895CF93C82F0E949A88677FC0FF2F
:1012C0006860CF910C94F488CF93C82F0E949A88BD
:1012D000C770687F6C2BCF910C94F488CF93C82F84
:1012E0000E949A88C770C295C07F6F786C2BCF918F
:1012F0000C94F48861157105C1F0DC011696ED912E
:10130000FC911797309731F417967C936E9316974C
:101310000895FC01828193810097D9F773836283DA
:10132000DB011596FC93EE93149708952AE00C9434
:101330007C72462F50E070E060E02AE00C947C72F2
:10134000AB01770F660B770B2AE030E00C94D37279
:10135000DC011696ED91FC9180E0309729F08F5FCB
:101360000280F381E02DF9CF0895CF93DF93FC0144
:10137000C281D3812097C1F088858F70823029F493
:1013800089859A85DF91CF910895853069F4CE01E2
:101390000E94A889882341F060E0CE010E94D48495
:1013A000FC0181859285EECF90E080E0EBCFDF926B
:1013B000EF92FF920F931F93CF93DF93EC017B018A
:1013C00040E052E00E941E2ED82E811171C063E1D0
:1013D0007EE180E799E00E94BF73D70119968D9155
:1013E0009C91009709F441C0DC01ED91FC91028CC5
:1013F000F38DE02D19958C0180E00231110520F468
:10140000F801E455FD4F8081982F9295907F898156
:101410008F70892B898368E07EE180E799E00E94E4
:10142000BF73B80180E799E00E94A08960E07EE187
:1014300080E799E00E94BF73698162956F7080E7D1
:1014400099E00E94998980E799E00E94C872898199
:1014500082958F70843068F4823098F58130B9F1CC
:101460001C821D821E821F8215C0F701008510E0BC
:10147000C3CF883039F0893099F780E090E0A6E951
:10148000B2E404C080E090E0A0EAB1E48C839D83E4
:10149000AE83BF8340E052E0B701CE010E94AC2D85
:1014A000CE010E94C02C60E07AE0C7010E949F3606
:1014B0008D2DDF91CF911F910F91FF90EF90DF90D5
:1014C000089584E68E838F818E7F8F831D828FEFB8
:1014D0008C83E0CF6F927F929F92AF92BF92CF9218
:1014E000DF92EF92FF920F931F93CF93DF93CDB7CD
:1014F000DEB7E4970FB6F894DEBF0FBECDBF7CAB6E
:101500006BAB1AAA19AA672B09F487C2FC012385C1
:10151000222329F09C01255F3F4F3AAB29AB5C01A8
:10152000E9A9FAA93097E1F4F501E588F688E11414
:10153000F10401F510E000E0CBA8DCA83601600E54
:10154000711EF3018081882309F458C0082E000C15
:10155000990B0E94A6C5F30180830F5F1F4FECCF4C
:101560008081882309F3CE01C1960E9469347C01F1
:10157000892BD1F2FEE0EF16F104E1F62BA93CA98C
:1015800019861A861B861C861D861E861F86188A4B
:101590008A858F70806C8A873E872D876EE0CE01AA
:1015A00009960E94FC2E29833A834B835C836D83CA
:1015B0007E838F839887E9A8FAA8CC24C3940985F1
:1015C0001A852B853C854D855E856F857889C5019B
:1015D0000E940537E4960FB6F894DEBF0FBECDBF6C
:1015E000DF91CF911F910F91FF90EF90DF90CF90FF
:1015F000BF90AF909F907F906F900895C114D104D9
:1016000081F1F6018081882361F18D3209F46DC08A
:1016100090ED980F9A3008F468C008E010E0853229
:1016200011F10EEF1FEF8B37F1F007E110E083327D
:10163000D1F09BE1692E9DE1792E01E010E0C3011C
:101640000E9493B8AC01B301C6010E94ACB8892BCB
:1016500051F00F5F1F4FF9E06F0E711C093111053A
:1016600071F70FEF1FEF19A61AA61BA61CA61DA641
:101670001EA61FA618AA8AA58F708AA709A785E0AB
:10168000E816F104A9F196E0E916F10411F407E176
:1016900010E09E2C6E2DCE0189960E94FC2E29878B
:1016A0003A874B875C876D877E878F87988B01157C
:1016B0001105A9F104F50E3F1F4F0CF0AEC1CE018C
:1016C000C3960E945B25092E000CAA0BBB0B00974A
:1016D000A105B10509F4D6C02AA52F70206A2AA752
:1016E0008DA79EA7AFA7B8ABCDC010E000E0BBCFE1
:1016F00008E110E0CECF0731110509F44BC10831E4
:101700001105E9F660E0CE0189960E94232F298B0E
:101710003A8B4B8B5C8B6D8B7E8B8F8B988F19826A
:101720001A821B821C828A818F7080668A83EBA951
:10173000FCA9309709F48EC08081882309F48AC0FF
:101740006BA87CA8F3018081882359F08D3249F081
:1017500080538A3030F0FFEF6F1A7F0A7CAA6BAAA1
:10176000EFCFC3010E9417B86C016EE270E0C301B5
:101770000E940EC6009709F45AC0FC010181003393
:101780000CF455C00A330CF055C0002E000C110BA0
:10179000005311096CE270E0C3010E940EC600976D
:1017A00009F04BC01CAA1BAA0115110509F449C078
:1017B0002AE02C9DC0012D9D900D11241C141D04A8
:1017C0001CF0119501951109080F191F012E000C2D
:1017D000220B330B0D831E832F833887692DCE0197
:1017E00001960E94FC2E298F3A8F4B8F5C8F6D8F54
:1017F0007E8F8F8F98A3DA80D2948FE0D8223E011B
:10180000F1E26F0E711C10E000E08BA99CA9892BFE
:1018100029F10330110511F10F5F1F4FCE01C3965F
:101820000E945B25F301819391933F01EECF10E07D
:1018300000E0B0CF09E010E0ADCF01969CAB8BABE0
:10184000B3CF8601DD0C220B330B8A818F70806A47
:101850008A83C0CF00E010E09801BCCFFAE0EF1619
:10186000F104E9F08BE0E816F10469F199E0E9167A
:10187000F10491F5CE0101960E94452FCE01899683
:101880000E944A34E9A8FAA8CC24C39409A51AA551
:101890002BA53CA54DA55EA56FA578A998CECE0138
:1018A00001960E94452F8AA5982F92959F7039F036
:1018B000923041F7653608F064E66EA7E3CF8F708B
:1018C00080628AA7F7CFCE0101960E94452FCE01F4
:1018D00089960E948A2FD6CF81E090E0D11002C075
:1018E00090E080E0800F911F8230910589F16CF4C7
:1018F000019721F163EF7DE189EC98E00E94BF73CD
:1019000089EC98E00E94C872BDCF8330910581F1C7
:10191000049781F71BA109A1CE0101960E94452FD2
:101920008AA58F7080628AA76FA788A970FB80F94B
:1019300088AB0EA71DA76DA17EA1C9CF88E0FE01CF
:101940003196DE01999601900D928A95E1F79ACF32
:1019500019A1CE0101960E94452F8AA58F70806340
:101960008AA76FA788A970FB80F988AB1EA78ACFCA
:101970001BA109A1CE0101960E94452F8AA58F7057
:1019800080628AA76FA788A970FB80F988AB0EA731
:101990001DA778CF60E0CE0189960E94232F29A34E
:1019A0003AA34BA35CA36DA37EA38FA398A7FE01CC
:1019B00031967F0110E000E08BA99CA9892B71F082
:1019C0000430110591F00F5F1F4FCE01C3960E94A6
:1019D0005B25F701819391937F01EECF03301105D1
:1019E00089F00430110509F04DCF9F812D813B8195
:1019F00049818AA58F7080658AA74FA73EA72DA72A
:101A000098AB40CF9D812B8139818AA58F708064EE
:101A10008AA73FA72EA79DA735CF90E080E0DACD1B
:101A2000CF92DF92EF92FF920F931F93CF93DF93AA
:101A300000D000D0CDB7DEB78C016C0188E0C80EB5
:101A4000D11C30E1E32EF12CF80181918F0190E05F
:101A500024E0959587952A95E1F7092E000CAA0BAD
:101A6000BB0B89839A83AB83BC83FE82ED82BE016C
:101A70006F5F7F4F8FEB98E00E94335DF8013197E5
:101A800080818F7090E0B0E0A0E089839A83AB837F
:101A9000BC83FE82ED82BE016F5F7F4F8FEB98E0CB
:101AA0000E94335D0C151D0579F626960FB6F89445
:101AB000DEBF0FBECDBFDF91CF911F910F91FF9081
:101AC000EF90DF90CF9008954F925F926F927F9248
:101AD0008F929F92AF92BF92CF92DF92EF92FF923E
:101AE0000F931F93CF936B017C01742EAC019B016C
:101AF0000E944BC36AE875E0811126C04601570178
:101B0000E894B7F82FEF3FEF4FE75FE7C501B40167
:101B10000E944BC381110CC02FEF3FEF4FE75FE7EF
:101B2000C501B4010E94E3BF6EE875E0181664F0C9
:101B30002FEF3FEF4FE75FE4C701B6010E94EBC212
:101B40001816ACF462E975E080E799E0CF911F9137
:101B50000F91FF90EF90DF90CF90BF90AF909F904C
:101B60008F907F906F905F904F900C946D722FEFDD
:101B70003FEF4FE75FECC701B6010E94E3BF87FD6F
:101B8000E1CF20E030E0A901C701B6010E94E3BF28
:101B900010E000E087FF0AC06DE280E799E00E9454
:101BA000CC728C01F7FAF094F7F8F094C0E060E0A2
:101BB00070E080E09FE37C1641F020E030E040E2FE
:101BC00051E40E9443C2CF5FF6CFA70196010E9465
:101BD000D7C12B013C010E94BCC24B015C012AE031
:101BE000BC01A40180E799E00E947C727C01E00EB8
:101BF000F11ECC23D1F1C501B4010E94E8BF9B01C5
:101C0000AC01C301B2010E94D6C14B015C016EE27E
